:020000040800F2
:1000000000000220E1DC000827DD000829DD0008EF
:100010002BDD00082DDD00082FDD000800000000AA
:1000200000000000000000000000000031DD0008BA
:1000300033DD00080000000035DD000879450008C8
:100040003BDD00083DDD00083FDD000841DD000824
:1000500043DD000845DD000847DD000849DD0008F4
:100060004BDD00084DDD00084FDD000851DD0008C4
:1000700053DD000855DD000857DD000859DD000894
:100080005BDD00085DDD00085FDD000861DD000864
:1000900063DD000865DD000867DD00084DC300086A
:1000A0006BDD00086DDD00086FDD000871DD000804
:1000B00061BB000875DD000877DD000879DD000808
:1000C0007BDD00087DDD00087FDD000881DD0008A4
:1000D00083DD000885DD00088D45000889DD000806
:1000E0008BDD00088DDD00088FDD000891DD000844
:1000F00093DD000895DD000897DD000899DD000814
:100100009BDD0008017A00089FDD0008A1DD0008E2
:10011000A3DD0008A5DD0008A7DD0008A9DD0008B3
:10012000ABDD0008ADDD0008AFDD0008E1790008B7
:10013000B3DD0008B5DD0008B7DD0008B9DD000853
:10014000BBDD0008BDDD0008BFDD000835D30008B9
:10015000C3DD0008C5DD0008C7DD0008C9DD0008F3
:10016000CBDD0008CDDD0008CFDD0008D1DD0008C3
:10017000D3DD0008D5DD0008D7DD0008D9DD000893
:10018000DBDD0008DDDD000810B5054C237833B950
:10019000044B13B10448AFF300800123237010BD5A
:1001A00030010020000000006C250108084B10B54C
:1001B0001BB108490848AFF300800848036803B939
:1001C00010BD074B002BFBD0BDE81040184700BF07
:1001D00000000000340100206C25010830010020DF
:1001E00000000000154B002B08BF134B9D46A3F5E4
:1001F000803A00218B460F461348144A121A0EF01B
:100200003AFA0F4B002B00D098470E4B002B00D032
:1002100098470020002104000D000D48002802D05E
:100220000C48AFF300800EF045F92000290002F0E1
:10023000A3FA0DF0E3FD00BF00000800000002205B
:10024000000000000000000030010020B04201204A
:1002500000000000000000002DE980488BB0504BEA
:100260001B68002B40F0A2824E4BD3F8C4309A0793
:1002700000F198824C4B4C4A1B68002B40F0BF8128
:100280004A4B1B78002B56D1494B1A78002A52D181
:10029000484B49491878494B464C1B880B804749C5
:1002A000002832D04648464D007800282DD04548D9
:1002B0002A70C05C2270762800F02B87424A43499E
:1002C00012880888511E89B2814202D33D4D1C0A12
:1002D0006C54023A92B23C4990420A809CBF394920
:1002E0008B543B4A1278012A40F20E87022A0CD125
:1002F000384B34491B781B025A1C92B2CB5C8A5C87
:1003000003EB02232D4A9BB2138040F262529342C8
:1003100000F0A88640F2C242934200F088862E4B3D
:100320001B7803F0FF04002B00F053852B4B1B6858
:10033000002B40F08984214B294A1B8821491268EF
:10034000CC5C002A56D043F6FE42934200F08083F4
:1003500043F6FF4293424DD1224B1B68002B00F025
:100360003886214B214A1B681F49D25C0133802B00
:100370000B6008BF0023D2B208BF0B6072B6194BE6
:1003800018491B68013B0B6062B6194B18499B79F1
:10039000CA7143F001030D2A8B7100F0438629E0F6
:1003A000D0010020FC030020D00800208242012060
:1003B00083420120EE02002002090020D80800201C
:1003C000F5030020A8250020F00200208042012033
:1003D000D801002000090020010000204C0100206D
:1003E000F8030020D4080020F40800205001002069
:1003F00074420120FF2C02F27381DFE814F04A11ED
:100400004311271187118011A011DF10C210A7100E
:10041000A01089107010691062105B102D1011105F
:10042000FC0FE00FC70FC00FB90FB20F8F0F7C0F7B
:10043000750F5E0F450F3E0F370F300F040FFC0E88
:10044000E90EC10EAC0EA50E9E0E970E910E890EF2
:10045000830E7D0E770E700E690E620E4B0E430EEC
:100460002A0E0B0EF80DF20DEC0DE60DD00DC80D99
:10047000C20DA50D920D8B0D840D7D0D630D4A0DE2
:100480004A0D4A0D4A0D4A0D4A0D430D4A0D3A0DCB
:100490003A0D3A0D3A0D3A0D3A0D330D3A0D2A0D3B
:1004A0002A0D2A0D2A0D2A0D2A0D230D2A0D1A0DAB
:1004B0001A0D1A0D1A0D1A0D1A0DFF0C1A0DF60C45
:1004C000F60CF60CF60CF60CF60C060DF60CED0C14
:1004D000ED0CED0CED0CED0CED0CDD0CED0CB50C9C
:1004E000B50CB50CB50CB50CB50CAC0CB50CA30C1F
:1004F000A30CA30CA30CA30CA30C9C0CA30C940C9A
:10050000940C940C940C940C940C8E0C940C860CFF
:10051000860C860C860C860C860C800C860C780C5F
:10052000780C780C780C780C780C720C780C6A0CBF
:100530006A0C6A0C6A0C6A0C6A0C640C6A0C5C0C1F
:100540005C0C5C0C5C0C5C0C5C0C560C5C0C4E0C7F
:100550004E0C4E0C4E0C4E0C4E0C3F0C4E0C030C25
:10056000030C030C030C030C030CEE0B030CE60B47
:10057000E60BE60BE60BE60BE60BE00BE60BD80B07
:10058000D10BC90BB30BAB0BA00B6B0B640B5C0B50
:10059000440B3C0B360B2E0BF70ABF0AAC0AA50A1C
:1005A0009F0A980A7C0A750A6B0A360A300A290AD9
:1005B000F609EF09D409CD09C00987096E09670951
:1005C00062095B0956094F0947091A09FE08F7082D
:1005D000E408DD08C508BE08B6088D08870880084D
:1005E0006008590849084208F107C707B307AC0774
:1005F00093078C077C07750768073507E706002413
:10060000B349B44814600DF085FE0646002800F09A
:10061000F6848DF821408DF822400DF05FFAAE4946
:1006200030460DF07FF9AD4930460DF07BF9AC490D
:1006300030460DF077F9AB4930460DF073F9AA4911
:1006400030460DF06FF9A94930460DF06BF9A84915
:1006500030460DF081F9A74930460DF07DF9A649E5
:1006600030460DF05FF90DF1230130460DF05AF9D7
:100670000DF1210130460DF055F99DF82130FF2B89
:1006800000F0AF8403F0200202F0FF055AB101210F
:100690009A480FF051FC9A4B1B6898680DF0CEFCFD
:1006A0009DF821300125C3F34203964A9649137001
:1006B00030460DF037F9954930460DF033F994493D
:1006C00030460DF02FF9934930460DF02BF9924941
:1006D00030460DF027F9914930460DF023F9904945
:1006E00030460DF01FF98F4930460DF01BF98E4949
:1006F00030460DF017F98D4930460DF013F98C494D
:1007000030460DF00FF98B4930460DF00BF98A4950
:1007100030460DF007F9894930460DF003F90DF127
:10072000220130460DF0FEF89DF82230002B00F03B
:10073000A281834A01231370824930460DF0F2F8FA
:100740000DF1220130460DF0EDF8694A9DF8223096
:1007500014887D4A03F003031370002C00F08E818F
:100760007DB97A4C04F540450DF1220130460DF07B
:10077000D9F89DF8223004F8013FA542F4D15C4B32
:100780001C88734B1C80734B00241C70724B1C70B4
:10079000724B1C70724B30461C600DF095FB714B18
:1007A0001C706DE500200CF089FC63E56E4B6E4912
:1007B0001B780133DBB20B706C490022102B0A60EE
:1007C00000F0FC834F4B6A4E1D78694B1B78AB429F
:1007D00027D0684B33F8154000942F2340F247226E
:1007E000102108200CF0BAFC40F2AF132722302170
:1007F000082000940CF0B2FC40F2AF1340F2472204
:1008000030214FF40A7000940CF0A8FC009440F2E0
:10081000CF1340F247224FF4D87108200CF09EFC11
:1008200035704A4B0693544B059300234FF4804B8D
:1008300004934FEAAB0505F038024FEA6B13CBF394
:100840000225154303F0C0034FEACB041D4304F017
:10085000F804EA08E30803EB4213484A06981178C3
:10086000474A10F8017F069003F5B043D25C21B1EE
:1008700005990978B94200F0CE803F4B04991606DD
:100880005F5400F1D68002F00703C2F3C20A194692
:10089000500607D50B4608330AF1080ADBB25FFAA7
:1008A0008AFA194664006D0028343035002F00F0B4
:1008B000A680FF2F00F0C88004F11009CDF81CB00D
:1008C0001FFA89F9802605F1010803978B4666E037
:1008D0004C040108F40200207B4201207A420120EE
:1008E00075420120744201207942012078420120A2
:1008F000D8080020F0020020000900205004010860
:1009000020010020E80800207742012076420120E3
:10091000DD020020DC020020DF020020DE020020D9
:10092000E1020020E0020020E3020020E2020020B9
:100930007F4201207E4201207D4201207C42012035
:10094000EE020020ED020020D8010020A765002063
:1009500002090020F403002082420120834201208A
:1009600084420120F5030020E1080020D00100208E
:10097000020000202C04010808090020EC020020DD
:10098000A8250020A44F023437F81BE0CDF800E082
:10099000A4B20CF0E3FB4C454FEA560617D0039B7C
:1009A0001E4204F10102434629462046EAD19A4BF1
:1009B000621C33F81A30009320460234434629461D
:1009C000A4B20CF0CBFB4C454FEA5606E7D1DDF85C
:1009D0001CB0049B059A01330132B3F5C05F049348
:1009E0000BF1010B05927FF424AF4FF440728B4959
:1009F0008B480DF035FE8B4A0123137034E4864B8F
:100A000033F81A30009329466B1C04F10F0220467C
:100A10000CF0A4FBDDE782490B44A3F5B0431B783F
:100A200093427FF42AAF804B1B78002BD1D1130661
:100A3000CFD57E4B1B78002B3FF425AFC2F3C2030A
:100A4000194602F0070A23E7734B33F81130D9E750
:100A5000774BD979062900F0D7820D2900F0D6828C
:100A6000744B186882680AF09FFC724B1B68986888
:100A70000DF0E4FABEE4704A13705DE60DF1260154
:100A800030460CF069FF6D4930460CF065FFBDF84B
:100A90002630023B9BB2ADF8263053B10DF1230155
:100AA00030460CF03FFF0134BDF82630A4B2A3421B
:100AB000F4D800238DF824308DF825300DF126016F
:100AC00030460CF049FF0DF1250130460CF02AFFAD
:100AD000BDF826204FF6FF739A429DF82530A3F10A
:100AE0000403DBB263D0042B4FF001085BD94FF64F
:100AF000FF7782B3524B00252C4603EB070912E027
:100B00009DF822A0BAF1ED0F32D04FF6FF739F424D
:100B100003D06B1C09F805A09DB20134BDF8263046
:100B2000A4B2A34217D90DF1220130460CF0FAFE0F
:100B3000B8F1000FE4D14FF6FF739F42EDD09DF85E
:100B4000223009F805300134BDF82630A4B2013551
:100B5000A342ADB2E7D87368013B002B736033DB6F
:100B600033685A1C3260187831460EF021FCA5E734
:100B70000DF1220130460CF0D5FE9DF82220631CB9
:100B8000ED2A9BB229D04FF6FF718F421AD0691C13
:100B900089B209F805A002351C4609F80120ADB25A
:100BA000BBE74FF00008274931F81370A1E74FF475
:100BB0008042042BADF82620F3D94FF6FF774FF093
:100BC000000897E71C46A8E71A4B314618680EF054
:100BD00049F8431C3FF4D3ADC6E709A930460CF0F1
:100BE000A1FE0DF1220130460CF09CFE9DF8241070
:100BF0000334A4B2002990D09DF8220000234FF6C0
:100C0000FF72974203F1010303D06A1C09F8050043
:100C100095B29942F3D180E72C040108A87D002009
:100C2000D0050020EC020020E1080020040900208B
:100C30007442012020010020EE020020D80800208C
:100C4000A8250020B40401089E499F480DF062FBCE
:100C50000546002800F0B8809C4B1C789C4B294628
:100C6000D8790EF0EDFC9A4B294698790EF0E8FC05
:100C7000974B294658780EF0E3FC954B2946187897
:100C80000EF0DEFC924B294658790EF0D9FC904BC1
:100C9000294618790EF0D4FC294600200EF0D0FC2D
:100CA000294600200EF0CCFC8A4B284619880CF00F
:100CB00093FE894B294618780EF0C2FC6400294641
:100CC00000200EF0BDFC294604F0FE000EF0B8FC3A
:100CD0007F4B2946D8780EF0B3FC7D4B2946987897
:100CE0000EF0AEFC7D4B294658780EF0A9FC7B4BEC
:100CF000294618780EF0A4FC784B2946D8780EF0D7
:100D00009FFC764B294698780EF09AFC734B294647
:100D100058790EF095FC714B294618790EF090FC2D
:100D20006E4B2946D8790EF08BFC6C4B294698798E
:100D30000EF086FC664B2946D87A0EF081FC644B97
:100D40002946987A0EF07CFC614B2946587A0EF0C1
:100D500077FC5F4B2946187A0EF072FC604B2946EF
:100D600018780EF06DFC5F4B294618780EF068FC81
:100D70005D4B294618780EF063FC362128460CF0AE
:100D80002BFE5A4B284619880CF026FE3424013CD1
:100D900029460020A4B20EF053FC002CF7D14FF4EA
:100DA0000042042128460CF0F5FD4FF44042052195
:100DB00028460CF0EFFD28464FF4804208210CF045
:100DC000E9FD28460DF080F8494A00231360FFF73B
:100DD000B2BA484B484E1968484D20460BF01CFBF0
:100DE0000DE0B3F5B97F00F0DF8040F27512934259
:100DF00002D1002C40F0FC8001200CF05FF9404B48
:100E00003F491B680022762B0A6023D05A2B02D060
:100E1000E7D8292BF0D1062CEED8DFE804F028160D
:100E20000479B645360001200BF048FC074600283F
:100E300000F014820FF06AF9042808D93946FF221D
:100E400030480FF06BF90CF025FD0CF047FE012047
:100E50000CF034F9274BFF2019680BF0DDFA2A4912
:100E600000220A60294A01231370FFF75FBA234B5F
:100E70001B780133DBB2042B08BF00232B701D4B02
:100E8000002019680BF0C8FAB6E71B4B93F88030C6
:100E9000002B00F04381002386F88030154B06209C
:100EA00019680BF0B9FAA7E701200BF015FB002831
:100EB00001F0A583014604480FF020F90C4A0123F4
:100EC0001360C4E788040108CC040020E80800206F
:100ED00074420120F002002000090020DC02002002
:100EE000EE020020ED020020D8010020D8080020EA
:100EF0004C010020E8020020FC030020000000203C
:100F0000DC080020DC010020E408002001000020B3
:100F100000200BF0D3FB0746002800F018810FF0EB
:100F2000F5F80428034692D91C1F934B934A0025D9
:100F30001D60934B10681D70924B16461D6010B1DA
:100F40000CF0C2FF35603C4420468F490FF0A0F8FA
:100F5000002801F068838D4920460FF099F8002899
:100F600001F0548320468A490FF092F800287FF45C
:100F70006EAF884C82480323FF22394623700FF05E
:100F8000CDF8804A0123136061E7834B1F68002F6F
:100F900000F0C880814B00241C60814B1C7006F05F
:100FA000DFFB7D4B1C6052E7052C3FF625AF7A4BEB
:100FB0000134204619680BF02FFA1DE7794B7A4966
:100FC0001B780A70B3FA83F3764A5B091370FFF754
:100FD000F9BB764B754A9B7923F001039371FFF7B8
:100FE00009BA0122234625468DF82120FFF75DBB73
:100FF000694B013C204619680BF00EFAFCE66C4880
:101000000DF026FCFFF73CB9092129E5694B18686A
:1010100082680AF0C9F9674B18680A2182680AF0E9
:10102000C3F922E5644A20231370FFF7E3B95B4B51
:101030001B68002B4FD15D4B5C4A9B7923F0010369
:1010400093715E4B5E4A1B885D48D25C591C89B225
:101050000233415C42EA01225A490A80574A13800E
:10106000FFF75DB9444B1A68574B93F80680002A86
:10107000E1D0DF7941494D4B0C681D7A5A7A9E7850
:101080004449DB7891F80090DFF8F0A0003718BFF2
:10109000012708F0010842EA052543EA0626002C4C
:1010A00001F09382B9F1010F01F0A082B9F1020FB2
:1010B000C1D13B4642463146284606F003F9002896
:1010C000B9D03A4B39499B79002243F001038B7127
:1010D0008A70CA70B5E7354BDA799C78D978187A76
:1010E0005B7AA2F1FF02B2FA82F241EA04215209CC
:1010F00043EA00202D4C07F035FE00289BD0A37951
:1011000043F00103A3719CE72E4A38231380FFF7B5
:1011100006B901339BB20B80FFF7D0B8012386F8E4
:101120008030BBE638460BF0D7F9F0B11B4B1B4CB7
:101130001F601B4B80461F7006F012FB40460EF0EE
:10114000E5FF042809D8144A012313607FE6124BF7
:10115000032019680BF060F94EE64146FF22104863
:101160000EF0DCFF01232360EDE70B4B0420196830
:101170000BF052F940E600BFF0080020F80800200C
:10118000F4020020D008002070040108780401084F
:1011900080040108E0080020E8020020EC0800209C
:1011A000A424002004090020E1080020744201204A
:1011B000DC01002020010020E4810020F00200205A
:1011C000A8250020D8080020DC020020382008F0E4
:1011D00063F8994B1B7813B9984B1B784BB1984B1C
:1011E0001A78002A37D0944900220A7093491A705D
:1011F0000A70944B93491B6848F2373293427FF64A
:101200002EA8914A91481268D0F8CC00A3F5034368
:10121000373B0B6002F16403A0B18D4A13608D4B24
:101220008B4A1B68884912680A600133894A022B7D
:1012300013607FF414A800211160874A0123137002
:10124000FFF70DB8824A12689342E8D9804A1268C3
:101250009342F7D8E3E701221A70CAE77F4B0220D6
:1012600019680BF0D9F8C7E57D4B7E4A1B887E4C88
:10127000D1797B4D734A7B4E126801339BB201F0EA
:101280000F00E45C2B8004F00F03C31A6D480D1BA4
:101290000732DB06ADB2026022D4B37923F010032B
:1012A000B371E243D2B2284609F05EFF284609F046
:1012B0002FFF6C4B6B489979694B41F002011A88FA
:1012C00081715D4B66491B7801320A8083E7644B6C
:1012D00063491B8801330B80584B01221A707EE74B
:1012E0000CF0CEFCF179DCE70721002005F014FAC0
:1012F000514B1B786FE7534B52491A68584B0432D5
:101300001B880A60564901330B80584B01221A7022
:10131000494B1B785FE70721002005F0F7F8464BA3
:101320001B7858E7444B1B78002B28D1434A12788E
:10133000F2B9444A11684B4A10795279063142EAAF
:101340000022404801604A490A80454A44491288BF
:1013500001320A803FE70721002007F0CBFF364B20
:101360001B7838E7302007F097FF334B1B7832E7C4
:10137000344A11683B4A0A31907AD27ADFE7314A1F
:101380001168384A0A31107A527AD8E7344B354A14
:101390001B883548D2792B49314D324C09680133CD
:1013A0009BB22B80C05C40EA02031846E371254BD8
:1013B0000731196009F098FE2E49E279A3798A5C19
:1013C00023F01301A171002A58D123F01703A37150
:1013D000234B23491A88184B01321B780A80FAE6FE
:1013E000204B1848D9799A79214B234C1B880068E7
:1013F0002488144E42EA0122591E89B2A14200F10A
:101400000B0012B2306028BF1748C2F30725A3F1C2
:1014100002039BB228BF455415499C420B8098BFDC
:101420001149D2B298BFCA540D4B0D491A88024BCC
:1014300001321B780A80CEE68242012083420120DD
:10144000F403002084420120D4010020FC0300208A
:10145000FC080020CC050020F5030020E802002055
:10146000D808002074420120A8250020EE020020A8
:10147000F0020020C0040108804201200CF0F8FBBB
:10148000A6E70721012005F047F9974B1B78A2E654
:10149000964B96491A68964B04321B880A60944909
:1014A00001330B80934B00221A708F4B1B7892E60E
:1014B0000721012005F02AF88B4B1B788BE68E4B19
:1014C0001A888A4B18688D4B541C9B5C911CA4B2E3
:1014D0008A4A125D884C43EA02222180884C844B60
:1014E00012B2A271C2F30722E271804A19887E4BC0
:1014F0000A3010607E4A1B78013111806BE60721AB
:10150000012007F0F7FE784B1B7864E6282007F0EF
:10151000C3FE754B1B785EE6754B794A1B8877488E
:10152000D2797249724D764C096801339BB22B8097
:10153000C05C80EA02031846E3716C4B0731196006
:1015400009F0D2FD6F49E279A3798A5C23F0130197
:10155000A1717AB923F01703A371654B64491A8806
:10156000614B01321B780A8035E603F07FF95E4B50
:101570001B7830E60CF07CFBEFE70221002005F041
:10158000CBF8594B1B7826E6584B5D485C4C5C49C0
:10159000C0781A68564B4979607154481B88E170CD
:1015A000043202605248227901330380A378237108
:1015B0004D4BA2701B780EE60221002004F0A6FF1E
:1015C000494B1B7807E6484B1B783BBB4E4A1278C9
:1015D000CAB9464A454C1168494A107952790431D2
:1015E000216042EA002242490A80F4E502210020FB
:1015F00007F080FE3C4B1B78EDE5202007F04CFE09
:10160000394B1B78E7E5394A384C11683C4A907AE7
:10161000D27A0831216042EA0022E4E7334A334CAF
:101620001168374A107A527A0831216042EA002262
:10163000D9E72F4B324A1B883048D2792B492C4DA1
:101640002F4C096801339BB22B80C05C00EA020377
:101650001846E371254B0731196009F045FDA37960
:10166000E179284823F00302415C42F01002A271A4
:1016700089B923F0070343F01003A3711C4B1C49E5
:101680001A88194B01321B780A80A4E507F064FE22
:10169000154B1B789FE50CF0EBFAEFE702210120D8
:1016A00005F03AF8104B1B7895E504F09FFF0E4BC0
:1016B0001B7890E50221012004F028FF0A4B1B78DB
:1016C00089E507F0C9FE084B1B7884E5022101205B
:1016D00007F010FE044B1B787DE5182007F0DCFDB9
:1016E000014B1B7877E500BF824201208442012034
:1016F000D8080020EE020020F0020020A8250020DB
:1017000074420120C004010883420120954B964A8F
:101710001B88964CD1799679954A934F106801337E
:101720009BB201F00F02E55C8E4C238005F00F03A5
:10173000D21A06F001044B1B121B1C1B8C4B0730EA
:10174000D206A4B2186023D426F01006BE71EA4374
:10175000D2B2204609F008FD834B2046DC7109F027
:10176000D7FC814B804899797E4B41F002011A8861
:101770008171804B7B491B7801320A802BE5794BC4
:1017800078491B8801330B807A4B01221A7026E5B9
:101790000CF076FAF979DAE70021084604F0BCFF8C
:1017A000744B1B7817E56F4B6F491B88C8796D49DF
:1017B0006F4A01339BB20B806C491268C95C6C4B59
:1017C0000B321A6009F0E0FC664B674A1B88D07147
:1017D000644A01331380674B1B78FCE40021084600
:1017E00004F094FE634B1B78F5E45F49604B0C7882
:1017F00061495D481A6809785A4B01705C491B8839
:10180000407804320A60574A013313805A4B5978A2
:101810001C70554B9A78584B587053489B784170C0
:10182000C17855488270C2784F4883700379524816
:10183000C17001794C48C27042794F4803714379B5
:101840004948017143714C494A4B4A711B78C2E4C3
:101850000021084607F04EFD464B1B78BBE41020E4
:1018600007F01AFD434B1B78B5E43E4B3E4A1B88FC
:101870003E4CD1793B4E3E4A3B4D126801339BB200
:1018800001F00F00E45C338004F00F03C31A384802
:1018900007320E1B0260D806B7B221D4AB7923F011
:1018A0001003AB71E243D2B2384609F05DFC2E4B17
:1018B0003846DE7109F02CFC2B4B2B489979294BCB
:1018C00041F002011A8881712A4B26491B780132A6
:1018D0000A8080E4012007F08BFD264B1B787AE418
:1018E0000CF0CEF9E979DDE70021012004F014FFC6
:1018F000204B1B786FE41E4A1A4B11681B881A4A4A
:101900001948D279007801F10B04013315499BB2D3
:101910000B801649C95C164B1C6009F0D7FC114BB3
:1019200010491A88134B01321B780A8053E40021B6
:10193000012004F0EBFD0F4B1B784CE4012007F075
:10194000E5FD0C4B1B7846E40021012007F0D2FC9A
:10195000084B1B783FE4082007F09EFC054B1B78E2
:1019600039E400BFD808002074420120A8250020D7
:101970008442012082420120DC0200209A4B9B4AD3
:101980001B889B4CD17990799A4A984F1268013301
:101990009BB201F00F06E55C934C238000F001033D
:1019A00005F00F041E4426446C181C44914B07326A
:1019B000F6061A604DD420F01000B8712A46204671
:1019C00009F0D2FB894B2046DC7109F0A1FB874B63
:1019D00086489979844B21F002011A888171864BDF
:1019E00081491B7801320A80FFF7F5BB81497E4BA4
:1019F0000C681B888149824A0D881288DFF8F0E163
:101A00007C4E591C981C80B289B21EF800701EF8DA
:101A10000110501E033380B29BB2A84201EB072194
:101A2000A2F102024FEA132728BF0EF8007092B20B
:101A300073489542028098BF6D48DBB298BF8354CB
:101A4000694B89B219806C4B113434601B78FFF7F5
:101A5000C2BB0CF015F9F979B0E70621002004F0BB
:101A60005BFE654B1B78FFF7B6BB07F091FA624B44
:101A70001B78FFF7B0BB0621002004F047FD5E4B4A
:101A80001B78FFF7A8BB5E4B594C1B885849594A35
:101A9000C95C1268581C80B20233205C584C238009
:101AA00041EA002350490B80524B0A321A60524BD4
:101AB0001B78FFF790BB0621002007F01BFC4E4B64
:101AC0001B78FFF788BB002007F0E6FB4A4B1B782A
:101AD000FFF781BB444B454A1B88454CD179424EA8
:101AE000444A424D126801339BB201F00F00E45C9E
:101AF000338004F00F0303443E480E190732DB061F
:101B0000B7B2026022D4AB7923F01003AB71224646
:101B1000384609F029FB354B3846DE7109F0F8FAF2
:101B2000324B32489979304B21F002011A88817189
:101B3000314B2D491B7801320A80FFF74CBB002046
:101B400007F056FC2C4B1B78FFF745BB0CF098F8C0
:101B5000E979DCE70621012004F0DEFD264B1B7845
:101B6000FFF739BB204B22481B88224A991C0133BE
:101B700089B29BB2415CC35C126803EB01231A4932
:101B80000B801C4B0A321A601B4B1B78FFF723BBE0
:101B90000621012004F0BAFC174B1B78FFF71BBB92
:101BA000002007F0B3FC144B1B78FFF714BB062191
:101BB000012007F09FFB104B1B78FFF70CBB04F0D4
:101BC000BBFE0D4B1B78FFF706BB04F0070004F0CB
:101BD00017FF094B1B78FFF7FEBA07F0F9FD064B1C
:101BE0001B78FFF7F8BA00BFD80800207442012024
:101BF000A825002084420120824201208042012049
:101C0000F0020020A74B1B7804F007043BB3A64B5F
:101C1000A5491B6803F10802231F012B0A6000D8A5
:101C20000434A24BA14A1B5DD279A04C1343184641
:101C3000E37109F059FA9E49E279A3798A5C23F0AD
:101C40001301A17102BB23F01703A371994B9949AA
:101C50001A88944B01321B780A80FFF7BCBA964B66
:101C60001B78A3B1904B90491A68231FDBB208324E
:101C7000012B0A60D5D80634E4B2D2E707F008FD9C
:101C8000884B1B78FFF7A7BA0BF0F2FFDEE7864B15
:101C9000854A1B6804331360C3E704F0070007F0AC
:101CA0004FFD804B1B78FFF796BA05F01DF97D4B71
:101CB0001B78FFF790BA04F0070005F073F9794B31
:101CC0001B78FFF788BA07F029FE764B1B78FFF7E1
:101CD00082BA04F0070007F089FE724B1B78FFF709
:101CE0007ABA07F0D9FE6F4B1B78FFF774BA04F08D
:101CF000070007F037FF6B4B1B78FFF76CBA09F052
:101D00000FFD684B1B78FFF766BA04F0070009F077
:101D10006DFD644B1B78FFF75EBA09F04BFC614B1D
:101D20001B78FFF758BA04F0070009F0A9FC5D4BD7
:101D30001B78FFF750BA072004F008FA594B1B78BC
:101D4000FFF749BA04F00701072004F03FFA554BAA
:101D50001B78FFF740BA544B53491A68514B043271
:101D60001B780A60FFF737BA4E4B1B7804F0070464
:101D7000002B28D04F4B1A884C4B187A5B7A4A4973
:101D8000013243EA002392B24C480968805603446A
:101D9000454813319BB2016049490888434998423C
:101DA00098BF4648095D98BFC154531C414A1380EF
:101DB0003C4B1B78FFF70FBA052004F0C7F9394BED
:101DC0001B78FFF708BA3C4B1B782BB3394B1A88AA
:101DD000364B987ADB7AD2E704F00701052004F04D
:101DE000F5F9304B1B78FFF7F6B904F00701042032
:101DF00004F0ECF92B4B1B78FFF7EDB9032004F04E
:101E0000A5F9284B1B78FFF7E6B9042004F09EF9EA
:101E1000244B1B78FFF7DFB9234B264A1968234B65
:101E2000214D18795B7912880731296043EA002334
:101E3000B2E704F00701032004F0C8F9194B1B783E
:101E4000FFF7C9B9022004F081F9164B1B78FFF7A0
:101E5000C2B904F00701022004F0B8F9114B1B7855
:101E6000FFF7B9B9012004F071F90E4B1B78FFF7A9
:101E7000B2B904F00701012004F0A8F9094B1B785E
:101E8000FFF7A9B9002004F061F9064B1B78FFF7B2
:101E9000A2B904F00701002004F098F9014B1B7867
:101EA000FFF799B982420120844201207442012047
:101EB000C0040108D808002083420120A825002082
:101EC00080420120A74BA7491A68A74B9B7904328F
:101ED0000A60DA07A54AA44912884CBF03F0FE0342
:101EE00043F0010323F002038B71A04B01321A80EF
:101EF0009F4B1B78FFF76FB9072004F0ABF99C4BA1
:101F00001B78FFF768B9072004F0C8FC984B1B78D2
:101F1000FFF761B9072004F01DFF954B1B78FFF711
:101F20005AB9904B8F481968924B06311A888F4BDB
:101F3000016090491B88013A0A808C4A0133138062
:101F40008B4B1B78FFF747B9884B864A1B88116873
:101F5000894C9A1C92B2581C80B2A45C864A125CCE
:101F6000854802EB042292B20333825C7E48C27140
:101F70007E4A13807B4B0D3119607D4B1B78FFF738
:101F80002AB904F0F7FD7A4B1B78FFF724B900213A
:101F9000084604F08FFA764B1B78FFF71CB9724B9A
:101FA000704A9B7970481168704A23F0120343F01D
:101FB000010383716B4B1288043119606B4B013242
:101FC0001A806B4B1B78FFF706B907F019FB684BBB
:101FD0001B78FFF700B904F0F1FB654B1B78FFF7A6
:101FE000FAB804F047FE624B1B78FFF7F4B85D4B7C
:101FF0005C4819685F4B06311A885C4B01605D498B
:102000001B8801320A80594A01331380584B1B78D0
:10201000FFF7E1B8554B584C1A88524B1968574B8B
:10202000901C1D88531C9BB280B2E35C205C03EBC8
:1020300000234C480D3101604B499BB29D42C97948
:1020400098BFE154494B03321A80494B1B78FFF784
:10205000C2B8464B484C1B88424A591C981C89B24E
:1020600080B2615C205C126801EB00214148018074
:102070003E4903330B803B4B0A321A603C4B1B78C2
:10208000FFF7A9B80021012004F014FA384B1B789F
:10209000FFF7A1B8334B334C1868334B0430D97970
:1020A0009A79324B206030481B8842F012028271CC
:1020B0002E4A013313802E4BC943C1711B78FFF7A1
:1020C0008AB8052004F0C6F8294B1B78FFF783B8BF
:1020D000052004F0E3FB264B1B78FFF77CB80520B6
:1020E00004F038FE224B1B78FFF775B804F0D2FAE3
:1020F0001F4B1B78FFF76FB804F056F91C4B1B7889
:10210000FFF769B804F0CEFC194B1B78FFF763B8F2
:102110000621002004F0CEF9154B1B78FFF75BB8C1
:1021200004F090FE124B1B78FFF755B8042004F022
:1021300091F80F4B1B78FFF74EB8042004F0AEFB6C
:102140000B4B1B78FFF747B8042004F003FE084B45
:102150001B78FFF740B804F007FA054B1B78FFF730
:102160003AB800BF8442012074420120D808002000
:1021700082420120F0020020A82500208042012098
:10218000A04BA14C1988A14B4A1C881C92B280B26A
:10219000A25C205C1B7802EB002292B2F3B19C4857
:1021A0009B4E05689B481435447A007A35609A4DF9
:1021B0002D88AA4224BF944EB454013292B2954263
:1021C0009CBF914CA0548F4A03311180FFF703B894
:1021D00004F078F88D4B1B78FEF7FDBF8F48007830
:1021E000002833D08A488A4E05688A481435C47A54
:1021F0003560807ADBE70621012004F05BF9834B30
:102200001B78FEF7E8BF824B82491A68814BC97977
:102210009B797F4804320260D8074FEA510248BFD9
:1022200042F08002C90777497A480988C2714CBFD9
:1022300043F0010303F0FE0323F012038371714B9B
:102240004A1C1A80714B1B78FEF7C5BF7048704E50
:10225000056870481035447935600079A7E7032098
:1022600003F0F8FF694B1B78FEF7B5BF032004F0BD
:1022700015FB664B1B78FEF7AEBF032004F06AFD2A
:10228000624B1B78FEF7A7BF624B62489A78DB78F7
:102290005F4943EA0223013B9BB20968594AC37074
:1022A0001B0A83705A4B128806311960554B013254
:1022B0001A80564B1B78FEF78EBF564B52489978C2
:1022C000DB78534A43EA01211268415C51484D4B87
:1022D000C1714F491B8807320A604A4A0133138093
:1022E0004A4B1B78FEF777BF012009F09FF8474B58
:1022F0001B78FEF770BF434B43481B88444A591C68
:1023000089B20233415612680B443E490B80404B60
:102310000C321A603D4B1B78FEF75DBF3C4B3C48CE
:1023200019683C4BDA799B790431DD074FEA4202A8
:102330000160384948BF42F00102D405CA71314AF0
:10234000344912884CBF43F0010303F0FE0323F02D
:1023500012038B712B4B01321A802C4B1B78FEF72A
:102360003ABF022003F076FF284B1B78FEF733BFFD
:10237000022004F093FA254B1B78FEF72CBF0220B5
:1023800004F0E8FC214B1B78FEF725BF214B2148C8
:102390009A78DB781E4943EA022301339BB209682D
:1023A000184AC3701B0A8370194B128806311960D2
:1023B000144B01321A80154B1B78FEF70CBF144BDF
:1023C00015491A68134B09889878DB7843EA00238B
:1023D0000F480732994202600E4A98BF0A49D279E3
:1023E00098BFCA54074B07491A88084B01321B781B
:1023F0000A80FEF7F0BE012003F0B2FF034B1B780A
:10240000FEF7E9BED8080020A8250020824201205E
:102410008442012074420120804201208342012035
:10242000A34BA44A1B88A44C1278A148591C89B21A
:10243000023361569F4C9BB2013A1944D2B289B221
:1024400022702ABB9D4A038012689C4B08321A6096
:102450009B4B1B78FEF7BFBE984B98481A68954B6C
:102460009449DB790432DE0702601BD48A795B0869
:10247000CB7102F0FE038E4A8E49128823F01203BC
:102480008B718B4B01321A808D4B1B78FEF7A3BEEC
:102490008A4B8A4A1B6801800D331360884B1B7876
:1024A000FEF799BE5B088A7963F07F03CB7142F037
:1024B0000103E0E7012003F0CDFE814B1B78FEF71E
:1024C0008ABE012004F0EAF97D4B1B78FEF783BE3B
:1024D000012004F03FFC7A4B1B78FEF77CBE754B65
:1024E00074481A785B78754943EA0223013B9BB232
:1024F00009686F4A43701B0A0370704B12880631DB
:1025000019606B4B01321A806D4B1B78FEF763BE6E
:10251000684B694819785B78684A43EA0121126878
:10252000415C6448624BC17164491B8807320A6090
:102530005F4A01331380624B1B78FEF74CBE0020CC
:1025400008F074FF5E4B1B78FEF745BE5B4B5D48A1
:10255000584C58491A68C079554BC979E0715748A9
:102560001B88043202605248A27901330380554B24
:1025700054489B79A371524BC17182711B78FEF74D
:102580002ABE4E4B4D481A684A4B4A49DB79043201
:102590001F06026000F1DA808A795B00CB7102F0DD
:1025A000FE03434A4349128823F012038B71404BC8
:1025B00001321A80424B1B78FEF70DBE002003F05B
:1025C00049FE3F4B1B78FEF706BE3F493F480BF0E4
:1025D000A1FE0446CAF8000000283EF42CADB9F173
:1025E000020F2CD0B9F1010F7EF425AD00974346C0
:1025F00032462946204605F0BFF8FEF760BD344B51
:102600000520196809F008FFFEF7F6BB314C2F488A
:102610000223FF22394623700DF080FD2E4A01234C
:102620001360FEF714BC2B4B284801243946FF22C7
:102630001C700DF073FD284B1C60FEF708BC05F004
:10264000CFF800287EF435ADFEF7F5BC1B4B2349CF
:102650001A68184B098818785B7843EA00231748F2
:10266000073299420260134A98BF1349D27998BF42
:10267000CA540F4B0E491A88114B01321B780A803D
:10268000FEF7A9BD002003F06BFE0D4B1B78FEF793
:10269000A2BD0A4B09491A68054B04321B880A601F
:1026A000034A01331380064B1B78FEF794BD00BF2D
:1026B000D808002074420120A8250020844201206F
:1026C00082420120DC0200204C040108F4020020B8
:1026D000E8020020E0080020F008002080420120ED
:1026E0001E4B1F481A8821460DF026FC1D4B1B6807
:1026F00098680BF0A3FC1C4B1B78FEF76CBD002008
:1027000004F028FB184B1B78FEF765BD174B1748E4
:102710001A785B78164943EA022301339BB20968B1
:10272000144A43701B0A0370114B1288063119605A
:10273000104B01321A800C4B1B78FEF74CBD002069
:1027400004F0ACF8084B1B78FEF745BD5B008A79B6
:1027500043F00103CB7142F0010322E7020900209C
:102760008C040108200100208242012074420120D3
:1027700084420120D80800202DE98048C7B005F028
:102780007BF8BB4A936803F00C03042B00F0088528
:10279000082B40F0F88450685368400203F03F0172
:1027A00040F1F4845068B34AB2FBF1F3C0F38812ED
:1027B00003FB02F3AE4A5268C2F3014201325200F7
:1027C000B3FBF2F3AA4EAC4AB068DFF8F8E2AB4FC5
:1027D000AB49AC4DAC4CC0F30310125CD3409A092A
:1027E000AEFB020292093B60A848531EC8222A6031
:1027F000F0274B6007220523002584F823708D60A5
:102800000A600360336C4FF0804443F0010333648B
:10281000238823F45C731B04012740F219411B0C2D
:102820002380E2622185A782A3899BB23B43A381D7
:102830001C220F2306A88DF818208DF819308DF86A
:102840001A308DF81B7001F0E9FF2388904A9149F6
:102850009BB23B43238013688B4241F08C808E4AAD
:102860001368B3F5E13F00F09780814B8B4D8C4CA2
:1028700000204FF4E1318DF8160011601A6B42F020
:1028800001021A631A6B42F001021A631A6C42F4D5
:1028900000321A642B6A23F470632B622B6A43F4B0
:1028A000E0632B622B6A23F470432B622B6A0221B4
:1028B00043F4E04303202B62012204238DF814101B
:1028C0008DF8150004A928468DF81720049301F00F
:1028D00051FF04A928460823049301F04BFFA38964
:1028E0006FEA43436FEA53439BB2A381238A23F4E5
:1028F00040531B041B0C2382A3899BB223F4B053C7
:1029000023F00C0343F00C03A381A38A23F4407348
:102910001B041B0CA38206A801F0E0FEA289089B01
:10292000604C12F4004F03EB83035F4A03EB830315
:10293000A2FB03235A4A14BF5B0C9B0C9289A4FB95
:10294000031040096421150400FB11334FEA001005
:1029500000F129841A013232A4FB0223C3F343138A
:1029600003434F4A51499BB2138193899BB243F46D
:10297000005393810B6843F020030B600122002376
:10298000262106A88DF818108DF819308DF81A3008
:102990008DF81B2001F042FF3B4B454ADA600124D1
:1029A0000023312206A88DF818208DF819308DF8F3
:1029B0001A308DF81B4001F031FF9DF81B308DF867
:1029C00019403B228DF81820002B40F0CA87394B64
:1029D0004FF00062C3F88420254D374C2B6B374EE7
:1029E000374F43F00C032B63636A23F00F036362DA
:1029F000636A43F00C036362636A23F0F00363626B
:102A0000636A43F0C0036362636A23F470636362C2
:102A1000636A43F440636362636A23F470436362EE
:102A2000636A43F440436362636A23F4702363621E
:102A3000636A43F440236362336A23F4706333624E
:102A4000336A43F44063336202234FF470622046DA
:102A50004FF000088DF81D308DF81C3006A90123B9
:102A600006928DF81F308DF81E8001F083FE2BE05A
:102A70000038024000127A00640000207400002038
:102A800010E000E01400002000ED00E060000020F5
:102A90000C210020A08601004823002000000240F5
:102AA000004400401F85EB51C5B3A2910C44004087
:102AB0000006FA0500E100E000080240000C0240B8
:102AC000C0050108632D3E050423304606A9069380
:102AD00001F050FE4FF48053204606A906938DF86E
:102AE0001F8001F047FE6B6C43F400636B642B6B3B
:102AF00043F480032B630D2001F0B4FD17F8010FA0
:102B00000028F9D1E24E3368002B40F02F87DFF820
:102B10009093DFF890A3DFF890830446074606A859
:102B2000CDF80490CDF808A0CDF8189000F0DCFFA7
:102B30000028C0F20A8358F8203003B11F70029BAE
:102B40000BB11F70029B48F82030002202A901A897
:102B500002F018FD0328054600F0E182002840F04D
:102B600064852146CB480DF0E7F901233360002549
:102B7000C94F8DF81D508DF81E508DF81F50396BC0
:102B8000DFF82883DFF828B3DFF828A3C34C41F02F
:102B90000101012639634046C02306A906938DF83A
:102BA0001C6001F0E7FD40214FF08003A8F81810E9
:102BB000A8F81830396B41F018014FF00308396359
:102BC00058464FF2B37306A98DF81C508DF81F506C
:102BD00006938DF81D8001F0CDFD4FF680735046B1
:102BE00006A9069301F0C6FD396B41F078013963FF
:102BF0004CF233714FF002095846069106A98DF840
:102C00001E508DF81F508DF81D808DF81C9001F01E
:102C1000B1FDDBF8201021F00F01CBF82010DBF81C
:102C2000201041F00C01CBF82010DBF8201021F02F
:102C3000F001CBF82010DBF8201041F0C001CBF8F8
:102C40002010DBF8201021F47021CBF82010DBF8E5
:102C5000201041F44021CBF82010DBF8201021F4A3
:102C60007001CBF82010DBF8201041F44001CBF8C4
:102C70002010DBF8241021F00F01CBF82410DBF832
:102C8000241041F00C01CBF82410DBF8241021F0C3
:102C9000F001CBF82410DBF8241041F0C001CBF890
:102CA0002410DBF8241021F47061CBF82410DBF839
:102CB000241041F44061CBF82410DBF8241021F0FB
:102CC0007061CBF82410DBF8241041F04061CBF8A0
:102CD0002410DBF8241021F07041CBF82410DBF82D
:102CE000241041F04041CBF824104FF68073504639
:102CF00006A9069301F03EFDDAF8201021F070419C
:102D0000CAF82010DAF8201041F04041CAF820102B
:102D1000DAF8241021F00F01CAF82410DAF8241090
:102D200041F00C01CAF82410DAF8241021F0F00167
:102D3000CAF82410DAF8241041F0C001CAF82410AF
:102D4000DAF8241021F47061CAF82410DAF824109B
:102D500041F44061CAF82410DAF8241021F47041DB
:102D6000CAF82410DAF8241041F44041CAF82410BB
:102D7000DAF8241021F47021CAF82410DAF82410AB
:102D800041F44021CAF82410DAF8241021F470012B
:102D9000CAF82410DAF8241041F44001CAF82410CB
:102DA000DAF8241021F07061CAF82410DAF824103F
:102DB00041F04061CAF82410DAF8241021F0704183
:102DC000CAF82410DAF8241041F04041CAF824105F
:102DD00058464FF4005206A9069201F0CBFCDBF8EE
:102DE000242022F47002CBF82420DBF8242042F4C3
:102DF0004002CBF824205846802306A9069301F010
:102E0000B9FCDBF82020DFF8B0C022F07042CBF82C
:102E10002020DBF8202042F04042CBF82020BB6B82
:102E20004FF0204E33430F200D2141F21002BB63BF
:102E3000079509950A950B950C950690089107A89A
:102E4000CEF8002007C8069F0C9B3B4343EA0010C6
:102E500040EA01210A980B9B41EA024242EA0050F3
:102E600040EA03636FF07042CEF80430CCF80020E3
:102E7000DEF800304FF0C0473343CEF80030052075
:102E80003E8001F059FB4FF0E00AE22216E000BF5D
:102E900008210020F0050108003802400000086009
:102EA000E80B0108102100204C2300200000024004
:102EB000000C024000100240040100A023234FF048
:102EC000040B3A8064202380A4F80090A4F800B09A
:102ED000A7F800A0268001F03DFBE6229323B02155
:102EE000A7F800A01F20A4F800804FF0B40C3A808F
:102EF000A4F800B0DF222380A4F800A0E8233980E2
:102F00004FF0330A082125804FF0B60E2580A4F833
:102F100000802080268012202280172625801822FB
:102F2000A7F800C0A4F800804FF0F00C23802580A3
:102F30002923A4F800A02180A0492580A4F80080BE
:102F40002580A7F800E0A4F800902080258022804A
:102F5000A4F8008025802680A7F800C0A4F800808F
:102F60003B800A6812F0010F14BF2B460823940718
:102F700048BF43EA09035007914C4FF0C04648BF91
:102F800043F0010336229BB20625BE273280FF2084
:102F90002380378001232580002520802380208006
:102FA0002580284625800B60328040F21F31258025
:102FB00004F002FD284640F2DF1104F0E9FC2C2366
:102FC0002946224633804FF448754FF4F073013B95
:102FD00011804FF00004FAD1013DF6D12946FF20BF
:102FE00009F01AFA774B784E93E803000A0C012394
:102FF0003064A6F844107548754986F84620347048
:1030000086F88150C6F8C45086F8C94086F8C84092
:1030100086F880300BF07EF90746002864D0DFF890
:10302000E88105E00023037006A80DF06FF8D0B921
:103030003A464FF4807106A80BF074F800284ED081
:10304000232106A80DF042F804460028EAD13B21CE
:1030500006A80DF03BF80028E6D0047006A80DF095
:1030600055F80028E4D0421E06AB1A44801A1378A3
:10307000093BDBB2172B77D93D2106A80DF026F8C6
:1030800004460028D4D000230370524906A80CF04F
:10309000FFFF01348146002800F02F834E4906A827
:1030A0000CF0F6FF8146002800F01F834B4906A86C
:1030B0000CF0EEFF002840F00083494920460CF058
:1030C000E7FF002840F0EF8201233A464FF4807179
:1030D00006A886F880300BF025F80028B0D10AF059
:1030E000C5FC38460AF0F0FED6F8C420364B12B9BB
:1030F0000322C3F8C4203B493B48FF22A1F140070B
:103100000DF00CF80AF0C6FB0AF0E8FCD6F8C43063
:10311000DA0700F135829E0778D4FDF79DF8013477
:103120000A2001F009FA0A2C7FF4F9AC2F4C304A3E
:1031300023683049D8680CF09FFB23682E48DB6871
:103140001B2201210CF0F8FB11E5284C284A2368CA
:103150002849D8680CF090FB23682848DB682022B7
:1031600001210CF0E9FB02E528FA03F303F0010367
:1031700083F00101002B3FF47FAF02F80119C24236
:103180007FF475AF78E71E4BFFF71CBB52681C4BF2
:10319000B3FBF1F3C2F3881203FB02F3FFF70ABBA0
:1031A000184BFFF70FBBD9003231A4FB0132C2F339
:1031B000421242EA0003FFF7D4BB00BFB000002078
:1031C0000000086008090108FC0300201409010838
:1031D0001009010820090108280901082C09010823
:1031E000380901083C040020DC01002020010020F7
:1031F000140601081C06010870060108840701086E
:103200000024F40000127A0013008000DFF8A0927E
:103210009C4CD9F830309C4F9C4E43F00103C9F8C8
:1032200030304FF4C05303224FF0000806A9204667
:10323000069302238DF81D208DF81C308DF81F3069
:103240008DF81E8001F096FA636A23F4704363627E
:10325000636A43F420436362636A23F47023636206
:10326000636A43F420236362D9F8443043F4804313
:10327000C9F84430D9F8343043F08003C9F8343009
:103280000AF008F98249834AC6F810834346F96771
:10329000C7F8802005F1C40205F1D400711906EBCE
:1032A000820201350F2D5360784C46F820304FF0E4
:1032B000000081F88C33EDD108210122E070A4F8E0
:1032C000B21340202170A2700421E2724FF4A07268
:1032D000A080617002207049E280704A20727048BC
:1032E0002161A26101F5907102F508726065E161EA
:1032F000A0F5E07001F50871A265A2F5E072206208
:10330000E16500F50870A1F5E8616262A2F5A462CA
:1033100020666161A0F5CC6001F59071C4F8CC2005
:1033200002F58072C4F89000C4F8941060306031E7
:10333000C4F8982060324FF0A043C4F89C00C4F851
:10334000A01060306031C4F8A42002F52662C4F8F1
:10335000A800C4F8AC1000F5D2505249C4F8D020EF
:1033600002F54052E360C4F8D400C4F8D810C4F8A1
:10337000DC209A6801F5405122F00102C4F8E41003
:103380009A60DA6801F5805142F04002C4F8E81012
:10339000DA604FF05021444AC4F8E01003F560634E
:1033A000C4F8EC20C4F80C310AF0D8FB627AF36858
:1033B000002A0CBF4FF434124FF474129A63142095
:1033C00009F046FEF378012B07D1F26893680521D6
:1033D00061F3440343F020039360F268DFF8AC80AC
:1033E000D3686FF39E7343F00053D360322009F02B
:1033F0002FFED6F80C3100241C60D8F81420337A44
:10340000DFF88880012B136816BF012164F30103E4
:1034100061F301031360404609F032FE72691368DC
:103420006FF382031360F37A012B254600F0888244
:10343000D8F80C301D4900220692069A42F020026C
:103440000692069A102060F38A120692069A1A6172
:103450001A69069203E01A690692013902D0069AA7
:103460009406F8D405F08AFD00230493049AF368C7
:103470000E4942F010020492049A1A611A690492E9
:103480001CE000BF00000240D84101202C3C01207C
:10349000040000201800002000080050000900501F
:1034A000000B00500030005000800050400D030021
:1034B000003802401A690492013902D0049AD006F9
:1034C000F8D405F05BFD3278BA4B6AB1233203EBD6
:1034D00082024FF0FF308C33002153F8044FA0607C
:1034E0001C689A42E160F8D1D6F8CC2013686FF3DB
:1034F00082036FF341036FF3C3036FF34513D904E2
:1035000002D443F480531360C82009F0A1FDF2688F
:10351000F478A94800234FF0FF3193615161516065
:10352000F2689C4208BF10236FF08041516143F064
:103530000C539061916943F4001343F008030B436B
:103540009361936843F001039360D7F880301B6860
:1035500098479A4B9A4ADA6043210123032203A831
:103560008DF80C108DF80E208DF80D308DF80F3081
:1035700001F054F9102405F06BF8013CFBD1CCE5C7
:10358000904C9148236B43F0020323630026802371
:1035900006A906938DF81C608DF81F6001F0EAF80B
:1035A000606C8A4B8A4A8B4940F480406064D868DA
:1035B00020F47040D860D86840F48050D860136818
:1035C00023F080031360536823F080035360136873
:1035D00043F080031360936823F080039360D36803
:1035E00023F08003D3600B6843F080030B60172245
:1035F000012304A88DF810208DF811308DF81230B9
:103600008DF8133001F00AF9236B6F4843F0020381
:10361000236306A9402306938DF81C608DF81F6074
:1036200001F0A8F8D7F8C43075E56B4C6B4A2368F5
:103630006B49D868013D0CF01FF9122D00F277811B
:1036400001A353F825F000BF0B390008F938000832
:103650003B310008E7380008D5380008C3380008B7
:10366000B13800089F3800088D3800087B38000802
:1036700059310008693800085738000845380008F3
:103680003338000821380008A337000895360008B1
:103690001D39000823685348DB68222201210CF001
:1036A0004BF9FFF764BA20464F490CF0F1FC0028B3
:1036B0007FF4BEAC86F88000BAE44C4906A80CF052
:1036C000E7FC8146002847D0494906A80CF0E0FCF9
:1036D00038BB484920460CF0DBFCB0B9D6F8C43002
:1036E00043F00103C6F8C430A2E421463F22424819
:1036F0000CF014FD86F87F909AE421463F223F4863
:103700000CF00CFD86F83F9092E43D4920460CF009
:10371000BFFC48BBD6F8C43043F00203C6F8C4303F
:1037200086E4384906A80CF0B3FC58B3364906A81D
:103730000CF0AEFC00287FF47BAC20460AF054FB72
:10374000324B2E4A0340002B03DA013B63F00103A6
:10375000013382F8C8306BE421463F222C480CF03C
:10376000DDFC86F8C09063E420462A490CF090FC0A
:1037700000287FF45DACD6F8C43043F00403C6F8EB
:10378000C43055E420460AF02FFB234B1B4A03406C
:10379000002B03DA013B63F00303013382F8C930E5
:1037A00046E423681D48DB682A2201210CF0C4F896
:1037B000FFF7DDB92C3C01200008008000ED00E09F
:1037C0000006FA05003802400004024000380140BB
:1037D000003C01400C3C014020010020140601087F
:1037E0001C060108B80801083C0901084009010845
:1037F0004C090108580901083C040020FC03002082
:103800005C090108640901087009010801000080D1
:103810007D04002060090108030000808C08010875
:1038200023689C48DB683B2201210CF085F8FFF7F8
:103830009EB923689848DB68412201210CF07CF88E
:10384000FFF795B923689548DB68242201210CF025
:1038500073F8FFF78CB923689148DB681D220121BA
:103860000CF06AF8FFF783B923688E48DB681822EA
:1038700001210CF061F8FFF77AB923688A48DB6808
:10388000222201210CF058F8FFF771B9236887480C
:10389000DB68212201210CF04FF8FFF768B923689B
:1038A0008348DB68272201210CF046F8FFF75FB957
:1038B00023688048DB68392201210CF03DF8FFF7CE
:1038C00056B923687C48DB681C2201210CF034F8CF
:1038D000FFF74DB923687948DB681A2201210CF003
:1038E0002BF8FFF744B923687548DB680D220121E6
:1038F0000CF022F8FFF73BB923687248DB6811220D
:1039000001210CF019F8FFF732B923686E48DB6823
:10391000362201210CF010F8FFF729B923686B4813
:10392000DB681B2201210CF007F8FFF720B92368A0
:103930006748DB680E2201210BF0FEFFFFF717B985
:103940008022E021D8F80C3062F30F0461F30F05F8
:10395000C0F26004C0F260055A629C62C3F8005174
:1039600068E506A800F05AFFFFF736B859480CF092
:1039700055FBFFF7FCB8116009F0E2FC336B43F034
:1039800002033363336B04F5013443F00203336302
:10399000204606A94FF480768DF81D508DF81F50F3
:1039A0008DF81C708DF81E70069600F0E3FE4FF443
:1039B0000073204606A906938DF81C508DF81D5003
:1039C0008DF81E508DF81F5000F0D4FE23699A0523
:1039D00003D46683384600F0AFFD4FF480763E4D49
:1039E0003746092405E06E83012000F0A5FD013C67
:1039F00006D02F83012000F09FFD2B699B05F2D597
:103A0000354C364D4FF480762683012000F094FD2E
:103A100023692B6B43F002032B632B6B43F00203F0
:103A20002B632B6A43F400132B622B6A23F40013DD
:103A30002B62636A23F00F036362636A43F004033B
:103A40006362636A23F0F0036362636A43F04003D6
:103A5000636202220123204606A98DF81C208DF8FE
:103A60001D208DF81E308DF81F30069600F082FE66
:103A70004FF4007306A92046069300F07BFE2B6CE2
:103A8000174A184943F400132B64116008F0F4F846
:103A9000FEF7E5BE500801080C080108E40701081C
:103AA000C4070108A8070108600701083C070108CE
:103AB00014070108D8060108B80601089C06010889
:103AC0008C0601085C06010824060108DC080108D0
:103AD000F8080108D8050108000402400038024037
:103AE00044230020A0860100016809B310B40C78BB
:103AF000202C09D93A2C16D00A4601E03A2B07D0DF
:103B000012F8013F202BF9D800205DF8044B7047D4
:103B100001318A4207D1302C05D1013202605DF8B3
:103B2000044B002070474FF0FF305DF8044B7047A6
:103B30004FF0FF30704700BF2DE9F041074688463F
:103B4000066861BBF5681DB3B3699D4228BF0125B6
:103B500033690BB3B3692C4606E0012815D0013058
:103B600058D0AC4218D0B36901349C4202D3012D25
:103B700012D902242146386804F018F80028ECD144
:103B8000012C02D9B3699C422CD30120BDE8F081FD
:103B900033690125002BDDD10020BDE8F0813046DE
:103BA00004F004F80128F0D9421C33D0B3699842DC
:103BB00043D33269002AEFD008F10104A34298BF31
:103BC00002242146386803F0F1FF0128DDD0431CB0
:103BD00020D0A0B3F568B369012D33D99D4228BF29
:103BE0004546B8E74FF0FF322146304604F040F832
:103BF00070B9B8F1000F11D0B8F1010FC5D9B36990
:103C00009845C2D241462246304604F031F828B1E8
:103C10000128BAD14FF0FF30BDE8F081B3693269B5
:103C2000F460023B9A4201D8013A3261337943F0A1
:103C3000010333712046BDE8F081BDE8F081002C1E
:103C40009ED1B369454686E708B1042070472DE947
:103C5000F04FDFF86892904E904C914D30704FF0DD
:103C6000010E2060C5F800E0C9F82C00D9F83C70BE
:103C7000DFF854828B4BDFF854C247F44A7747F0A1
:103C80000207C9F83C704FF07469C8F808901F68C3
:103C900027F001071F601F6827F001071F60212719
:103CA000186058609860D86018615F61C8F8089023
:103CB000D3F800907C487D4F09EA0C0C4CEA0000D8
:103CC0001860D3F814C07A48A8F59B38A8F5C078D6
:103CD0004CF0070C4FF40079C3F814C0C3F80490FB
:103CE000C3F80880D960196841F01001196019689B
:103CF00041F020011960196841EA0E011960C7F806
:103D000000E0036883B05202022B009200F0A3800F
:103D1000684F00224FF0100B4FF4007A4FF040092B
:103D20004FF48068FA6087E8000CC7F80890C7F87D
:103D3000108009F02FFB584608F058FA002841D0AF
:103D40005D490B687BB923686BB933785BB94FF079
:103D5000FF3305E0226832B9327822B9013B02D044
:103D60000A68002AF6D00023544A0B60536B13F400
:103D7000805400F086804FF0FF3401E0002C6DD0BD
:103D8000536B13F4805704F1FF34F7D12A68444D84
:103D9000012A6ED0002C6AD03846484B3E4940F28A
:103DA000FF529A6333785BB10878C4B208F0AAFA7C
:103DB0000028FBD1201C18BF012003B0BDE8F08F04
:103DC0000446F3E73E4AF8601268C7F8089002FA22
:103DD0000BF24FF0370BC7F8108087E8040809F0A2
:103DE000D9FA584608F002FA0028A9D117224FF054
:103DF000010BF8607A600192C7F80890C7F810804C
:103E0000C7F800B009F0C6FA019A104608F0EEF9BA
:103E1000002895D11922009BF8607A6000923B60DF
:103E2000C7F80890C7F8108009F0B4FA009A104655
:103E300008F0DCF9002883D1224B4FF0FF319022AB
:103E4000C3F804A0D8601861C3F814B019609A6070
:103E500009F0BAFA74E7530A009359E72B68104D3A
:103E6000012B04D108F038FA2C60002895D10420E9
:103E700093E708F031FA2F60002C8ED100288CD106
:103E8000F5E72B68064D012B01D0204685E708F0A9
:103E900023FA2C6081E700BF882400208C240020B6
:103EA000E8230020586402404054A3088C85254232
:103EB0006C2400205C42012090240020002C014052
:103EC000043C0120143C0120006402403F801CF0AF
:103ED00083690BB9042070472DE9F04F056920353F
:103EE000B5F5001F83B003D3042003B0BDE8F08F05
:103EF000C5F308068846044607684EBB416901338E
:103F0000836161B3B7F80A9009F1FF3919EA5529BD
:103F10001ED1384603F04AFE0128824627D9B0F167
:103F2000FF3F34D0BB69984223D2831E019307F12F
:103F30003408C4F814A0BB690199023B994204D229
:103F4000B7F80A90FB6A01FB0939C4F8189001E040
:103F500007F134084644E66125610020C5E73B8946
:103F6000B3EB551FF4D80023A3610420BDE7022062
:103F7000BBE7B8F1000FF6D061692046FFF7DCFD22
:103F8000824630B90720B0E778898345D1D0012037
:103F9000ABE70128EBD0B0F1FF3FF8D0FB7843BB93
:103FA000BB69AAF10202023B9A42019227D3002385
:103FB0000093009B3B6307F13408434607F50D71FE
:103FC000002203F8012B9942FBD14FF0000B06E0D1
:103FD0007878FFF739FE0028D6D10BF1010B7889EC
:103FE000009B834503EB0B0241464FF00103EFD3E7
:103FF000CBE7384604F0BAF80028D1D0C7E77A8971
:10400000FB6A019901FB02330093D2E708B1042057
:1040100070472DE9F04FDFF810927B4D7B4C7C4EC2
:1040200028704FF0010C2060C6F800C0C9F82C00C1
:10403000D9F83CE0DFF8F481764B774F4EF44A7EB6
:104040004EF0020EC9F83CE04FF07469C8F80890D1
:10405000D3F800E02EF0010EC3F800E0D3F800E042
:104060002EF0010EC3F800E04FF0210E18605860EA
:104070009860D8601861C3F814E0C8F80890186810
:10408000DFF8AC91DFF8ACE1DFF8AC81074047F036
:104090000A6040F45530186058694FF4007740F0DA
:1040A000070058615F60C3F80890D96019685B4FDA
:1040B00041F010011960196841F020011960196878
:1040C00041EA0C011960C8F800C0DEF8003083B086
:1040D000022B4FEA422B4FF000034FF400724FF0D7
:1040E00010084FF0400A4FF480693A60019208BF0F
:1040F0004FEA5B2BFB60C7F80480C7F808A0C7F83D
:10410000109009F047F9404608F070F8019AF8B9A4
:10411000434B01905A604FF0FF31902219609A6032
:10412000022101221861D9604FF012085A6109F08A
:104130004BF90198F860C7F800B0C7F808A0C7F8B5
:104140001090C7F8048009F025F9404608F04EF8B1
:1041500034490B687BB923686BB92B785BB94FF096
:10416000FF3305E0226832B92A7822B9013B02D038
:104170000A68002AF6D000232B4A0B60536B13F415
:10418000005437D04FF0FF3400E004B3536B13F406
:10419000005704F1FF34F8D132681D4E012A21D0B6
:1041A000F4B13846204B184940F2FF529A632B78FD
:1041B0005BB10878C4B208F0A5F80028FBD1201C38
:1041C00018BF012003B0BDE8F08F0446F3E7336861
:1041D0000F4E012B04D108F07FF834600028E1D1A4
:1041E0000420DFE708F078F83760002CDAD10028E7
:1041F000D8D1F5E73368064E012B01D02046D1E730
:1042000008F06AF83460CDE7882400208C24002070
:10421000E8230020586402403F801CF05C420120EB
:10422000143C012090240020002C01400064024036
:10423000802C01406C2400208C85254238B5036B0E
:104240008B4218D0C37804460D467BB92A46012319
:1042500004F134016078FFF7D9FE002818BF4FF051
:10426000FF3525630CBF0020012038BD03F07EFF21
:104270000028EBD038BD002038BD00BF00224FF031
:10428000FF3310B5C27003630446FFF7D7FF08B1D0
:10429000042010BD94F8331294F832324AF65522B5
:1042A00043EA0123934201D0032010BD94F8343037
:1042B000EB2B05D01833DBB2012B01D9022010BD46
:1042C00094F86A30462B07D194F86B30412B03D118
:1042D00094F86C30542B15D094F886300A4904F1C8
:1042E0008702463B8B34002BE8D112F8013B11F8D2
:1042F000010FA242A3EB0003F5D1002B14BF022053
:10430000002010BD002010BDF40901082DE9F84F70
:104310000B78D0F800902F2B0C46824641D05C2BB6
:104320003FD0D9F81430836023781F2B43D90AF18A
:1043300020080AF12B062025434603F8015BB3420F
:10434000FBD123782E2B3ED00027384604F1FF3EC8
:104350004FF0080C1EF8013F202B00F1010040F245
:10436000C9802F2B4AD05C2B48D02E2B3AD0BC458D
:1043700035D91A063DD4222B31D06D4901E09A423D
:104380002DD011F8012F002AF9D1A3F16102192AC9
:1043900001D8203BDBB208F807300137DAE714F820
:1043A000013F2F2BFBD05C2BF9D00023CAF808303B
:1043B00023781F2BBBD880238AF82B305046BDE8CA
:1043C000F84F09F01BB88AF8203063782E2B40F0A4
:1043D0009E808AF82130A3782E2B40F09280062010
:1043E000BDE8F88FBCF10B0FF9D008274FF00B0C8C
:1043F000B0E703F07F034F4AD35CBCE72044044698
:1044000010F8012B2F2AFAD05C2AF8D0002FE6D022
:104410009AF82020E52A04BF05228AF82020202BC4
:104420008CBF002304238AF82B305046DAF8007042
:1044300008F0E4FF60BBDAF818103846FFF7FEFE1C
:1044400030BBDAF81C201378002B49D092F80BC04F
:104450000CF03F038AF80630D37A1B0712D4964635
:104460009AF820101EF80B3B01325B1A0AF1210169
:1044700043B912F8013B11F801BB9645CBEB03039E
:10448000F6D1A3B100215046FFF722FD0028D2D07B
:1044900004289AF82B302FD198063CD559077FF580
:1044A0004BAF80238AF82B300020BDE8F88F9AF8B4
:1044B0002B305B072DD41CF0100F1FD0DAF8103012
:1044C00099F8001009F13402C3F3080313440329D7
:1044D000D87E9A7E42EA002205D0CAF808202BE74F
:1044E0009AF82B30D8E7597D1B7D43EA012342EA35
:1044F0000342F2E7044489E7BDE8F88F0520BDE8F0
:10450000F88F03222F2B0BD1144420238BE7022298
:10451000F8E7BDE8F88F5A07F0D50420BDE8F88F1A
:104520005C2BF1D0202B3FF65AAF144424237AE7BA
:10453000FC09010874090108044B054A1B6803FBC8
:1045400000F010601368002BFCD1704714000020AD
:10455000D8230020064B074A1B68012B18BFB0FB6D
:10456000F3F0013010601368002BFCD1704700BFDE
:1045700060000020D8230020034B1A6812B11A688B
:10458000013A1A60704700BFD823002030B42B4B8B
:1045900099891A888C0602D592B2900623D4274AAC
:1045A0009189138809069BB201D51B0601D430BC42
:1045B00070474FF67F73224913800B68002B31D070
:1045C0002048214B02689B5C0132802A026004BFB4
:1045D000002202600A681948DBB29BB2013A0A6005
:1045E000838030BC70474FF6DF71184A19809B8872
:1045F00012689BB212B9DAB2032A1AD0144A1168AF
:104600007F29CCD81349144D0C68DBB2601C2B55A4
:104610007F2888BF0023086088BF0B6013680133C0
:104620001360BCE70D4A136823F08003136030BCAD
:1046300070470B4A01211160E0E700BF00440040D1
:10464000DC230020E42300205423002078000020F5
:10465000D4080020D4230020500100200C44004046
:10466000E02300200E4A13687F2BFCD830B40D4B9A
:104670000D4D1C68611C7F291960C0B288BF0021E4
:10468000285588BF196072B613680133136062B68B
:10469000064A136843F08003136030BC704700BFC4
:1046A000DC23002050230020542300200C44004031
:1046B000034B5B6B034214BF01200020704700BF17
:1046C000002C0140044B82B003440022019201936C
:1046D000019B186802B07047142C014010B4214CA3
:1046E000A36803F00C03042B1BD0082B1CD01E4B1B
:1046F00003601C4A1D499468C4F303140C5DE34035
:1047000043609468C4F382240C5D23FA04F484604B
:1047100092685DF8044BC2F342328A5CD340C360B6
:104720007047134B0360E4E76368616813F4800F1C
:10473000636818BF0E4C01F03F020CBF0A49B4FB7E
:10474000F2F1C3F3881308BFB1FBF2F101FB03F2EE
:10475000044B5B68C3F3014301335B00B2FBF3F32B
:104760000360C6E7003802400024F4007C0000200B
:1047700000127A000022F0B513460126032704E058
:104780000133102B02F102022FD00D6806FA03F458
:1047900034EA0505F4D1D0F800E007FA02F5ED435C
:1047A0000EEA050EC0F800E091F804E0D0F800C071
:1047B0000EFA02FE4EEA0C0EC0F800E091F804E09A
:1047C0000EF1FF3EBEF1010F07FA02FC0ED9C468DC
:1047D00024EA0C04C460CC79C568944001332C43AE
:1047E000102BC46002F10202CFD1F0BDD0F808E076
:1047F00005EA0E05856091F805E085680EFA02FE6F
:104800004EEA05058560456825EA040444608C7914
:1048100045689C40A4B22C434460D8E7F0B4114BE7
:104820004578D968827807780F4EC943C1F30221D1
:10483000C1F10404E4B20F2305FA04F40B41E4B21D
:1048400013402343F2191B01DBB282F800330378D3
:10485000012203F01F015B098A4046F82320F0BCC7
:10486000704700BF00ED00E000E100E02DE9F84FE7
:10487000914D924E2888431C9BB22B80F15CA1F194
:1048800040027B2A00F2B485DFE812F045043F04C1
:104890003A04350418049A007C00BE03B903B3033C
:1048A000AE03E10218049A007C00920080037A03B0
:1048B000DC02D70218049A008700B6019E03980311
:1048C00093038E0318049A00AB009200A903A3037C
:1048D000AD05A80518049A007C00220598059205EC
:1048E0008903850318049A007C00E704C904750352
:1048F0004003030318049A008700B20570033A02CC
:104900008301FB0018049A00AB00B205B205B205A2
:10491000B205B205B205B205B205B205B205B205DF
:10492000B205B205B205B205B205B205B205B205CF
:10493000B205B205B205B205B205B205B205B205BF
:10494000B205B205B205B205B205B205E602ED0147
:10495000C2015B01B205B205B205B2052201B60083
:10496000B2049504B205B205B205B2054A04530576
:1049700017022203B205B205B205B2054002960243
:10498000CA03ED034E494F4C0A68831C08320026C7
:104990002B800A602670BDE8F88F4949494C0A68A7
:1049A000831C083201262B800A602670BDE8F88F30
:1049B00043490A68831C09322B800A60BDE8F88FDE
:1049C000414F3F4C3B882268F15C581C80B2023357
:1049D000305C3B800E3241EA00232B802260BDE830
:1049E000F88F3749374C0A68831C083202262B801F
:1049F0000A602670BDE8F88F344C3148677994F826
:104A000004800268E17947EA0828103216F8087035
:104A1000026007F00F0E01F00F0026786278CEEBEF
:104A20000000C91BC0068FB242EA062600F1788555
:104A3000A27902F0EF02A27139064CBF42F0800267
:104A400002F07F02A27108F1FF30711E80B289B2BC
:104A5000060A6071080A2070267161701B480029DF
:104A600040F03E8502F0FB028271002F00F0458588
:104A700002F0BF0242F002020133A2712B80BDE8B6
:104A8000F88FC31C821C9BB292B2F15CB35C0C4FDA
:104A9000DFF834E03A6803EB01239BB25C1CA4B25C
:104AA000F15C345D031D01EB042114322B80AEF860
:104AB00000103A60BDE8F88FD8080020A825002033
:104AC00084420120D8010020F0020020744201201D
:104AD000B44FB54C3968B54AA37894F803E0B2F8FE
:104AE00000C094F8008062781031396027796179CC
:104AF0004EEA032341EA07219C459CBF775CF754AB
:104B000042EA08225E1E0139531E8AB2B6B29BB237
:104B1000170A6271A44A63704FEA162E190AE670EA
:104B200084F802E0277121709279002B00F0E18473
:104B300042F0040222F01202831CA2712B80BDE815
:104B4000F88F994CDFF85CE262792779DEF8003063
:104B50006178207842EA07271033F25DCEF8003002
:104B600006F0B4FB2378A279013BDBB22370002B63
:104B700000F0D28402F0BF027B1C29889BB2180A85
:104B800042F00202013163712071A2712980BDE8F7
:104B9000F88F854CDFF81C822079B8F80020DFF808
:104BA00004E26179A379DEF8006041EA002103F0B4
:104BB000010CC2F30B076744C1F30B0038440F36F6
:104BC0008F18CEF80060C604674400F1BB8423F060
:104BD0001003A371384606F0B7FA3B0A3846237132
:104BE000677106F065FAA2792B8822F00202013380
:104BF000A2712B80BDE8F88F6A496D4C0A686A4B38
:104C00002478DC710932831C2B800A60BDE8F88FA0
:104C1000644F654C3A68637994F804E061782078D1
:104C200010323A6043EA0E2706F0AEFA5F4B227864
:104C30001B88BB4298BFF0555B487B1C9BB2013A76
:104C4000190AD2B26371217122708379002A00F0AF
:104C50004C8403F0BF032A8843F002030132A3719E
:104C60002A80BDE8F88F504C4E49607994F8048052
:104C70000A68E77940EA0828103216F808000A6046
:104C800000F00F0E07F00F0126786278CEEB0101DD
:104C90003F1AC806BFB242EA062600F14784A2794D
:104CA00002F0EF02A27139064CBF42F0800202F01E
:104CB0007F02A27108F10100C7E63B4C394F94F81E
:104CC000049063792078DFF8E48043EA0929617869
:104CD00006F05AFAB8F80020334B4A4598BF06F858
:104CE00009002078013809F10102C0B21FFA82F9E7
:104CF0002070002800F0D8833B6815333B60E6E75E
:104D0000294BD879BDE8F84F04F02CBC264CDFF8CD
:104D10009CE094F8009094F8018094F802C0E27846
:104D2000637921791F4FBEF800B0D7F800E048EA58
:104D3000092942EA0C22C9EB020A43EA01211FFABF
:104D40008AFA0B465A4503F1FF3C02F1FF3824BFB3
:104D5000F35CB3541FFA88F252451FFA8CF3F1D179
:104D600009F1FF339BB294F806C0E270C9EB010170
:104D700003EB430389B2C3EBC3030EF110061E44D9
:104D80004FEA112E831C120A2CF0160061710021CB
:104D900084F804E03E602B80A270A07121706170E5
:104DA000BDE8F88F84420120744201208042012036
:104DB00000090020F0020020BA4CDFF8ECB2A27922
:104DC00094F80090617894F80480637922F04002AE
:104DD000A27141EA092943EA0828A24616F8087098
:104DE000E27907F00F0002F00F0108F1FF33091A12
:104DF00009F1FF39D21B1FFA83F8CB061FFA89F994
:104E000097B200F168839AF8063003F0EF038AF84E
:104E1000063017F0800F03F07F02A24963F07F0392
:104E200000F01583A371B9F1000F00F0FF82DBF8E9
:104E300000301533CBF80030D0E70120BDE8F84F43
:104E400004F0A6BB0120BDE8F84F04F019BD002016
:104E5000BDE8F84F01F002BB934F924C3968934A7A
:104E6000A37894F803E0B2F800C094F80080627868
:104E700010313960277961794EEA032341EA07212D
:104E80009C459CBF775CF75442EA08225E1C0131C6
:104E90003AE6831CC21C844C844992B29BB2B75C34
:104EA000F35C2268098803EB07231432804F2260E9
:104EB0009BB2804C3A888B4228BFE25401339BB2AC
:104EC00099429CBF120AF254031D2B80BDE8F88F53
:104ED000744C754F94F804806379207843EA08286D
:104EE00016F808206178DFF8BC9106F0EFF9207819
:104EF000013808F10108C0B21FFA88F820700028B4
:104F000000F080823B6815333B60E9E7654C684FF1
:104F1000637921793A88DFF890C194F806E0DCF8EB
:104F2000000043EA0121C2F30B06C1F30B039B1BF4
:104F30000EF001069B1BC2EB01080F30DB04C6EB31
:104F40000806CCF8000000F10B832EF01003A371CB
:104F5000D243304692B206F0F7F8330A3046667113
:104F6000237106F0A5F8A2792B8883E50720BDE818
:104F7000F84F01F03DBF0020BDE8F84F04F0F2BA51
:104F8000484B9878BDE8F84F04F0ECBA0220BDE831
:104F9000F84F01F02DBFBDE8F84F01F005BA02202F
:104FA000BDE8F84F06F0BABA0120BDE8F84F01F0AD
:104FB00055BA0120BDE8F84F06F0B0BA394BD878A1
:104FC000BDE8F84F04F0CEBA0320BDE8F84F01F079
:104FD0000FBF344B1879BDE8F84F04F0C3BA042072
:104FE000BDE8F84F01F004BF0020BDE8F84F06F01F
:104FF00095BA2C4B5878BDE8F84F04F0B3BA0120AD
:10500000BDE8F84F01F0F4BE2749264C0A682A4B48
:10501000E4791C700932831C2B800A60BDE8F88F8C
:10502000204C214F94F8049063792078DFF87C803D
:1050300043EA0929617806F0A7F8B8F80030194A60
:105040004B4598BF06F809002078013809F1FF3375
:10505000C0B21FFA83F92070002800F014823B6868
:1050600015333B60E6E70F4C0F4F94F804806379EB
:10507000207843EA082816F808206178DFF82490A1
:1050800006F024F92078013808F1FF38C0B21FFA81
:1050900088F82070002800F0B5813B6815333B602C
:1050A000E9E700BF744201208442012080420120D0
:1050B000F0020020A825002000090020C249C34CAE
:1050C0000A68E3790832802B0A6000F035825E427C
:1050D0001A07B6B240F04082A27922F01002A27103
:1050E000DA433046D2B2002106F03EF83046E6718F
:1050F00006F00EF837E70020BDE8F84F04F048BA94
:105100000020BDE8F84F04F0BBBBB04B1878BDE8F9
:10511000F84F04F027BA0020BDE8F84F01F068BE50
:10512000AA4CDFF8ACE294F8009094F8018094F86F
:1051300002C0E27863792179A34FBEF800B0D7F8B6
:1051400000E048EA092942EA0C2209EB020A43EA94
:1051500001211FFA8AFA0B465A4503F1010C02F1AC
:10516000010824BFF35CB3541FFA88F252451FFABA
:105170008CF3F1D109F1FF339BB294F806C0E270D1
:10518000494403EB430389B20EF11006C3EBC3039A
:1051900033444FEA112E0230120A2CF016066171C8
:1051A000002184F804E03B602880A270A671217081
:1051B0006170BDE8F88F854CDFF80CE262792779E1
:1051C000DEF800306178207842EA07271033F25D7C
:1051D000CEF8003006F07AF82378A279013BDBB2F2
:1051E0002370002B00F0958102F0BF027B1EC4E407
:1051F000754F764C3A68637994F804E061782078CA
:1052000010323A6043EA0E2705F0BEFF704B227859
:105210001B88BB4298BFF0557B1E6C480EE56A4A5E
:105220006A4E1368717830780C33136005F0ACFF68
:10523000044680B205F058FF664AB379125D23F048
:105240000201B171002A40F0938123F00603B3718B
:105250002B8801332B80BDE8F88F5C4C5A4F627964
:105260005B482179B0F800E042EA01213A68765CB7
:1052700002F112008E453860E279574F04D802F0EF
:105280000F0040EA0610785422F00F0242EA16128C
:1052900052B24E4ED0B2E071B179002840F0358163
:1052A00041F04001B171002A4A4A125CB4BF61F07A
:1052B0007F0101F07F01A171002A35D1A27902F0AE
:1052C000FB0222F012020133A2712B80BDE8F88F9D
:1052D0003E4C3D4862793E492779B1F800E0DFF85D
:1052E000F8C042EA07270268BE4502F112010160D8
:1052F000F25DE17906D801F00F00160946EA0010C8
:105300000CF8070021F00F0102F00F020A432F49A9
:10531000E2718879002A40F0F48040F04000887102
:105320002C498A5C002AC9D008F0A2FCA2792B88FB
:10533000C7E7264CDFF890B0A27994F80090617826
:1053400094F80480637922F04002A27141EA0929AD
:1053500043EA0828A24616F80870E27907F00F0021
:1053600002F00F01091AD21B09F1FF3908F10103FC
:1053700097B2CA061FFA89F91FFA83F800F1A680CE
:105380009AF8063003F0EF038AF8063017F0800F22
:1053900003F07F020D4963F07F0370D0A371B9F170
:1053A000000F43D0DBF800301533CBF80030D2E7E4
:1053B000064B5879BDE8F84F04F0D4B80520BDE895
:1053C000F84F01F015BD00BF844201207442012056
:1053D00080420120C0040108A82500200220BDE869
:1053E000F84F04F0D5B80220BDE8F84F04F048BAF1
:1053F00061480AF0A1FD614B1B689868BDE8F84F51
:1054000008F01CBE396899F806202B8889F80580B9
:1054100010314FEA182842F04202013389F8048023
:10542000396089F806202B80BDE8F88F544984F84C
:1054300005800A6884F800904FEA1823103223711F
:1054400084F801900A60A37903F0FB0303E4A271DE
:10545000002F7FF4E8AC42F040034FEA18264FEAF1
:1054600019208B7181F805800E7181F80190087008
:1054700042F04403B9F1000F7FF4EDABE3E7A27112
:10548000002F8CD1E7E73C689079298882F8059055
:105490004FEA1923103440F04200013113713C608F
:1054A00090712980BDE8F88F386899792A8883F847
:1054B000059010304FEA192941F04201013283F87A
:1054C0000490386099712A80BDE8F88F08F0D8FB05
:1054D0009AF806305AE708F0D3FB9AF8063098E4B9
:1054E00042F004028271FFF7C0BA43F04003FFF7B5
:1054F000B2BB02F0FB02FFF71DBB42F04002FFF718
:10550000B9BA20F0400088710AE701F0BF01B1711B
:10551000C9E642F0400269E642F04002FFF72CBBC8
:1055200008F0AEFBA2792B88FFF786BA08F0A8FB3B
:10553000A2792B88FFF7B7BBA2794FF6807642F0AD
:105540000402CAE508F09CFB21796379B8F80020D1
:1055500043EA0121FFF73EBB08F092FBE379BFE588
:1055600008F08EFB217963793A8843EA0121EFE460
:1055700008F07EFB6CE600BF0C0A01082001002049
:10558000844201202DE9F04F00238FB00B600C46C0
:10559000FEF7AAFA002813DB784B53F820509DB190
:1055A00025602B781BB16B78002B00F0D480C0B243
:1055B000002368702B7058B103200FB0BDE8F08F46
:1055C0000B200FB0BDE8F08F0C200FB0BDE8F08FBE
:1055D0006B4B6C4E596A706041F400615962596AB4
:1055E000694AB06021F40061596230605368674FC6
:1055F000674CF06023F4FD4323F07F0343F0760310
:1056000053600321012311603B6076224FF48063D5
:1056100023613061327520606060A060E06007F057
:10562000B9FE4FF480330893089B2BB909E0089B1F
:10563000013B0893089B23B18020FFF739F800282D
:10564000F5D0089B002BB7D04F4F40F2FF53BB6300
:105650004FF4D57308204021002223604FF480636B
:1056600023616060A160E26007F094FE4FF4803334
:1056700009937B6B13F0450F0CD1099A52B139464F
:1056800001E0099A32B1099B013B09934B6B13F07E
:10569000450FF6D0099A12B1580740F1FF833A4BF3
:1056A00004229A6300274FF0370840224FF48063AA
:1056B0002760E760C4F80480A260236107F06AFEF7
:1056C0004046019706F092FD0023372740214FF412
:1056D00080622360E3606760A160226107F05AFE88
:1056E000384606F083FD00287FF466AF284FDFF8C8
:1056F00098A00695804600234FF037094FF0400BE5
:105700004FF480652360E360C4F80490C4F808B0E7
:10571000256107F03FFE484606F068FD00287FF44B
:105720004BAF019BC7F808B043F0004343F480132C
:105730002922F8603D613B607A6007F02BFEDAF8C1
:10574000340010F0450FFAD010F0040005D00E4BD5
:1057500004229A6330E718462FE740F2FF53CAF855
:105760003830FEF7AFFF002808F10108064B11DBC7
:105770004FF6FF739845BED11EE700BF4C230020B3
:105780000038024070240020002C0140A0802542F7
:105790005C4201204FF6FF729045069D3FF40CAF2E
:1057A000420040F1AB82DFF8A8830222C8F8002053
:1057B0001B689F073FF400AF914600230221C022DF
:1057C0002360E3604FF480636160A260236107F0AF
:1057D000E1FD02F071F900287FF4EEAEFEF772FFF2
:1057E000D64F38600420FEF76DFF78600820FEF782
:1057F00069FFB8600C20FEF765FFB9F1020FF86091
:1058000003D9B9F1060F40F0EE83002340220321B3
:105810002360E3604FF48063A2606160236107F05E
:10582000B9FDC74A536B13F0450FFBD058078ED410
:1058300013F0010040F0D083C14A1369DBB2032B9F
:105840007FF4BAAE40F2FF539363FEF73BFF10F4D0
:10585000604F7FF4B1AE030CBA4A0692190413608C
:105860000922C0236260A36000224FF4806321609C
:10587000E260236107F08EFD02F01EF900287FF43C
:105880009BAEB14B0193FEF71DFFAF4B8146042049
:10589000C3F80090FEF716FFAB4B58600820FEF7E8
:1058A00011FFA94B98600C20FEF70CFFA64BD860A7
:1058B0000023A34833604268337522F4FD4222F08E
:1058C0007F024260019AA1495268D8F80080736053
:1058D0004FEA196E5FFA8EF04FEA901A4FEA126C97
:1058E00081F800A0C9F3074BC9F3072A4FEA0C1C43
:1058F000CEF3830E00F003005FFA89F981F801E02E
:10590000887081F803B0069881F804A081F80590AA
:10591000A1F806C0B1F806C0D0F800B0B360100A14
:10592000C2F307491FFA8CFC5FFA80FE4CEA191C8F
:105930004FEADE1A09F00F09A1F806C0B8F1010F0D
:1059400081F80890C0F3801C81F809A0C0F34019C9
:10595000C0F3001A81F80AC0F36081F80B9033613C
:1059600081F80CA081F85680A1F854B0DFF8D8C1B6
:105970004B7340F2D582B8F1020F00F09B82DCF845
:105980000800019A4FEA4E0303F07E03CEF3801E17
:1059900081F819E0D2F80CA08B7691F81AE03A68F9
:1059A0004FEA1A63C0B24EEAD01E4FEA830C00F0F1
:1059B0007F0081F81AE00CF00C0CC8764FEAD31E79
:1059C000C3F34110C3F3820381F81CE048778B775F
:1059D00081F81FC091F81FE04FEA1A4C5FFA8CF96A
:1059E0004FEA1A234EEA991ECCF3401C81F81FE0BF
:1059F00009F0010981F820C05FFA83FE4FF0000C26
:105A000081F821C081F822904FEADE1981F82390B5
:105A1000C3F3801981F82490C3F3401981F82590CD
:105A2000CAF34600C3F30019C2F3074AC3F3810364
:105A300081F826904FEA0A2A81F827300EF0030EEB
:105A4000130E4FF0010981F828E081F8290081F850
:105A50002A9081F82C30A1F82EA0CB8D7868DFF841
:105A6000F4A01FFA83FEC2F307234EEA03031206D3
:105A7000CB850A630A6B4FEA106E42EA0E420A6354
:105A80000B6BC4F80CC04FEA102C0CF47F4C4CEAA2
:105A900003030B630B6BBA68FF68C0F3072C4CEA77
:105AA000030C4FEA124EC1F830C04FEA0E634FEAC2
:105AB000126CC0B281F8340081F835C08B63886BFA
:105AC0004FEA022E0EF47F0E4EEA00008863886BC8
:105AD000120202F47F4202438A638A6B42EA17622F
:105AE0008A6391F83CE03A0CC2F3031012024EEACA
:105AF000000002F4706281F83C00CA87CA8FC7F3C5
:105B0000072E92B24FEA0B4042EA0E024FF0070B0B
:105B1000C7F3460E40234FF48067CA87206081F8A0
:105B200040E0C4F804B0A36081F84190276107F019
:105B300031FC584606F05AFB0EE000BF5824002006
:105B4000002C0140043C012048240020F0230020C8
:105B50006C2400205C42012000287FF42DADB8F1B8
:105B6000030F3FF429ADB8F1020F00F2BA80FEF73F
:105B7000A9FD10F000707FF41FAD4FF0100B402313
:105B80004FF008080A900B90CAF80C00CAF80830C9
:105B9000CAF810708AE8000907F0FCFB584606F0C6
:105BA00025FB00287FF408AD069BCAF80C001A6894
:105BB000CAF8107002FA0BF240234FF0370B8AE854
:105BC0000408CAF8083007F0E5FB584606F00EFB5B
:105BD000834600287FF4F0ACC84A30204FF0FF33F2
:105BE0000221C2F8048013609060C2F810B0C2F8BD
:105BF00014904FF03308D16007F0E6FB4023CAF859
:105C000000B0CAF80830CAF80CB0CAF81070CAF868
:105C1000048007F0BFFB404606F0E8FA00287FF456
:105C2000CBACDFF8DC820DF12409C24604E0FEF7BC
:105C30003FFD002840F0D981D8F83420B04F40F221
:105C40002A6313404FF40010002BF0D00820FEF719
:105C50002FFD002800F013820823BB63ACE440F260
:105C6000FF53BB630A9B1BBA59037FF5A5AC069B88
:105C7000E0601B684FF0370A1B044FF040094FF4F7
:105C8000806884E80804C4F80890C4F8108007F01D
:105C900081FB504606F0AAFA9A4B00287FF48CACA0
:105CA00002220624D860C3F80890C3F8108083E865
:105CB000140007F06FFB204606F098FA00287FF4E6
:105CC0007BAC30607B68307523F4FD4323F07F03A9
:105CD00043F400634FF400627060B06030617B6039
:105CE000F26000212846FEF7C9FA02281AD00428DB
:105CF00038D0012840F200810D205EE41B689B072C
:105D00003FF45AACDFF81082D8F80090B9F1040FD4
:105D10007FF453AD7C4B0193D3F800907B4B7C4FC9
:105D20000693C5E50AAC264605F5FE7005F50F7726
:105D300010F8063C43B1018810F8012C10F8023C21
:105D400042EA012243EA02231030B84246F8043BFB
:105D5000EED10EAF54F8046B36B90320A742F9D147
:105D60000428C9D1012028E431462846FEF786FAE6
:105D70000128F3D895F8402095F83F3043EA0223F4
:105D8000B3F5007FB8D195F84B1095F84A3053EA37
:105D9000012340F02681B5F85A1095F8593095F84E
:105DA000582043EA012342EA032195F84470E9614F
:105DB0007B1E012BAF709FD895F841309AB201FB42
:105DC00007F76A81002A97D05A1E1A4294D195F893
:105DD000452095F8464042EA042422072C818BD1C5
:105DE00095F8480095F8472052EA002209D1B5F805
:105DF00056E095F8550095F8542040EA0E2042EA06
:105E0000002295F843E095F8420050EA0E203FF456
:105E100073AF00EB141EBE447245FFF46DAFDFF8A4
:105E2000FCC0CEEB0202B2FBF3F35A1E62453FF612
:105E300063AF4FF6F572934200F2EC8040F6F572D4
:105E4000934200F2D780023330440EEB0602AB617E
:105E50006862EA622E62002C3FF44EAF03EB43020D
:105E6000384403F0010303EB5203A862012203F25A
:105E7000FF13B1EB532FFFF43FAF4FF0FF338021FF
:105E80002B61EB60297123492A700B8801339BB287
:105E900000200B80EB806861FFF78FBB590602D5AD
:105EA000174B40229A631C4B01221A604FF080432B
:105EB000019309E4130403F47C130B61DCF808007C
:105EC0000B69020E43EA02230B610B69C0F3074220
:105ED00013430B610A690023013243F10003DB0421
:105EE00043EA52334FF4007CD204CB648A64C0F39B
:105EF000072EC1F850C044E500263BE7143C0120C2
:105F0000002C01405C42012048240020043C012078
:105F100058240020682400206C240020F4FFFF0F88
:105F2000830203F440630B610B69DCF80800920004
:105F300002F47F7213430B61D1F810C0020E030C00
:105F40005FFA82FE4FEA43094CEA9E1C0EF0070AF4
:105F500009F00609C2F3C20EC3F34212C3F382036F
:105F6000C1F810C081F814E081F815A08A75CB75CE
:105F700081F818900B7EC0F3072E43EADE130B76F0
:105F80000B6907930B7E91F808904FF0010C0233D8
:105F90000CFA03F30CFA09FC4FEAE37AA3FB0C2397
:105FA000CDE90423CDE90223079BC1F850C003F1DA
:105FB0000109059B0CFB0A330393029BA3FB0923F6
:105FC000CDE90423059A039B09FB03230593DDE92F
:105FD0000423C1E91223D4E45A4B01229A63FFF748
:105FE000EBBA1946E1E6012336E4DAF8803049F8E5
:105FF000043F21E6023330440EEB0602AB616862D7
:10600000EA622E62002C3FF477AE3844A8625B004F
:1060100002222CE795F85F7095F85E202E6202331D
:106020003044B64452EA0722AB616862C5F82CE0FE
:106030007FF462AE002C7FF45FAEB5F8627095F825
:10604000610095F860209B0040EA072003F2FF13EF
:1060500042EA0022B1EB532FAA62FFF44DAE95F84D
:10606000651095F8643043EA01234FF0FF32802138
:10607000012B2A61EA6029710AD0032203E702207A
:10608000FEF716FB002849D00223BB63FFF794BA42
:10609000711C2846FEF7D2F80028EED195F833227D
:1060A00095F832322C7143EA02234AF65522934284
:1060B000E3D1E88E95F8352095F83430224942EA4C
:1060C000002243EA02238B42D7D1B5F81A0295F891
:1060D000192295F8183201F1FF5101F5005142EAF9
:1060E0000022203143EA02238B42C6D1B5F81E625A
:1060F00095F81D02B5F8224295F8211295F81C2258
:1061000095F8203240EA062041EA042142EA0022C2
:1061100043EA01232A61EB600322B4E62020FEF764
:10612000C7FA18B12023BB63FFF746BA4FF40070DB
:10613000FEF7BEFA00283FF492AD4FF40073BB6344
:10614000FFF73ABA002C014052526141F0B5194BA9
:106150001B783BBB184B1B788BB9184F18493E680E
:10616000184C91F804E04A792388174D07363E60B1
:1061700042EA0E22AA5C0A5401332380F0BD104982
:10618000104C114D23888E7ACA7A0C4F01339BB282
:1061900042EA062215F903E03E687244133692B2D1
:1061A0003E60E7E70649074C074D23880E7A4A7A96
:1061B000EBE700BF8242012083420120844201209C
:1061C00074420120D8080020A825002010B41C4BE0
:1061D0001B78C3B11B4C031F012B226898BF0430EE
:1061E000A1F1040302F1080298BFC0B2012B2260A2
:1061F00023D9154A154C1388615C2154013313804F
:106200005DF8044B7047124B1B788BB10D4C031F8C
:10621000012B226898BF0630A1F1040302F10802A5
:1062200098BFC0B2012B2260E3D80631C9B2E0E7C3
:10623000044A136804331360DBE70431C9B2D8E7BA
:106240008242012084420120D808002074420120AB
:106250008342012030B4154B1B7873B1031F012B0F
:106260001DD91349134D0B88134C5A1C92B202339B
:10627000AA5C0B80225430BC7047104B1B784BB18A
:10628000031F012BEDD80E4A136806300B33C0B242
:106290001360E6E70A4A136807331360E1E7084A28
:1062A000136804300B33C0B21360DAE78242012076
:1062B000D8080020A8250020744201208342012034
:1062C00084420120F0B4204B1B78002B28D11F4BB7
:1062D0001F481B781F4C8BB903881F4E22681F4D27
:1062E000591C023389B29BB2775CF15C6F71013348
:1062F0000A32038029712260F0BC70470388164E71
:106300002268164D591C023389B29BB2775CF15C4E
:10631000EF7201330E320380A9722260F0BC704725
:106320000B480C4C03880C4E22680C4D591C023350
:1063300089B29BB2775CF15C6F7201330E320380DD
:1063400029722260F0BC7047824201208342012002
:10635000D808002084420120A82500207442012092
:10636000F0B50D4E0D4F32880D4C0E4D931C511C47
:106370009BB289B217F803E07B5C216803EB0E2324
:106380009BB2033205EB400732801A0A0A3105F846
:10639000102021607B70F0BDD8080020A8250020C7
:1063A000844201207442012070B4264C2649228880
:1063B000264E531C901C80B29BB20D5CCB5C307897
:1063C00003EB05239BB2002828D12148007890B91F
:1063D000581C80B2CB5C0E5C1E481F4D016803EB5D
:1063E00006239BB21E0A10312E716B7101600332BD
:1063F000228070BC7047581C80B2CB5C0E5C154884
:10640000154D016803EB06239BB21E0A1431AE72D0
:10641000EB7201600332228070BC7047581C80B25E
:10642000CB5C0E5C0B480C4D016803EB06239BB262
:106430001E0A14312E726B7201600332228070BC0E
:10644000704700BFD8080020A82500208242012004
:10645000834201208442012074420120F0B5114E94
:1064600011493288114C124D931C571C9BB2BFB27C
:1064700011F803E0CB5D03EB0E239BB25F1CBFB2B0
:10648000CB5CCF5D216803EB07239BB2033205EBA6
:10649000400732801A0A143105F8102021607B7001
:1064A000F0BD00BFD8080020A825002084420120AC
:1064B0007442012070B4114D114B2A889E7901233A
:1064C000D41803FA01F10232A4B292B2314010B1F1
:1064D000B1FA81F1490931B90A492A800B680733B9
:1064E0000B6070BC7047084B0648195D03680C339D
:1064F00042FA81F203602A8070BC7047D8080020FD
:106500007442012084420120A8250020F0B5DFF864
:1065100054C0114E114C3288DCF8003094F806E07B
:106520000F4F0A33541CA4B2CCF800300123951C41
:1065300003FA01F13C5DADB20EEA010110B1B1FA0E
:1065400081F1490911B903323280F0BD7B5D04EB62
:1065500003243480F0BD00BFD8080020744201201D
:10656000A82500208442012010B41B4B1B7823BBBC
:106570001A4B1B4A1B781B4893B91479537901684D
:1065800043EA042301339BB21C0A06315371147190
:106590000160154A1388013313805DF8044B70477E
:1065A000947AD37A016843EA042301339BB21C0A2C
:1065B0000A31D37294720160EBE7094A0948147AF0
:1065C000537A016843EA042301339BB21C0A0A315F
:1065D000537214720160DCE7824201208342012081
:1065E0007442012084420120D8080020F0B5214BDC
:1065F0001C7824B32049214A0B6892F809E0177AE5
:1066000017330B601E491F4B09881D881E484B1C01
:106610009BB2A94210F801C0C65C28BF00F801E097
:10662000AB4228BFC7540CBB184B1B78D3B982F8B8
:1066300005C01671164A138801331380F0BD134B41
:106640000D491B780D4A33B10B6892F80BE0977A2D
:1066500017330B60D6E70B6892F805E01779133310
:106660000B60CFE782F80BC09672E3E782F809C0AF
:106670001672DFE782420120844201207442012029
:10668000F002002080420120A82500208342012042
:10669000D808002010B41B4B1B7823BB1A4B1B4A95
:1066A0001B781B4893B914795379016843EA042392
:1066B000013B9BB21C0A0631537114710160154AEB
:1066C0001388013313805DF8044B7047947AD37AB2
:1066D000016843EA0423013B9BB21C0A0A31D372CE
:1066E00094720160EBE7094A0948147A537A016809
:1066F00043EA0423013B9BB21C0A0A315372147211
:106700000160DCE7824201208342012074420120C3
:1067100084420120D80800202DE9F041214D224B70
:106720002A889F79214E541CA4B2012302F1020E43
:1067300003FA01F1345D1FFA8EFE394010B1B1FA4F
:1067400081F1490931B3DFF870C0DFF86880BCF827
:1067500000301749D8F800000F8816F80EE0591ECF
:1067600089B211300332B94292B2C8F80000A3F1E5
:1067700002030E489BB224BF4FEA122800F80180A2
:106780009F42ACF8003098BFF25404EB0E232B80EC
:10679000BDE8F08107490B6803320A332A800B6099
:1067A000BDE8F081D808002074420120A82500200F
:1067B0008042012084420120F00200202DE9F843AC
:1067C0002F4B1B78002B38D02E4F2F4D3B88697AEA
:1067D000DFF8C4902D482C7A026801339BB241EA5D
:1067E000042419F903103B800C441732A4B2026050
:1067F00019F8048008F00F03013B08F1FF36DB06AF
:10680000B6B23AD4AB7923F01003AB71FE22414605
:10681000304604F0A9FC1E4B1B883046A34298BFAB
:1068200009F8046004F060FCAA793B8842F0020297
:106830000133AA713B80BDE8F883164B1B787BB10E
:10684000104F114D3B88AC7ADFF84C900F48E97A35
:10685000026801339BB241EA042119F90340C2E7FF
:106860000A4A094D13682C796979064FDFF8289098
:106870000B33136041EA0424BAE707F001FAC5E7D5
:1068800082420120D8080020744201208442012065
:106890008042012083420120A825002070B5214BB1
:1068A0001B7806462BB320490A68031F0832012BC8
:1068B0000A6033D91D4DAC5D04F00F03013B013C70
:1068C000DB06A4B227D4AB7923F01003AB71FE2210
:1068D000A95D204604F048FC2046AC5504F004FCB9
:1068E0001349AB790A8843F0020301320A80AB7185
:1068F00070BD104B1B784BB10B490A68031F08325F
:10690000012B0A60D6D80636F6B2D3E7064A1368DA
:1069100004331360CEE707F0B3F9D8E70436F6B2D4
:10692000C8E700BF82420120844201207442012056
:10693000D8080020834201202DE9F0412A4B1B7822
:10694000002B35D0294C2A4D2A482A882A4E277AEE
:10695000637A3168013292B243EA072387562A806C
:106960003B4413319BB23160C65CE179DFF87C8037
:1069700006F00F0201F00F039B1A8F1BDB06BFB25C
:106980002DD498F8063023F0100388F80630F2432F
:10699000D2B2384604F0E8FB384604F0B9FBA279DD
:1069A0002B8842F002020133A2712B80BDE8F081F6
:1069B000124B1B783BB10D4C0D4D0E482A880E4EE4
:1069C000A77AE37AC5E70C49084C0A682679637907
:1069D000074D084807320A6043EA0623C4E707F078
:1069E0004FF998F80710D2E7824201207442012043
:1069F000D8080020A82500208442012083420120DD
:106A000070B5234B1B78064643B322490A68031F1F
:106A10000832012B0A6037D91F4DE979AC5D01F0CE
:106A20000F0304F00F029B1A0C1BDB06A4B227D441
:106A3000AB7923F01003AB71AA5DD243D2B22046EA
:106A400004F092FB204604F063FB1449AB790A88FA
:106A500043F0020301320A80AB7170BD104B1B780A
:106A60004BB10C490A68031F0832012B0A60D3D8C6
:106A70000636F6B2D0E7074A136804331360CBE753
:106A800007F0FEF8E979D7E70436F6B2C4E700BFAD
:106A9000824201208442012074420120D808002053
:106AA0008342012070B52E4B1B7823B32D492E4C09
:106AB0000A68207A637A0F3243EA00235E000A6094
:106AC0001905354640D4A37903F0EF03320A667204
:106AD000227203F0FD02E8032349A27144BF42F091
:106AE00001028A71214A5CBF23F003038B71138872
:106AF0000133138070BD1E4B1B4C1B7819498BB1A1
:106B00000A68A07AE37A0F3243EA00235E000A6043
:106B10001A0535461CD4A37903F0EF03320AE67256
:106B2000A272D6E7207963790A6843EA00235E00FF
:106B30000B321B0535460A600ED4A37903F0EF0330
:106B4000320A66712271C4E707F09AF8A379BDE7AB
:106B500007F096F8A379E1E707F092F8A379EFE759
:106B6000824201208442012074420120D808002082
:106B70008342012070B5394B1B785BB3384C394BDD
:106B8000627A3948257A1B88016842EA0525C5F3EF
:106B90000B06C3F30B021D440F31B3180160D90477
:106BA0002E464FD4A37903F0EF032A0A65722272AE
:106BB00003F0FD02F0032A49A27144BF42F0010232
:106BC0008A712A4A5CBF23F003038B711388013357
:106BD000138070BD264B224C1B78CBB1214BE27A3F
:106BE000A57A1B88204842EA0525C5F30B060168F3
:106BF000C3F30B021D44B3180F31DA042E460160B3
:106C000024D4A37903F0EF032A0AE572A272CFE736
:106C1000144B627925791B88134842EA0525C5F390
:106C20000B060168C3F30B021D44B3180B31DB04E0
:106C30002E4601600ED4A37903F0EF032A0A657192
:106C40002271B5E707F01CF8A379AEE707F018F852
:106C5000A379D9E707F014F8A379EFE7824201207E
:106C600074420120F002002084420120D808002054
:106C7000834201202DE9F8432F4B1B78002B37D09E
:106C80002E4E2F4D3388697ADFF8C4902D482C7A28
:106C9000026801339BB241EA042419F903103380DE
:106CA0000C441732A4B2026019F8047007F00F0305
:106CB0000133DB0607F101083AD4AB7923F0100366
:106CC000AB7139460122404604F04EFA1E4B1B8838
:106CD000A342AB7998BF09F8048023F00203404631
:106CE000AB7104F001FA338801333380BDE8F883D7
:106CF000164B1B787BB1114E114D3388AC7ADFF8FF
:106D000050901048E97A026801339BB241EA0421AD
:106D100019F90340C3E70B4A094D13682C796979C7
:106D2000064EDFF82C900B33136041EA0424BBE7D6
:106D300006F0A6FFC5E700BF82420120D808002068
:106D400074420120844201208042012083420120BC
:106D5000A825002070B5214B1B7806462BB320498F
:106D60000A68031F0832012B0A6033D91D4CA55D48
:106D700005F00F030133DB0605F1010527D4A379E4
:106D800023F01003A3710122A15D284604F0ECF961
:106D9000A555A379284623F00203A37104F0A4F9B2
:106DA000114A13880133138070BD104B1B784BB10F
:106DB0000B490A68031F0832012B0A60D6D8063631
:106DC000F6B2D3E7064A136804331360CEE706F041
:106DD00057FFD8E70436F6B2C8E700BF8242012069
:106DE0008442012074420120D808002083420120FF
:106DF00038B5104A104C136861780C33054620787A
:106E0000136004F0C1F9605504F06EF9A3790B49E1
:106E100023F00202A271625D8A5C3AB923F0060394
:106E2000A371074A13880133138038BD06F020FF91
:106E3000F7E700BF8442012074420120C00401082A
:106E4000D808002010B52449244C0A68A3790432DC
:106E50000A60DA06E1792ED50622D80726D49929C8
:106E600024D803F01200022805D0122801F00F00E8
:106E700028D0092828D803F0EF03A3719B0789B213
:106E80004ABF8A1A521892B21046E27104F02CF9E5
:106E9000E3791349114ACB5CD3B9937923F0040306
:106EA0009371104A13880133138010BD6032D2B23F
:106EB00043F00103D5E701F00F02092A8CBF062237
:106EC0000022CAE70528D6D843F01003A371D5E7FE
:106ED00006F0CEFEE5E700BF8442012074420120A7
:106EE000C0040108D8080020F8B5274B1B78002BF8
:106EF0002CD0264C264D27482A88274E277A637A9D
:106F00003168013292B243EA072387562A803B4414
:106F100013319BB23160E279C35C1C4E13401846BA
:106F2000E37104F0E1F8A379E1791C4823F003024E
:106F3000415C42F01002A271F9B923F0070343F05B
:106F40001003B3712B8801332B80F8BD144B1B78D1
:106F50003BB10E4C0E4D0F482A880F4EA77AE37AAC
:106F6000CEE70D49094C0A6826796379084D09482E
:106F700007320A6043EA0623CDE706F079FE2B8844
:106F800001332B80F8BD00BF8242012074420120F2
:106F9000D8080020A825002084420120C004010850
:106FA0008342012010B51F4B1B7813B31E490A689A
:106FB000031F0832012B0A6030D91C4C235CE27994
:106FC00013401846E37104F08FF8A379E17918486B
:106FD00023F00302415C42F01002A271D9B923F000
:106FE000070343F01003A371124A1388013313807F
:106FF00010BD114B1B784BB10B490A68031F0832B7
:10700000012B0A60D9D80630C0B2D6E7064A136809
:1070100004331360D1E706F02BFEE5E70430C0B27D
:10702000CBE700BF8242012084420120744201204C
:10703000C0040108D808002083420120F8B5436845
:10704000013B002B04460E46436010DB0268511CD6
:1070500001601578013B002B636019DB23685A1C23
:107060002260187845EA002535800120F8BD0D4FD3
:107070000146386807F0F6FD421C054610D13B6812
:107080000948DB681D22012108F056FC0020F8BDEC
:10709000044F2146386807F0E5FD431CEFD0E1E7D7
:1070A0006368D7E720010020300A010870B5436803
:1070B000013B002B04460D46436006DB03685A1C67
:1070C000026018782870012070BD094E01463068B2
:1070D00007F0C8FD431CF5D133680648DB681D2264
:1070E000012108F029FC204606F0EEFE002070BDCC
:1070F00020010020500A01082DE9F04F85B00F460D
:107100000DF10E01924601939DF838908046FFF7ED
:10711000CDFF00285DD00F9B9DF80E509E1E6DBBCD
:10712000B9F1000F66D10DF10F09002E00F0A78014
:107130003A46AB460DF10F0913E0019BDBB1B2F506
:10714000804F18D35A4B9DF80F1099540BF101033F
:107150001FFA83FB01325E4592B285EA010540F2D7
:107160008E80494640460092FFF7A0FF009A0446F1
:1071700080B3DA45E1D89DF80F10E7E7B9F1000FC9
:1071800069D00DF10F09002E00F084804FF0000B44
:107190000DF10F0912E0019BC3B1B7F5804F15D374
:1071A000434B9DF80F20DA550BF101031FFA83FBC7
:1071B00001375E45BFB285EA02056BD949464046B4
:1071C000FFF774FF044628B1DA45E4D89DF80F2094
:1071D000EAE70446374D38482B6823220121DB6853
:1071E00008F0AAFB2B68D86806F028FF204605B0F7
:1071F000BDE8F08F002E57D02F460DF10F094946FC
:107200004046FFF753FF01370446BFB20028E1D0E4
:107210009DF80F30BE4285EA0305F0D800264946A6
:107220004046FFF743FF04460028D3D09DF80F30B7
:10723000AB4231D01F4C2148236823220121DB6857
:1072400008F07AFB2368D86806F0F8FE0024204690
:1072500005B0BDE8F08F26B34F460DF10F09494642
:107260004046FFF723FF01370446BFB20028B1D0E4
:107270009DF80F30BE4285EA0305F0D8CEE70C4BEF
:10728000DA5D3AB90E4A92F880201AB93B4480215F
:107290005A7399730126C2E73446204605B0BDE80B
:1072A000F08F0DF10F09BAE72E460DF10F09B6E781
:1072B000A825002020010020700A0108940A010876
:1072C000FC0300202DE9F04F89B0B34EB34D02927C
:1072D00082468946039300242968B04F4B68013BDE
:1072E000002B4B60C0F2AD810B685A1C0A60187805
:1072F000A0F11003202B00F29181DFE813F055017B
:10730000EC00D8008F0183008F018F018F018F0166
:107310008F018F018F018F018F018F018F01790004
:10732000340030008F018F018F018F018F018F0199
:107330008F018F018F018F018F018F018F017501E7
:10734000A346DBF8000082689368013B002B936042
:10735000C0F2B38113680A21581C10601970012013
:1073600009B0BDE8F08FD5F8008007A94046FFF7C7
:107370009DFE0028AFD09DF81C10894808F0DCFD68
:107380009DF81C30002B00F09C814FF0000B0DF19C
:107390001E070EE0DEF800305A1CCEF8002083F8FD
:1073A00000C00BF1010B9DF81C305FFA8BFB5B45B5
:1073B000C6D939464046FFF779FE774C00288AD077
:1073C00030689DF81EC0D0F808E0DEF80830013BB8
:1073D000002BCEF80830DDDADEF818209342614643
:1073E000724602DBBCF10A0FD4D107F0E9FFD8E7FF
:1073F0000DF11E012868FFF721FE002840F057819B
:10740000044669E72C680DF11A012046FFF716FEC5
:10741000002800F0348107A92046FFF70FFE00285E
:1074200000F02D8106A92046FFF740FE00283FF41A
:1074300052AF0DF11E012046FFF700FE002800F0BC
:107440001E810DF117012046FFF730FE00283FF4A2
:1074500042AF0DF1170120469DF81770FFF726FE89
:1074600000B30DF1170120469DF81780FFF71EFEAF
:1074700000283FF430AF9DF817304FEA082848EA5B
:10748000034858EA070818BF002702D10AE0B845A8
:1074900008D90DF119012046FFF708FE0137BFB2E8
:1074A0000028F4D13368986806F0C8FD13E72C680B
:1074B0000DF11E0720463946FFF7C0FD30B13946B1
:1074C0002046FFF7BBFD00287FF405AF3368354841
:1074D000DB682222D7E02C680DF11E0720463946D2
:1074E000FFF7ACFD00283FF4F6AE39462046FFF723
:1074F000A5FD00283FF4EFAE39462046FFF79EFD7C
:1075000000283FF4E8AE39462046FFF797FD0028F3
:107510003FF4E1AE39462046FFF790FD00283FF4E6
:10752000DAAE39462046FFF789FD00283FF4D3AE96
:1075300007A92046FFF7BAFD00283FF4CCAE394634
:107540002046FFF77BFD00283FF4C5AE6368013B92
:10755000002B6360C0F2B8802268511C216017784C
:10756000013B002B6360C0F2DA802268511C21606D
:1075700092F80080013B002B6360C0F2B08023686A
:107580005A1C2260187847EA082747EA004301930B
:10759000039B009320461DE020010020F8080020F6
:1075A000300B0108DC0A01082F680DF11E01384676
:1075B000FFF744FD044600286DD007A93846FFF7C1
:1075C0003DFD0446002866D0BDF81C30039A0092A9
:1075D00038460193029B4A465146FFF78DFD01282C
:1075E00004467FF479AEBAE62C6807A92046FFF777
:1075F0005DFD70B19DF81C305A1E0DF11E01204634
:107600008DF81C20002B3FF466AEFFF74FFD0028DD
:10761000F0D133684948DB681D2234E0484C4949C1
:1076200023680246D86808F027F92368D86806F06E
:1076300005FD286806F048FC0020286009B0BDE878
:10764000F08F3068DFF8F8B007F00CFB411C7FF4D6
:107650004FAEDBF800303C48DB681722012108F010
:107660006BF9DBF80030D86806F0E8FC386806F003
:107670002BFC002320463B6009B0BDE8F08F336847
:107680003248DB682222012108F056F93368D868B5
:1076900006F0D4FC1FE633682D48DB682222012166
:1076A00008F04AF93368D86806F0C8FC14E6BDF85B
:1076B0001E10284808F040FC51E60A2107F080FE21
:1076C0004DE6DFF87CB03CE61D4B306821469B461A
:1076D00007F0C8FA421C07462DD0636840E7184BF4
:1076E000306821469B4607F0BDFA431C7FF44BAF40
:1076F000134B1B68DB6818481D22012108F01CF998
:10770000DBF800301548DB682222012108F014F96B
:10771000DBF80030D86806F091FC0024DCE5084B6B
:10772000306821469B4607F09DFAB0F1FF3F804646
:10773000DED063681EE73368DCE700BF440B010856
:1077400020010020640B01088C0B0108000B0108CC
:10775000B80A0108240B0108300A0108A40B01082B
:1077600010B5044C206818B106F0AEFB002323606E
:1077700010BD00BFA42500202DE9F04385B00E46C2
:107780000DF10E011746984605469DF83090FFF71B
:1077900055FC78B1BDF80E400194CDF800904346F9
:1077A0003A4631462846FFF7A7FC0446204605B076
:1077B000BDE8F083084D2B68044622220121DB68D6
:1077C000064808F0B9F82B68D86806F037FC204660
:1077D00005B0BDE8F08300BF20010020B80A010811
:1077E000F0B585B0064601AC0DF10E0721463046D6
:1077F000FFF75CFC01340546C8B1BC42F6D101A8D4
:107800000722184908F0A6F80546F8B99DF80B209C
:107810001A2A08D0144B15491B68D86808F02CF8B0
:10782000284605B0F0BD0125284605B0F0BD0E4C38
:107830000F48236820220121DB6808F07DF82368C7
:10784000D86806F0FBFB284605B0F0BD064B09489A
:107850001B681622DB68012108F06EF80025284617
:1078600005B0F0BDEC0B0108200100200C0C010854
:10787000C80B0108F40B01083F49404BD1F88820A0
:107880003F4842F47002C1F888201A68002142F093
:1078900001021A6099601A6822F0847222F4803220
:1078A0001A6058601A6882B022F480221A60D96087
:1078B000009101911A6842F480321A6003E0009A44
:1078C000B2F5C06F09D01A6802F400320192009A32
:1078D00001320092019A002AF1D0284B1B6813F460
:1078E000003318BF01230193019B012B00D0FEE759
:1078F000224B24491A6C42F080521A640A6842F4FE
:1079000080420A609A689A609A6842F400429A60DB
:107910009A6842F4A0529A601A6822F080721A6043
:107920001968164A8801FBD4174B5360136843F05B
:10793000807313601168114B8901FBD5134A40F223
:1079400005711160126802F00702052A00D0FEE7F7
:107950009A6822F003029A609A6842F002029A60E2
:107960009A6802F00C02082AFAD1034B4FF0006229
:107970009A6002B0704700BF00ED00E0003802409E
:107980001030002400700040042A4007003C0240F0
:1079900070B4084B4FF0C045C0F30F242B26C1F341
:1079A0000F22C0B2C9B22E801C8018801A801980A4
:1079B00070BC70470000086070B4084B4FF0C045C1
:1079C000C0F30F242A26C1F30F22C0B2C9B22E8001
:1079D0001C8018801A80198070BC704700000860F5
:1079E000054B1A6812F0C05F05D0044901204FF022
:1079F000046208609A60704700640240902400208E
:107A000038B54FF48070FCF753FE38BB0220FCF70A
:107A10004FFEA8B90820FCF74BFE002830D12020EB
:107A2000FCF746FE28BB1020FCF742FE00282ED1B2
:107A30004FF40070FCF73CFE00282FD11B4904E0F6
:107A40001B4A1A49022393630B70194AD36B23F420
:107A5000434323F03A03D3630B7838BD13491448EA
:107A6000144B00254FF4807401220D7084631A605A
:107A7000EBE70F4A0D492020062390630B70E4E7E3
:107A80000B4A0A490820042390630B70DDE7084A7B
:107A900006491020052390630B70D6E7044A03497A
:107AA0004FF40070072390630B70CEE7882400200A
:107AB000002C01408C2400200A4A536B13F0450F20
:107AC000FBD05A0709D413F00100064B15BF012063
:107AD00040F2FF5298639A637047024B04229A6304
:107AE00003207047002C01400A44013811F8013B83
:107AF00000F8013F9142F9D1704700BF2DE9F04FE6
:107B000085B00C460391017802900093002945D07E
:107B100002F10803234D019304F10C060198B6F518
:107B2000F07FA0F1080730D2B0F5487F2DD21E4B70
:107B3000DDF80CB00C2202FB013202F1FF3A00F139
:107B4000FF394FF0C048494638461AF8014FFFF751
:107B500033FF58465946FFF71BFF2C23A8F8003087
:107B6000BDF838C0BDF800E00723012000FA03F299
:107B7000224214BFA5F800E0A5F800C013F1FF33BE
:107B8000F4D20BF1010BB345DDD1029B13F8011FB9
:107B90000293019B083301930029BFD105B0BDE8D2
:107BA000F08F00BF00000860340C0108012919D9CA
:107BB000F8B58269914208D20278022A06460C463C
:107BC00029D0032A10D0012A01D00120F8BD416A32
:107BD00004EB540501EB5521FCF730FB68B34FF083
:107BE000FF30F8BD01207047416A01EBD411FCF76A
:107BF00025FB0028F3D1A10001F4FE7106F1340346
:107C00005A185B5C5088527842EA002043EA002010
:107C100020F07040F8BD416A01EB1421FCF70EFB27
:107C20000028DCD1610001F4FF7106F134035A1819
:107C30005B5C507843EA0020F8BDC5F30803716A25
:107C40006F1C334401EB5721304693F83450FCF756
:107C5000F5FA0028C3D1C7F30803334493F834007E
:107C6000E30745EA00204CBF0009C0F30B00F8BD54
:107C70002DE9F84F0678022E04460D46174652D0DD
:107C8000032E2FD0012E04D04FF002084046BDE84D
:107C9000F88F416A05EB550901EB5921FCF7CEFA43
:107CA00080460028F2D1EB0709F1010B04F1340AF8
:107CB000C9F308094ED51AF8093003F00F0343EA57
:107CC00007130AF80930616AE67001EB5B21204670
:107CD000FCF7B4FA002847D1CBF3080BDA44C7F31A
:107CE00007174DE0416A01EBD511FCF7A7FA804672
:107CF0000028CBD1AD0005F4FE7504F134014B1919
:107D000027F070475A88120402F0704217434F550B
:107D10003E0A380C01223F0E98705E70DF70E270F0
:107D20004046BDE8F88F416A01EB1521FCF786FA61
:107D300080460028AAD16D0005F4FF7504F13403D4
:107D40005919C7F307205F5501224870E270404679
:107D5000BDE8F88F0AF80970616AE67001EB5B21F3
:107D60002046FCF76BFA08B180468FE7CBF3080B8F
:107D7000C7F303271AF80B2022F00F021743DA4447
:107D800001238AF80070E37080E700BF0EB42DE98C
:107D9000F04F8EB0179B03F00302012A43D0022A52
:107DA00035D032B14FF0FF300EB0BDE8F04F03B028
:107DB00070470126AB4D074600242B46D3F82822F6
:107DC00012F0010F03F50B730DD00134082CF5D11F
:107DD00006F00EF8172303604FF0FF300EB0BDE839
:107DE000F04F03B07047324601A968460097FDF78F
:107DF000C9FB00282FD04FF40B7000FB04F40023C4
:107E00002B5105F0F5FF4FF4FA630360CAE79C05B8
:107E10001BD413F4806F0CBF03260B2613F0080F3E
:107E200018BF3326C6E79D0509D413F4806F0CBF35
:107E300002260A2613F0080F18BF3226BAE713F4F9
:107E4000806F0CBF12260A26F4E713F4806F0CBF74
:107E500013260B26E2E79DE80A0002A80293FCF72E
:107E600055FA002872D19DF93330002BC3DB16F090
:107E70001C0F00F0D8809DF80E3013F0110FBAD10E
:107E8000300700F1F180DDF804E0DEF83010099BE6
:107E90004FF40B7202FB0452116253629EF8000011
:107EA000D97E9A7E032842EA012100F0D4804FF463
:107EB0000B7202FB04F2A81802F128078160597FB7
:107EC000B3F81EC01B7F45F802E041EA0C2243EAEA
:107ED0000223C360BEF80630838000222F4406745C
:107EE00007F500713B464274C261426103F8012B01
:107EF0008B42FBD1B10640F186804FF40B7909FB30
:107F00000459D9F80C60002E7DD0C9F81460BEF871
:107F10000A80D9F808104FEA482846454DD9C8EBE1
:107F2000060602E0464548D91E46D9F80000FFF78C
:107F30003DFE01280146C8EB060301D9421CF1D1E0
:107F40004FF40B7303FB0453996154E716F01C0FB5
:107F50003FF451AF04287FF44EAF02A8029F05F012
:107F60004DFA00287FF447AF08993846FCF766F9C8
:107F700000287FF440AF099B1B78E52B03D001213B
:107F800002A8002B62D108993846FCF757F900285F
:107F90007FF431AF099B024603F1200103F8012B66
:107FA0008B42FBD10B220AA90998FFF79DFD46F0F1
:107FB00008060123F6B2FB7062E74FF40B7000FB7A
:107FC0000450C6F308038161EBB1DDF804E0DEF88C
:107FD00018300239023B9942BFF40DAFBEF80A30A7
:107FE000DEF82C2001FB0322002A3FF404AF02EB51
:107FF0005622C2619EF8010039460123FCF706F8BB
:1080000000287FF4F8AE4FF40B7303FB0453E01C1D
:10801000D3F8282242F00102C3F828220EB0BDE8AE
:10802000F04F03B070479DF80E30D9063FF5E3AE30
:10803000B20702D5DF073FF5DEAE3007DDF804E01A
:108040007FF523AF46F04006F6B21EE7FBF740FF90
:10805000002889D0CFE6587D1A7D42EA002241EA05
:10806000024124E7702601200199099B0A78DF7EEE
:10807000987E032A40EA072770D0CB229A734220C9
:1080800050224FF0B20E5A7483F80FE01874099B17
:108090002022DA72099B00229A76DA760878032881
:1080A00004BF1A755A75099B002201201A775A7766
:1080B0009A77DA77C87017B9DDF804E0C2E7012FC4
:1080C0007FF699AEDDF80880D8F818309F42BFF4EB
:1080D00092AE019B4046D3F830B0B9462BE0012860
:1080E0003FF489AEB0F1FF3F3FF485AEB9F1010F27
:1080F0007FF681AED8F818309945BFF47CAE49467A
:1081000000224046FFF7B4FD00287FF474AED8F893
:108110001810D8F810308A1E934208D298F804201C
:10812000013342F00102C8F8103088F804208A4573
:1081300007D20298D1464946FFF738FD824600280B
:10814000CDD159460198FCF779F8DDF804E0013FFC
:10815000CEF80C7000283FF475AF4CE6587D1A7DC0
:1081600042EA002247EA024787E700BF70B500F104
:1081700034060446026B407831460123FBF764FD68
:1081800060B9216B636AE269E070CB1A93420546DD
:1081900002D2A378022B03D0284670BD012070BD07
:1081A0000A44607831460123FBF74EFD284670BD36
:1081B00038B1036813B11A783AB9134609200B6035
:1081C000704703460B60092070478088DA88904228
:1081D00003D0002309200B6070475A78002A16BF8D
:1081E000002300200920EAE7F0B583B00E4601A97C
:1081F0000446FFF7DDFF002864D1607C002861D1D0
:10820000E368B34204D2227C12F0020F08BF1E467C
:10821000002263696261002E56D0019A57897F025D
:10822000002B54D0013B721EB3FBF7F1B2FBF7F207
:108230008A424CD37A421340A2696361F61A12B3A0
:10824000BE426ED9F61B11E0FBF776FC0246002811
:108250007BD0531C59D0012A4AD9019B9B699A4271
:1082600046D2B742A2615BD26369F61B257C3B44D0
:10827000AD07114620466361E6D411462068FFF73A
:1082800095FC0246E5E71646E2689A4264D2227CF3
:10829000E36042F04002C3F308032274002B59D07C
:1082A000E269964235D094F91030002B24DB04F1BA
:1082B0002805019B2946587832460123FBF7A6FE84
:1082C00018BBE66103B0F0BD304603B0F0BDA26854
:1082D00012B10023A261B2E711462046FBF72CFC45
:1082E0000128024604D0431C0FD0A0606369F1E767
:1082F0000220607403B0F0BD019B04F1280558789A
:1083000029460123FBF7A0FC28B10120607403B0CB
:10831000F0BD0020D6E7237C03F07F032374C8E779
:1083200063693344C6F30800636188B101988169C9
:10833000023A02398A42DBD24189C06A02FB010259
:10834000002AD5D002EB56269EE7064663699BE7D6
:10835000064699E71846B5E7C3F308039EE700BF52
:108360002DE9F0471F4682B0002388463B6001A9F3
:1083700016460446FFF71CFF28B9607C18B9227C1A
:10838000910703D4072002B0BDE8F0876369F34288
:1083900028BFDE43F6B977E004F12809C0F500757F
:1083A000B54228BF354648442A464146FFF79CFB64
:1083B000237C63F07F0323743B682B443B60636939
:1083C000E2682B449A4238BF1A46761BA844636180
:1083D000E26058D0C3F308000028DDD1019AB2F85A
:1083E0000A9009F1FF3919EA53290DD1002B44D124
:1083F000A06800285FD001287BD0431C3AD0A36836
:10840000A061019A03B9A06094F91030002B43DBFE
:10841000A3699169023B02398B426AD25089D56ABD
:1084200000FB0353002B64D05FEA562A09EB0305D7
:1084300013D009EB0A03834288BFC9EB000A5346F5
:10844000507841462A46FBF7FFFB98B9E169491B82
:108450008A4541D84FEA4A25AEE7E36960699D4203
:1084600017D0E368984204F128092BD3E561C0F3E3
:10847000080093E70120607485E7A1692046FBF7B7
:108480005BFB0028B7D1227C42F04002227400201E
:1084900079E704F12809E9E75078E269012304F15A
:1084A0002801FBF7D1FB0028E4D1237C019A03F0DB
:1084B0007F032374ACE749462046FBF73DFB0028C9
:1084C00099D1E0E75078494601232A46FBF79EFD03
:1084D0000028CFD16069C9E708EB41214FF4007251
:1084E00004F12800FFF700FB237C03F07F032374D3
:1084F000B0E70220607446E72DE9F04F1E4683B0D6
:1085000000230F46336001A914460546FFF750FECD
:1085100028B9687C18B92B7CDA0703D4072003B08C
:10852000BDE8F08F6B69EA68C3EB0208A04528BF7D
:10853000A04605F12809B8F1000F36D183E0019972
:10854000B1F80AB00BF1FF3B1BEA532B3CD0A869F2
:108550008B690238023B984277D24A89CB6A02FB88
:108560000030002871D05FEA58240BEB000A34D0A9
:108570000BEB0403934288BFCBEB020448782346FD
:1085800052463946FBF742FD00283AD195F91030A2
:10859000002B4BDB64023368234433606B69B8EB18
:1085A0000408234427446B614DD0C3F3080100291C
:1085B000C5D0C1F50074444528BF4446494422460D
:1085C0003846FFF791FAE6E7F3B9A86801283CD9E5
:1085D000431C16D00199A861BAE7EA6992450AD00E
:1085E00095F91030002B14DB487801235246494698
:1085F000FBF70CFD28B96969C5F81CA0C1F3080197
:10860000D7E7012068748AE7A9692868FFF7CEFADE
:10861000DCE7487801234946FBF716FB0028F0D138
:108620002B7C019903F07F032B74DDE7E869CAEB2B
:1086300000008442AED907EB40204FF40072494657
:10864000FFF752FAA6E7002069E70220687466E7A0
:108650002DE9F04194B00223AD4D8DF80F30D5F8DF
:108660001023AC4C2ABB2278002A3FD09A4200D07B
:108670002370D4F880301B69984704F00BFFD4F8BE
:1086800080305B689847E36FA3495B68A0489847D0
:108690000023A5F89035A5F89235A5F89435A5F8EE
:1086A0009635A5F89835A5F89A35237014B0BDE82D
:1086B000F08123780A2BF9D801A252F823F000BFE9
:1086C000ED8600084987000873860008AD8600081B
:1086D000C5870008E587000801880008238700088F
:1086E00001870008AD8600081D880008D5F8103302
:1086F000002BDBD001236420237004F0A9FCD5E714
:10870000D4F88030834C9B6B98470128CED1E36F1F
:108710007F481B68214698470028C7D1052323704E
:10872000C4E7237F0022013BA2740A2BBED8DFE8F6
:1087300013F0C7010402E501620236027A0219024F
:10874000AB018C017A016D01D4F880309B689847A9
:1087500000216F4801F078FC802160716C4801F0C5
:1087600073FC20716A4804F08BFCD4F88030DB681D
:108770009847D5F8CC20D4F880301068C0F3414039
:1087800084F821000422227000F003009B699847BE
:108790000025A07994F8213094F8202021790190C7
:1087A00000955B4801F06AFCA079019094F82130B3
:1087B00094F8202061790095554801F05FFC14B0D1
:1087C000BDE8F081A378092B3FF670AFDFE813F026
:1087D000F500E700AF00A600770063004F003B0004
:1087E0008B003400E36F4B4C9B6849482146984707
:1087F0008DF80F009DF80F304BB90623237055E715
:10880000E36F4449DB68424898478DF80F009DF8B4
:108810000F0004F06FFE14B0BDE8F08104F03AFEE2
:10882000D4F880305B689847E36F3B495B68384811
:10883000984714B0BDE8F081D4F880305B6B98475E
:108840000823237032E794F83200324C002800F0FD
:10885000178204A904F066FE00287FF427AFD4F83D
:10886000803004A81B6B98470823A3701EE794F878
:108870003100284C002800F0F38104A904F052FED6
:1088800000287FF413AFD4F8803004A8DB6A98473F
:108890000723A3700AE794F830001E4C002800F06C
:1088A000E78104A904F03EFE00287FF4FFAED4F86F
:1088B000803004A89B6A98470623A370F6E6E08EF2
:1088C000144C04F067FE00287FF4F0AED4F880303A
:1088D00004F150025B6A04F13E0104F13400984750
:1088E0000523A370E2E60B4E94F83930E3820025AD
:1088F00009270748257531462B462A462583658377
:10890000677502F06DFD00287FF4D0AEB770CDE63C
:108910002C3C0120D8410120F8410120092004F01D
:1089200039FE00287FF4C2AE0423A370BEE6C64E13
:10893000C64F00252B462A464FF0050E2575258388
:10894000658331460125384684F815E0E58202F05A
:1089500047FD00287FF4AAAE022004F079FBD6F888
:10896000803086F820501B6A984796F8203031797D
:108970000322B2701BB107EB411787F8AC33B34D3C
:10898000284604F0D3FA94F8203061791BB105EB46
:10899000411585F8AC33AD4804F0C8FA86E61220DC
:1089A00004F016FF00287FF481AED4F88030A84888
:1089B000DB6998470223A37078E6082004F008FFDB
:1089C00000287FF473AE94F82930A048A37104F016
:1089D00057FB6179A37905EB41120126B2F8B20386
:1089E000A670984202D00BB1A2F8B233974804F0B7
:1089F0009DFA2179A37905EB4115B5F8B2239A4286
:108A0000C9D0002BC7D0A5F8B233C4E7A37B8E4AE8
:108A10000133DBB2022BA37340F23F81082153786C
:108A20009174137042E66379874A1D4495F89B332D
:108A3000DBB2012B00F02C81022B00F04C81032BC8
:108A40007FF434AE0B23237730E661797F4801F160
:108A5000150205EB4212022305EB411682F8143190
:108A60000023C2F818316F18012286F8AE33C6F819
:108A7000BC33C6F8C03386F8C52387F89B3304F0AF
:108A8000AFF90A23237711E623796F496F4A1D4412
:108A900095F89B33DBB2012B00F0FA80032BD1D089
:108AA00052696C4892680D8A008892B2521B8242C9
:108AB000C8D8042B7FF4FAAD4A788B740A70F5E5B8
:108AC0006179654F614801F1150305EB431305EB2F
:108AD0004112032683F814610D44C3F81871082667
:108AE000002382F8AE33C2F8C033C2F8BC6385F805
:108AF0009B3304F075F902232377D7E52179A26827
:108B0000A789524801F1150305EB4313022683F8A8
:108B1000146105EB4116C3F818210D44002301220E
:108B2000C6F8C03386F8AE23C6F8BC7385F89B330D
:108B300004F056F904232377B8E56379474A2B44B8
:108B4000116893F89B33DBB28B4218BF1360012B83
:108B500000F0A680032B7FF4A9AD0B22052322771A
:108B6000A374A3E52179394801F1150205EB4212FE
:108B70006F18022605EB4115002382F814610126C7
:108B8000C2F81831C5F8BC33C5F8C03385F8AE63F8
:108B900087F89B3304F024F90823237786E561796D
:108BA000A789A6684B0105EB030E01F115024FF0F2
:108BB000000801F11E008EF8AE8305EB42182B442D
:108BC00005EB401005EB42124FF0010CCEF8BC73E0
:108BD000C8F818610D440026022780F805C0C3F8C4
:108BE000C0631A4882F8147185F89B6304F0F8F8A2
:108BF000062323775AE52379134A2B4493F89B33B2
:108C0000DBB2012B5ED0042B5FD0032B3FF41AAFF5
:108C10006B69104A9B68218A12889BB25B1A934247
:108C20003FF610AF42E56379074A1D4495F89B3340
:108C3000DBB2012B4CD0042B50D0022B7FF4FFAEC3
:108C40000523137732E500BFD84101202C3C0120D9
:108C5000FA410120A8250120EC4101208C000020D0
:108C6000D4F880302648DB6A98470723A3701DE5B7
:108C7000D4F8803022489B6A98470623A37015E5F4
:108C8000D4F880301E481B6B98470823A3700DE56D
:108C9000637823700D23237708E50123137705E517
:108CA000237D618B174A23F07F03DBB2D9B11649CC
:108CB00041F288300880EBB9052313776B699B6814
:108CC0002382F3E409231377A2E753781370EDE4CA
:108CD00007231377EAE409231377E7E45378137043
:108CE0000C231377E2E40849322008802BB90723CC
:108CF0001377E3E703231377E0E709231377DDE72F
:108D000034180108D8410120A825012070B5134D61
:108D1000134C82B0002628464FF6FF734FF41672AC
:108D200034210096FEF7EAFE284607F0EFF94FF4EB
:108D30007843C50005F516722046009334214FF69E
:108D4000FF73FEF7DBFE009605F5187220464FF61E
:108D5000FF733421FEF7D2FE02B070BD94240020D0
:108D6000381801082DE9F84FDFF80892D9F80030DB
:108D7000054688461646002B00F0D5809A68794F44
:108D8000013A002A9A603868C0F283801A6810217C
:108D9000501C18601170D9F800403868A368013B76
:108DA00008F1020B002BA3604FEA2B2AC0F2B2801D
:108DB0002368E822591C21601A70A3683868013BB7
:108DC000002BA360C0F29D8023680322591C216000
:108DD0001A70A3683868013B002BA360C0F285803D
:108DE00023685A1C226083F800B0A3683868013BEE
:108DF000002BA3606EDB23685A1C226083F800A05E
:108E0000A3683868013B002E14BFFF260026002B04
:108E1000A36057DB23685A1C22601E70B8F1000F54
:108E200026D0A844DFF850A11FFA88F808E023688C
:108E30000135ADB25A1C4545226083F800E017D0D9
:108E4000A3681AF805E03868013B002BA3608EEA9E
:108E50000606ECDAA26993427146224602DBBEF1B5
:108E60000A0FE4D10135ADB206F0AAFA4545E7D1C3
:108E7000A3683868013B002BA36013DB23685A1CEE
:108E800022601E70D9F8000005F0D8F80120BDE876
:108E9000F88F99698A42BFF679AF1A46102106F019
:108EA0008FFA78E7A269934201DB0A2EE6D12246C7
:108EB000314606F085FAD9F8000005F0BFF8012028
:108EC000BDE8F88FA2699342A4DA2246314606F043
:108ED00077FAA3E7A26993425FFA8AF101DB0A29D4
:108EE00089D1224606F06CFA8AE7A26993425FFABA
:108EF0008BF102DB0A297FF473AF224606F060FA99
:108F000073E7A2699342BFF65FAF2246032106F0E2
:108F100057FA5EE7A2699342BFF64AAF2246E821BC
:108F200006F04EFA49E71049104805F0F3F90446F7
:108F3000C9F80000A0B10346072201210C4806F041
:108F4000FBFC21461A2006F07BFB2146012006F09F
:108F500077FB2146102006F073FBD9F800300DE7AF
:108F6000BDE8F88F2001002088040108A424002017
:108F7000EC0B0108A4250020A825002082B00023C6
:108F80000193019B0133332B0193FAD902B070474F
:108F90002DE9F041A54BA64D1B78A64982B01BB91F
:108FA000A54B1A78002A4AD02B889A1C92B201331A
:108FB000885C2A809BB200F00706CA56062100F0A2
:108FC000F803382B00F2FF80DFE813F05800FD00B3
:108FD000FD00FD00FD00FD00FD00FD00D800FD00CE
:108FE000FD00FD00FD00FD00FD00FD00E900FD00AD
:108FF000FD00FD00FD00FD00FD00FD007A00FD000C
:10900000FD00FD00FD00FD00FD00FD009000FD00E5
:10901000FD00FD00FD00FD00FD00FD00A800FD00BD
:10902000FD00FD00FD00FD00FD00FD00BF00FD0096
:10903000FD00FD00FD00FD00FD00FD0042002B884D
:1090400001339BB22B80C85C00F007010E46B6E7E7
:1090500001AF7A4C384604F0BDFD9DF80630A27988
:10906000D9074CBF42F0010222F001025B08062E34
:10907000A2711FFA83F84CD0A35514E001AF384613
:1090800004F0A8FD9DF806306C4C1906A27900F199
:10909000C3805B0022F0010203F0FE08A271062EDD
:1090A00037D004F80680404602F01EF8A2792B88DB
:1090B00022F012020133A2712B8002B0BDE8F081D0
:1090C0005E4C01AF384604F085FDA3799DF806207B
:1090D000D9074FEA520848BF48F08008D0074CBF74
:1090E00043F0010323F00103A371D8E701AF384631
:1090F000524C04F06FFD9DF80600A37901064CBFA9
:1091000043F0010323F00103062EA3714FEA400848
:10911000C7D13946404604F051FDC4E701AF384697
:10912000464C04F057FD9DF80600A379C2074CBFDA
:1091300043F0010323F00103A371030646BF400877
:1091400040F080084FEA5008A9E701AF38463B4C91
:1091500004F040FD9DF80630A27918064FEA43035B
:109160004CBF42F0010222F0010243F00103062E3F
:10917000A2711FFA83F8CCD0A35594E701AF38460B
:1091800004F028FD9DF806002C4CC207A3793DD5BC
:10919000400843F0010340F08008A3717FE7274CAB
:1091A00001A804F017FDA3799DF8062003F0010340
:1091B00043EA4203062E9FB218BFA35560D038463B
:1091C00001F0A6FF72E700F0C003802BC0F3C204D9
:1091D00047D0C02B34D0402B7FF46FAF01A804F0F0
:1091E000F9FC9DF806002041144CA379C20748BF42
:1091F00003F0BB032A8858BF43F0440323F0020363
:1092000043F010030132A3712A8056E723F00103D3
:109210004FEA5008A37142E74FEA430848F00108BB
:1092200042F001035FFA88F8A37138E78242012017
:10923000D8080020A8250020834201207442012084
:1092400001A804F0C7FC01209DF80630A040184397
:10925000062E00B219D00F4B98552B8801332B8066
:109260002BE701A804F0B6FC01209DF80630A040D1
:10927000062E23EA0000EED101A904F09FFCECE7E2
:1092800001A9384604F09AFC99E701A980B204F0DC
:1092900095FCE2E774420120F0B5114FDFF850E091
:1092A000104A114D3B88DEF8004016882A88591E66
:1092B00089B20B340132B142CEF8004092B204D3ED
:1092C0000A4C4FEA122E04F801E0023B9BB29E4288
:1092D00098BF06493B8098BFCA542880F0BD00BFA4
:1092E000F002002080420120D8080020A82500209C
:1092F00084420120134A0123927903FA01F11140BB
:1093000010B1B1FA81F1490941B90F480F4902681A
:109310000B880532013302600B807047F0B40C4DAE
:109320000C4E2B88084CF15C2268084F581C80B208
:109330000233305C2B8041EA00230B323B802260F9
:10934000F0BC70477442012084420120D8080020FC
:10935000F0020020A825002070B41D4B1B780BB331
:109360001C481D4B0268197A5B7A0F32026043EA8F
:1093700001211A4C1A4A238810885A1E92B282423E
:1093800002D3184D0E0AAE54023B9BB2984298BFCE
:10939000144A238098BFD154134A13880133138091
:1093A00070BC7047114B0B481B7843B10A4B0268E5
:1093B000997ADB7A0F32026043EA0121D9E7064B42
:1093C000026819795B790B32026043EA0121D0E728
:1093D000824201208442012074420120F0020020D8
:1093E00080420120A8250020D808002083420120C7
:1093F000F0B4134A1349144E144F0D8833883C6857
:1094000002EB400112F810004A78591E89B242EA74
:1094100000220B34A94212B23C6003D30C48C2F3C1
:1094200007244454023B9BB29D4298BF08493380B5
:1094300098BFCA54074A138801331380F0BC7047A1
:109440007442012080420120F00200208442012069
:10945000A8250020D8080020F0B4254B1B78002B4D
:109460002FD1244B244E1B78244F3288244CB3B97F
:10947000501C80B2BB5C385C2168224D43EA00235B
:1094800002321BB232800A31C3F307222A716B7198
:1094900021601D4A138801331380F0BC7047501CB3
:1094A00080B2BB5C385C2168164D43EA002302326F
:1094B0001BB232800E31C3F30722AA72EB72216015
:1094C000E7E70D4E0D4F32880D4CBB5C21680D4D0A
:1094D000501C80B20232385C328043EA00231BB257
:1094E000C3F307220E312A726B722160D1E700BFED
:1094F0008242012083420120F0020020A8250020A2
:109500008442012074420120D8080020F0B5DFF821
:1095100050E00F4CBEF800200E4FA35C0E4E3D688D
:10952000511C89B20232645C0C49AEF8002043EA57
:1095300004231BB23488C3F3072201F8102001EB87
:1095400040010A3501343D604B703480F0BD00BFEE
:10955000A825002084420120D80800207442012060
:10956000F002002038B5074C074D236869780246A1
:109570000C332878236001F0A9FE044A13880133D4
:10958000138038BD8442012074420120D808002095
:10959000F0B5164D164C2988DFF860E0154E4A1CD0
:1095A0008B1C97B29AB2E35DA25C134F03EB0223CC
:1095B0000EEB40021EF810E052783F8830689BB2F4
:1095C00042EA0E2212B29F4298BFE25401339BB28C
:1095D0009F4298BFC2F3072200F1140001F103017A
:1095E00098BFE25430602980F0BD00BFD808002049
:1095F000A8250020844201208042012074420120DD
:1096000070B41C4B1B78F3B11B491C481C4D0388DC
:109610001C4C0E7A4A7A216801339BB242EA062238
:10962000ED5613312A4492B22160174C2488591CFC
:1096300089B29442018002D8114C615CA15402337A
:10964000038070BC7047114B1B783BB10A490B4833
:109650000B4D03880B4C8E7ACA7ADCE7094C064B1B
:1096600021681D795A7905480A310388216042EA48
:109670000522DAE78242012074420120D808002046
:10968000A82500208442012080420120834201203D
:10969000F8B5244B1B7843B3234C244D24482A8827
:1096A000244E277A637A3168013292B243EA072363
:1096B00087562A803B4413319BB23160E279C35C08
:1096C000194E53401846E37101F00EFD1A49E27934
:1096D000A3798A5C23F01301A171EAB923F017037F
:1096E000B3712B8801332B80F8BD144B1B783BB131
:1096F0000D4C0E4D0E482A880E4EA77AE37AD2E71B
:109700000C49094C0A6826796379084D08480732E4
:109710000A6043EA0623D1E704F0AAFA2B88013352
:109720002B80F8BD8242012074420120D80800201D
:10973000A825002084420120C004010883420120A2
:1097400010B51D4B1B78F3B11C490A68031F083282
:10975000012B0A602CD91A4C235CE279534018463D
:10976000E37101F0C1FC1749E279A3798A5C23F027
:109770001301A171CAB923F01703A371124A138808
:109780000133138010BD114B1B784BB10B490A6894
:10979000031F0832012B0A60DDD80630C0B2DAE7B9
:1097A000064A136804331360D5E704F061FAE5E76D
:1097B0000430C0B2CFE700BF8242012084420120C2
:1097C00074420120C0040108D8080020834201200F
:1097D000F8B5244B1B7843B3234C244D24482A88E6
:1097E000244E277A637A3168013292B243EA072322
:1097F00087562A803B4413319BB23160E279C35CC7
:10980000194E13431846E37101F06EFC1A49E279D0
:10981000A3798A5C23F01301A171EAB923F017033D
:10982000B3712B8801332B80F8BD144B1B783BB1EF
:109830000D4C0E4D0E482A880E4EA77AE37AD2E7D9
:109840000C49094C0A6826796379084D08480732A3
:109850000A6043EA0623D1E704F00AFA2B880133B1
:109860002B80F8BD8242012074420120D8080020DC
:10987000A825002084420120C00401088342012061
:109880002DE9F0414700224CDFF88CE014F810502D
:1098900062792179DEF80060013742EA0121E35D57
:1098A000804643EA0523A079C3F30B05C1F30B02FD
:1098B000521B00F00105CB1A521B0F365D1BD3045F
:1098C000CEF800601CD420F01000A071E35D14F805
:1098D000182043EA0222D24392B2284601F034FC17
:1098E0002B0A28462371657101F0E2FB0949A3792F
:1098F0000A8843F0020301320A80A371BDE8F081B7
:1099000004F0BEF92179637943EA0121DEE700BF63
:1099100074420120D8080020844201202DE9F04142
:109920002C4B1B78002B39D02B4C2C4E2C483288DA
:109930002C4D277A637A2968013292B243EA0723D1
:10994000875632803B4413319BB22960C75CE17972
:10995000A279DFF8848007F00F0001F00F031B1AD3
:1099600002F001055B1BC81B451BDB06ADB22CD406
:1099700022F0100288F80620FA43D2B2284601F0FD
:10998000F3FB2846E57101F0C3FBA279338842F06E
:1099900002020133A2713380BDE8F081124B1B78C3
:1099A0003BB10D4C0D4E0E4832880E4DA77AE37A2E
:1099B000C1E70C49084C0A6825796379074E0848C5
:1099C00007320A6043EA0523C0E704F059F998F822
:1099D0000710D1E78242012074420120D8080020FC
:1099E000A8250020844201208342012070B5254B28
:1099F0001B7806466BB324490A68031F0832012B03
:109A00000A603CD9214DE979AC5DAA7904F00F00D8
:109A100001F00F031B1A02F001000C1B1B1A241A81
:109A2000DB06A4B227D422F01002AA71AA5DD243A9
:109A3000D2B2204601F098FB2046EC7101F068FBA1
:109A40001349AB790A8843F0020301320A80AB71F3
:109A500070BD104B1B784BB10B490A68031F0832CD
:109A6000012B0A60CED80636F6B2CBE7064A136859
:109A700004331360C6E704F003F9E979D6E7043646
:109A8000F6B2BFE7824201208442012074420120E5
:109A9000D8080020834201202DE9F8432B4B1B7886
:109AA000002B37D02A4C2B4D2B482A882B4E277A57
:109AB000637A3168013292B243EA072387562A80DB
:109AC0003B4413319BB23160C65CE179DFF8809092
:109AD00006F00F0201F00F039B1A8F1BDB061FFA23
:109AE00087F82ED499F8063023F0100389F8063051
:109AF000F243D2B2404601F037FB4046E77101F035
:109B000007FBA2792B8842F002020133A2712B805D
:109B1000BDE8F883124B1B783BB10D4C0D4D0E4840
:109B20002A880E4EA77AE37AC3E70C49084C0A68E4
:109B300026796379074D084807320A6043EA06230D
:109B4000C2E704F09DF899F80710D1E7824201209E
:109B500074420120D8080020A8250020844201205A
:109B600083420120F8B5234B1B7806464BB32249AC
:109B70000A68031F0832012B0A6038D91F4CE179AB
:109B8000A55D01F00F0305F00F029B1A4D1BDB06CC
:109B9000AFB228D4A37923F01003A371A25DD243FE
:109BA000D2B2384601F0E0FA3846E57101F0B0FA79
:109BB0001349A3790A8843F0020301320A80A37192
:109BC000F8BD104B1B784BB10B490A68031F0832D4
:109BD000012B0A60D2D80636F6B2CFE7064A1368E0
:109BE00004331360CAE704F04BF8E179D6E7043692
:109BF000F6B2C3E782420120844201207442012070
:109C0000D808002083420120044B05491A7802201D
:109C100008700AB100221A70704700BFAC00002023
:109C200060260120014B01221A7070476026012036
:109C3000002070470023C0F810331846704700BF5B
:109C40000123C0F810330020704700BF2DE9F04F0A
:109C50004D4ADFF848E101789EF800404B4DDFF8AF
:109C600040C102F11006012311E014EA030709D1F3
:109C70002968B2F800802CF8118001312029296070
:109C800018D001780232B2424FEA430314D011EAED
:109C90000307EAD11C42F5D0D5F80090118809F1EC
:109CA000010841F40071B8F1200F2CF81910C5F823
:109CB0000080E6D12F60E4E7354F8EF800103D6854
:109CC000DFF8D0C0DFF8D0A0DFF8C090DFF8D0B068
:109CD0004FF0000E811CF046013010F8016F06B302
:109CE0006DB19CF80030B34243D02A4A002303E010
:109CF00012F8014FB4423DD00133AB42F8D13AF8EB
:109D000016204AB1D9F80040631C202B08BF4346F7
:109D10002BF81420C9F800300EF1010EBEF1060F29
:109D2000DBD1F5B1DFF864901A4BD9F800001A4E78
:109D3000DFF86C801D444FF0000C13F8012B36F84F
:109D4000122042F400743AB128F810400130202863
:109D50004FF0010C08BF0020AB42EED1BCF1000F68
:109D60000ED1C7F800E072460A48BDE8F04F04F093
:109D700077BC0023AB420CF80380CDD10678BEE758
:109D8000C9F80000EDE700BF40180108B425012024
:109D900058260120AC25012050180108AA250120D1
:109DA000B8250120F8B53E4D95F845300446042B02
:109DB00023D8DFE803F03C243C13030000230122F6
:109DC00021270B26CA820F754E750B834B831A46CB
:109DD00001F006FB88B985F84500F8BD00230A228A
:109DE00021264A750E75CB820B834B831A4601F0F0
:109DF000F7FA00284FD003284DD00120F8BD294B99
:109E00004FF4085000221B89C882812706260A8346
:109E10004B830F754E7504F58872204601F0E0FA09
:109E20000028EAD1032385F845300120F8BD4FF41E
:109E300004500022812706260923C8820A830F7551
:109E40004E754B8304F58872204601F0C9FA00284C
:109E5000D3D194F8130194F81211124B94F81861AD
:109E600094F8172194F810711F7001EB002194F8F9
:109E7000110194F81471598002EB062294F816111E
:109E800094F81561587001201F715E7199711A81E3
:109E900085F84500F8BD042385F845300120F8BD5C
:109EA000F82501204C260120F8B5484C94F84230A2
:109EB0000546052B20D8DFE803F0211F1F302703BC
:109EC0004369B4F84A709B68B4F84C603F489AB252
:109ED000B3B2D31ABB421BD290F84020AB1893F810
:109EE0009B63012E4FD13A4B1A78012A04D1026D9F
:109EF00000215268197090470020F8BD236D1B683F
:109F00009847042384F842306B699B68DB07F3D4DD
:109F1000032384F842300020F8BD94F8401094F8F0
:109F200046704B01C61801F1150200EB42120120E8
:109F300086F8AE0305EB4110C2F81841C6F8BC73B1
:109F400090F8C46306B1022682F8146190F8C42325
:109F50002B446F1882F00102002680F8C42387F892
:109F60009B632846C3F8C06302F03AFF052384F8D8
:109F70004230174A6B69012111709B689BB2A4F8AB
:109F80004C300020F8BD93F89B33042BB4D190F8EB
:109F900048300B8313F0800F02F11E0305EB4313CF
:109FA0004FF000004FF002074FF00106C8824883CF
:109FB0000F754E7514BF18715871002328461A4644
:109FC00001F00EFA0028A3D096E700BFF825012083
:109FD000B225012070B51A4C94F840100546E9B935
:109FE00094F84110164E19B9164B00221A7070BD24
:109FF000284602F0D5FE96F84130072B07D805EB2E
:10A000004305B5F88C35C3F30E03A5F88C35002352
:10A0100084F841300B4B00221A7070BD02F0C0FE74
:10A0200094F84030072B07D805EB4303B3F88C2591
:10A03000C2F30E02A3F88C25002384F84030CFE74A
:10A04000F8250120B225012030B400F28A52002305
:10A0500032F9024F002CDDB205DA0133082BF7D1BB
:10A06000FF2030BC704700EB43006FEA41416FEACC
:10A070005141A0F88C15284630BC7047F8B500EB6C
:10A08000410500EB4114B5F88C559DF8187084F823
:10A09000AC2305F07F06C5F3C01584F8AD6384F8E2
:10A0A000AE53BDF81C6084F8AF33002584F8B1735B
:10A0B000A4F8B26384F8C45384F8C55313B90123D8
:10A0C00084F8B03302F032FF0020F8BD2DE9F043F0
:10A0D00091F84430364D0622012B83B00C4685F8AA
:10A0E000422007D0D1F880301B6C9847012003B084
:10A0F000BDE8F08391F84530012B074654D0022B80
:10A1000004BF2C4B2B6594F8561094F85230B4F8D9
:10A11000540085F84830002285F8422085F8452013
:10A120000929234AA5F8460098BF0A21A2F84A1037
:10A1300094F84260022E28BF02267EB3013EF6B29A
:10A140001A0604EBC606A0464FF003091946384626
:10A150001CD485F84330FFF777FF014685F84100AE
:10A16000B5F8460094F8213094F820200190CDF8FD
:10A1700000903846FFF782FFB0450FD098F85A306C
:10A180001A0608F1080819463846E2D585F8443021
:10A19000FFF75AFF014685F84000E1E7064B002033
:10A1A000187003B0BDE8F083044B2B65ABE700BF2C
:10A1B000F8250120A4000020B225012090000020F5
:10A1C00080B485B000AF78607B68D3F890301B68AE
:10A1D000BB60FB7A43F08003FB72FB7A43F04003E1
:10A1E000FB727B68D3F89030BA681A600023FB607A
:10A1F000BB7B43F02003BB737B68DB68FA685A6162
:10A20000012318461437BD465DF8047B704700BF34
:10A2100080B588B000AF78600023FB7200237B61BB
:10A220003B7D43F010033B757B68DB687A68D2683E
:10A2300091697A69D2430A409A617B68DB681B6A3C
:10A24000BB613B7EC3F30303DBB2FB72FB7ADBB281
:10A250007A6822339B0013449B681B68FB60BB7EBB
:10A26000C3F34303DBB2022B40F08D803B8BC3F37F
:10A270000A139BB2002B40F38580FB7ADBB27A682D
:10A2800015335B01134403F58C731B68002B79D0E5
:10A29000FB7ADBB27A6815335B01134403F58C73E8
:10A2A00019683B8BC3F30A139BB21A46786802F015
:10A2B000BBFE3B7EC3F30303DBB218463B7EC3F316
:10A2C0000303DBB27A6815335B01134403F58C7327
:10A2D0001B683A8BC2F30A1292B21A44796800F1F1
:10A2E00015035B010B4403F58C731A603B7EC3F3CB
:10A2F0000303DBB218463B7EC3F30303DBB27A6889
:10A300005B01134403F570731B683A8BC2F30A12A6
:10A3100092B21A44796843010B4403F570731A60D2
:10A32000FB7ADBB27A685B01134403F570731B6838
:10A33000FB61FB7ADBB21A467B68D432F96943F8D9
:10A340002210FB7ADBB27A6822339B0013449B68AD
:10A350001B693B617B8AC3F3C9039BB2002B11DDF0
:10A36000FB7B43F08003FB73FB7B6FF38613FB7374
:10A37000FB7ADBB27A6822339B0013449B68FA684D
:10A380001A6000E000BF3B7D43F010033B757B6823
:10A39000DB687A68D26891697A690A439A61012315
:10A3A00018462037BD4680BD80B59CB000AF7860B0
:10A3B00039607A683B6822339B0013449B68FB66D4
:10A3C000FB6E9B68BB66FB6EDB687B66BA6E7B6E62
:10A3D0001340BB667A683B6822339B0013449B683A
:10A3E0001B683B6600237B6697F8683003F0040324
:10A3F000DBB2002B1DD00023FB603B7B43F004034A
:10A400003B73FA68FB6E9A607A683B6822339B0064
:10A4100013449B68DB683B613B7C43F002033B7465
:10A420007A683B6822339B0013449B683A69DA6080
:10A4300093E097F8683003F02003DBB2002B09D0DB
:10A4400000237B613B7D43F020033B757A69FB6E03
:10A450009A6082E097F8683003F00803DBB2002BC3
:10A460003BD07A683B6822339B0013449B68DB68CF
:10A47000BB613B7E43F002033B767A683B68223344
:10A480009B0013449B68BA69DA607A683B6813449E
:10A4900003F5637305221A700023FB613B7F43F0D1
:10A4A00010033B77FA69FB6E9A6000233B6297F8D2
:10A4B000203043F0080387F820303A6AFB6E9A6038
:10A4C00097F868306FF3041387F868303B68DBB2A5
:10A4D0001946786802F064FC3FE097F8693003F0B1
:10A4E0000403DBB2002B38D07A683B6822339B0030
:10A4F00013449B68DB687B6297F8243043F00203C7
:10A5000087F824307A683B6822339B0013449B68A9
:10A510007A6ADA603B68DBB21946786802F040FC80
:10A520000023BB6297F8283043F0100387F82830E7
:10A53000BA6AFB6E9A607A683B68134403F56373EA
:10A5400008221A700023FB6297F82D3043F00403B1
:10A5500087F82D30FA6AFB6E9A6097F8693003F03D
:10A560000203DBB2002B27D07A683B6822339B00C2
:10A5700013449B68DB683B6397F8303043F0020379
:10A5800087F830307A683B6822339B0013449B681D
:10A590003A6BDA603B68DBB21946786802F000FC7F
:10A5A00000237B6397F8353043F0020387F835309A
:10A5B0007A6BFB6E9A60CBE197F8683003F0010389
:10A5C000DBB2002B00F09B807B68DB78012B17D17E
:10A5D0007A683B6822339B0013449B681B69FB65C8
:10A5E0007A683B685B01134403F56F731B68FA6D6F
:10A5F000C2F31202991A7B683A68D43243F82210E7
:10A600007A683B68134403F5637301221A707A6811
:10A610003B68C4339B00134400225A600023BB6391
:10A6200097F8383043F0010387F83830BA6BFB6E87
:10A630009A6097F8623003F00C03DBB2002B06D06F
:10A6400097F8623003F00C03DBB2082B39D17A683B
:10A650003B6822339B0013449B68DB68FB6397F8DD
:10A660003C3043F0020387F83C307A683B68223381
:10A670009B0013449B68FA6BDA603B68DBB21946B7
:10A68000786802F08DFB00233B6497F8403043F07C
:10A69000100387F840303A6CFB6E9A607A683B682A
:10A6A0001E335B01134404331B7883F00103D9B2DA
:10A6B0007A683B681E335B01134404330A461A7000
:10A6C00045E197F8623003F00C03DBB20C2B40F04D
:10A6D0003E8197F8633043F0200387F863307A684F
:10A6E0003B6822339B0013449B683A6E1A607A6879
:10A6F0003B68134403F29B3301221A7028E197F858
:10A70000683003F00203DBB2002B7DD07A683B682F
:10A7100022339B0013449B68DB687B6497F84430CA
:10A720006FF3410387F844307A683B6822339B001B
:10A7300013449B687A6CDA607A683B68134403F5CB
:10A7400063731B78DBB2012B07D17A683B68134433
:10A7500003F29B3301221A704AE07A683B68134483
:10A7600003F563731B78DBB2052B07D17A683B686E
:10A77000134403F29B3304221A7039E07A683B6871
:10A78000134403F563731B78DBB2062B08D07A6899
:10A790003B68134403F563731B78DBB2082B0ED1BF
:10A7A0007A683B68C4339B00134400225A607A687D
:10A7B0003B68134403F29B3303221A7018E097F8A6
:10A7C000623003F00C03DBB20C2B11D17A683B68CA
:10A7D0001E335B01134404331B7883F00103D9B2A9
:10A7E0007A683B681E335B01134404330A461A70CF
:10A7F0000023BB6497F8483043F0020387F84830E1
:10A80000BA6CFB6E9A60A3E097F8683023F07F0380
:10A81000DBB2002B3BD07A683B6822339B001344A9
:10A820009B68DB68FB6497F84C3043F0020387F8C1
:10A830004C307A683B6822339B0013449B68FA6C67
:10A84000DA607A683B68C4339B0013445B685A1C27
:10A8500079683B68C4339B000B445A607A683B6854
:10A86000134403F5637306221A703B68DBB2194682
:10A87000786802F095FA00233B6597F8503043F072
:10A88000800387F850303A6DFB6E9A6060E097F86D
:10A89000683003F01003DBB2002B59D097F8623018
:10A8A00003F00C03DBB20C2B1CD17A683B6822331B
:10A8B0009B0013449B68DB687B6597F8543043F03A
:10A8C000020387F854307A683B6822339B001344B4
:10A8D0009B687A6DDA603B68DBB21946786802F0F3
:10A8E0005FFA21E097F8623003F00C03DBB2002B33
:10A8F00006D097F8623003F00C03DBB2082B13D1BB
:10A9000097F8633043F0800387F8633097F863303B
:10A910006FF3861387F863307A683B6822339B00B5
:10A9200013449B683A6E1A607A683B68134403F5D7
:10A93000637303221A700023BB6597F8583043F005
:10A94000100387F85830BA6DFB6E9A6000E000BFC4
:10A95000012318467037BD4680BD00BF80B59AB050
:10A9600000AF786039607A683B6822339B001344FB
:10A970009B687B667B6E9B683B667B6EDB68FB65DA
:10A980003A6EFB6D13403B667A683B6822339B004E
:10A9900013449B681B68BB6597F8603003F00403A1
:10A9A000DBB2002B1DD00023BB603B7A43F00403D5
:10A9B0003B72BA687B6E9A607A683B6822339B0070
:10A9C00013449B68DB68FB603B7B43F002033B73F3
:10A9D0007A683B6822339B0013449B68FA68DA600C
:10A9E00060E297F8603003F02003DBB2002B09D05F
:10A9F00000233B613B7C43F020033B743A697B6E50
:10AA00009A604FE297F8613003F00203DBB2002B4B
:10AA100023D07A683B6822339B0013449B68DB6831
:10AA20007B613B7D43F002033B757A683B682233D0
:10AA30009B0013449B687A69DA603B68DBB2194675
:10AA4000786802F0ADF90023BB617B7E43F002031E
:10AA50007B76BA697B6E9A6024E297F8603003F0E7
:10AA60000103DBB2002B33D07A683B68C4339B0010
:10AA7000134400225A607A683B6822339B001344D7
:10AA80009B68DB68FB613B7F43F002033B777A689E
:10AA90003B6822339B0013449B68FA69DA603B6889
:10AAA000DBB21946786802F07BF900233B6297F825
:10AAB000203043F0010387F820303A6A7B6E9A60B9
:10AAC0007A683B68134403F5637301221A70E9E165
:10AAD00097F8603003F00803DBB2002B2ED0002380
:10AAE0007B6297F8243043F0080387F824307A6AB1
:10AAF0007B6E9A607A683B6822339B0013449B68A4
:10AB0000DB68BB6297F8283043F0020387F82830EF
:10AB10007A683B6822339B0013449B68BA6ADA6008
:10AB20003B68DBB21946786802F03AF97A683B680C
:10AB3000134403F5637305221A70B3E197F860308C
:10AB400003F01003DBB2002B35D07A683B68C433C6
:10AB50009B00134400225A607A683B6822339B00B2
:10AB600013449B68DB68FB6297F82C3043F00203C8
:10AB700087F82C307A683B6822339B0013449B682B
:10AB8000FA6ADA603B68DBB21946786802F008F9C5
:10AB900000233B6397F8303043F0100387F83030E0
:10ABA0003A6B7B6E9A607A683B68134403F5637373
:10ABB00003221A7076E197F8603023F07F03DBB24E
:10ABC000002B3BD07A683B6822339B0013449B6880
:10ABD000DB687B6397F8343043F0020387F8343046
:10ABE0007A683B6822339B0013449B687A6BDA6077
:10ABF0003B68DBB21946786802F0D2F87A683B68A5
:10AC0000C4339B0013445B685A1C79683B68C433A7
:10AC10009B000B445A607A683B68134403F56373E6
:10AC200006221A700023BB6397F8383043F0800384
:10AC300087F83830BA6B7B6E9A6033E197F86030F2
:10AC400003F04003DBB2002B35D07A683B68C43395
:10AC50009B00134400225A607A683B6822339B00B1
:10AC600013449B68DB68FB6397F83C3043F00203B6
:10AC700087F83C307A683B6822339B0013449B681A
:10AC8000FA6BDA603B68DBB21946786802F088F844
:10AC900000233B6497F8403043F0400387F840308E
:10ACA0003A6C7B6E9A607A683B68134403F5637371
:10ACB00004221A70F6E097F8613003F00403DBB267
:10ACC000002B39D07A683B6822339B0013449B6881
:10ACD000DB687B6497F8443043F0020387F8443024
:10ACE0007A683B6822339B0013449B687A6CDA6075
:10ACF0003B68DBB21946786802F052F80023BB6467
:10AD000097F8483043F0100387F84830BA6C7B6EF0
:10AD10009A607A683B68134403F5637308221A70DB
:10AD20000023FB6497F84D3043F0040387F84D305F
:10AD3000FA6C7B6E9A60B5E097F8603003F002031E
:10AD4000DBB2002B00F0AE807A683B6822339B00B8
:10AD500013449B68DB683B6597F850306FF3410301
:10AD600087F850307A683B6822339B0013449B6815
:10AD70003A6DDA607A683B68134403F563731B78B5
:10AD8000DBB2012B20D17A683B68134403F29B337A
:10AD900001221A7097F85A3003F00C03DBB2082B2B
:10ADA00074D17A683B681E335B01134405331B780A
:10ADB00083F00103D9B27A683B681E335B01134408
:10ADC00005330A461A7062E07A683B68134403F55B
:10ADD00063731B78DBB2032B07D17A683B6813449B
:10ADE00003F29B3302221A7051E07A683B681344E5
:10ADF00003F563731B78DBB2042B16D17A683B68CA
:10AE00005B01134403F56C731B78012B05D13B6880
:10AE1000DBB21946786801F0AFFF7A683B681344EB
:10AE200003F29B3302221A7031E07A683B681344C4
:10AE300003F563731B78DBB2052B07D17A683B6897
:10AE4000134403F29B3304221A7020E07A683B68B3
:10AE5000134403F563731B78DBB2062B17D17A68B2
:10AE60003B68C4339B0013445B68032B0FD17A68A3
:10AE70003B68134403F29B3303221A707A683B68E1
:10AE8000C4339B00134400225A6000E000BF00233B
:10AE90007B6597F8543043F0020387F854307A6D9D
:10AEA0007B6E9A60012318466837BD4680BD00BF9F
:10AEB00080B588B000AF78600023FB610023BB61E0
:10AEC0000023FB6000237B6100233B617B68D3F898
:10AED000CC301B687B617B68D3F8CC301B683B614E
:10AEE0003B7C6FF382033B743B7C6FF341033B7409
:10AEF0003B7C6FF3C3033B743B7C6FF345133B74A4
:10AF00003B7D03F00203DBB2002B0CD03B7C43F013
:10AF100002033B743F4B1B685B6878689847BB69CA
:10AF200043F00103BB613B7D03F00803DBB2002B60
:10AF300052D03B7C43F008033B743B7D03F0040399
:10AF4000DBB2002B48D0334B1B685B6878689847AE
:10AF5000BB7D03F00603DBB2042B05D0BB7D03F001
:10AF60000603DBB2022B31D17B685B691B68FB6097
:10AF7000BB7D03F00603DBB2042B15D17B685B6954
:10AF800041F270725A603B7B03F00303DBB2022B89
:10AF90001FD07B681B7A022B03D10221786802F054
:10AFA0003DF80123FB6116E07B685B694BF680325C
:10AFB0005A603B7B03F00303DBB2012B0BD0012172
:10AFC000786802F02BF80123FB6104E00123FB61A8
:10AFD00002E000BF00E000BF3B7D03F02003DBB2D6
:10AFE000002B07D03B7C43F020033B74BB6943F04C
:10AFF0000103BB61FB69002B02D0786802F040F8C6
:10B000007B68D3F8CC303A691A60BB6918462037A0
:10B01000BD4680BD3C180108704700BF704700BFA7
:10B02000014B00221A70704760260120014B00225C
:10B030001A7070476026012001207047014B0422DE
:10B040001A70704760260120704700BF704700BF2C
:10B05000704700BF704700BF704700BF022802D989
:10B06000014B00221A70704760260120014B032219
:10B070001A70704760260120014B03221A70704736
:10B0800060260120014B03221A70704760260120C0
:10B09000014B03221A70704760260120034B02788F
:10B0A000DA704178827819705A7070475C260120F6
:10B0B0000C4A9379C1034CBF43F0010303F0FE0334
:10B0C00081B2937151B103F0BF03937101044CBF7E
:10B0D00063F07F0303F07F039371704743F04003F5
:10B0E0009371F3E774420120084A937910F0FF0F3F
:10B0F00014BF03F0BF0343F04003010693714CBF3C
:10B1000063F07F0303F07F03937170477442012063
:10B110000C4A9379C1054CBF43F0010303F0FE03D1
:10B1200010F0FF0F937114BF03F0BF0343F040030F
:10B13000010693714CBF63F07F0303F07F039371AB
:10B14000704700BF744201204A40D30B04D14840ED
:10B15000030401D502F08CBD024A937923F0040365
:10B1600093717047744201204A40D30904D148408A
:10B17000030601D502F07CBD024A937923F0040353
:10B180009371704774420120FE2938B505D01F29FC
:10B1900070D07F292CD0FF2038BDC043C3B2DD075B
:10B1A0004ABF384AFF2010789C0702D5354A5278AA
:10B1B0001040590702D5334A927810401A0702D539
:10B1C000304AD2781040DD0602D52E4A127910405E
:10B1D0009C0602D52B4A52791040590602D5294ABD
:10B1E000927910401A06D7D5264BDB79184038BD26
:10B1F000030642D444004FF4003002F0ADF80028BA
:10B20000F9D1214D21482B889BB243F480732B80C8
:10B2100002F02AF90028BED044F00100C0B2288212
:10B220001B4802F021F90028B5D02B8B2B889BB24C
:10B2300043F480632B802B8823F480631B041B0C56
:10B240002B802B889BB243F400732B804FF400308B
:10B2500002F082F80028F9D10E4802F005F9002822
:10B2600099D0094A108A13889BB243F480631380F3
:10B27000C0B238BD084B187838BDFF288BD1074BBA
:10B28000187838BDB40000200054004001000010C0
:10B29000020000104000001072420120BC0000209B
:10B2A000084B094A1B784021D8074CBF11835183B2
:10B2B00013F0020F044B4FF0800214BF1A835A831D
:10B2C000704700BFBC00002000000240FE290CD0E7
:10B2D0007F2900D0704703060CD5FF28FAD12A4BEE
:10B2E00002F003021A70FFF7DBBF284B02F00702DF
:10B2F0001A70704770B5144645004FF4003002F0E4
:10B300002BF80028F9D1224E224833889BB243F40F
:10B310008073338002F0A8F8002834D033881E48A8
:10B320009BB205F0FE0543F480633380358202F062
:10B330009BF840B31948338B02F096F818B3A3B2C8
:10B340003382652405E0013C4FF0320017D0F9F755
:10B3500001F9124802F000F80028F4D0104801F07A
:10B36000FBFF0028EFD00A4A13889BB243F4007316
:10B3700013800C4801F0F0FF0028FAD170BDBDE841
:10B38000704000F0E3BC70BDBC000020E808002065
:10B390000054004001000010020000108000001066
:10B3A00004000010100000109368013B002B10B443
:10B3B000936008DBCCB21368581C106019702046EB
:10B3C0005DF8044B70479469A34202DBCCB20A2CAF
:10B3D000F1D15DF8044B03F0F3BF00BF704700BF2D
:10B3E000C87801280ED002280AD10B7F0D2B18D067
:10B3F0000B2B13D00C2B03D10123CB7003207047F0
:10B400000120704730B40D788A60072402224D7005
:10B410000C708B810877CA7030BC70470123CB70E9
:10B42000704701230020CB700877704770B5364D08
:10B43000364A15F81040127805EB40035B7843EA72
:10B4400004232AB36A7A2C7A314842EA0424016838
:10B45000C4F30B06C3F30B0232440F31D204016074
:10B460001C4445D4AB7903F0EF03220A6C722A72B4
:10B4700003F0FD01E003244A55BF23F0030341F02C
:10B48000010193719171234A13880133138070BDB8
:10B49000214A1F481278AAB1EA7AAC7A016842EAD6
:10B4A0000424C4F30B06C3F30B0232440F311C44D3
:10B4B000D304016020D4AB7903F0EF03220AEC72CD
:10B4C000AA72D5E76A792C79016842EA0424C4F3A8
:10B4D0000B06C3F30B0232440B31D60401601C444B
:10B4E0000ED4AB7903F0EF03220A6C712A71BFE727
:10B4F00002F0C6FBAB79B8E702F0C2FBAB79DDE73F
:10B5000002F0BEFBAB79EFE77442012082420120DA
:10B5100084420120D8080020834201202DE9F04117
:10B52000214CDFF88CC06379217914F81050A2798E
:10B53000DCF800704600013643EA0121A35D804635
:10B5400043EA0523C1F30B0002F00105C3F30B0E20
:10B5500028440B4470440F371D44C304CCF80070DA
:10B560001AD422F01002A271A35D14F81820284604
:10B5700043EA0222FFF7E8FD2B0A28462371657192
:10B58000FFF796FD0949A3790A8823F002030132E7
:10B590000A80A371BDE8F08102F072FB2179637922
:10B5A00043EA0121E0E700BF74420120D8080020EF
:10B5B000844201202DE9F8432B4B1B78002B36D019
:10B5C0002A4C2B4D2B482A882B4E277A637A3168D8
:10B5D000013292B243EA072387562A803B44133153
:10B5E0009BB23160C65CE179DFF8809006F00F0312
:10B5F00001F00F0213448F19DB061FFA87F82DD4D0
:10B6000099F8063023F0100389F806303246404698
:10B61000FFF7AAFD4046E771FFF77AFDA2792B8874
:10B6200022F002020133A2712B80BDE8F883134B94
:10B630001B783BB10D4C0E4D0E482A880E4EA77A52
:10B64000E37AC4E70C49094C0A6826796379084D06
:10B65000084807320A6043EA0623C3E702F010FBFA
:10B6600099F80710D2E700BF8242012074420120FE
:10B67000D8080020A8250020844201208342012010
:10B68000F8B5224B1B7806463BB321490A68031FD5
:10B690000832012B0A6036D91E4CE179A55D01F014
:10B6A0000F0205F00F0313440D44DB06AFB226D49E
:10B6B000A37923F01003A371A25D3846FFF754FD70
:10B6C0003846E571FFF724FD1349A3790A8823F072
:10B6D000020301320A80A371F8BD104B1B784BB1F5
:10B6E0000B490A68031F0832012B0A60D4D80636BA
:10B6F000F6B2D1E7064A136804331360CCE702F0D0
:10B70000BFFAE179D8E70436F6B2C5E782420120F4
:10B710008442012074420120D80800208342012085
:10B720002DE9F0412B4B1B78002B37D02A4C2B4EA8
:10B730002B4D32882B48277A637A0168013292B206
:10B7400043EA0723AF5632803B4413319BB201607A
:10B75000E179A079EF5CDFF8808000F0010301F06F
:10B760000F029D1807F00F022A44CD191D44D3067D
:10B770002BD420F0100088F806003A462846FFF740
:10B78000F3FC2846E571FFF7C3FCA279338822F069
:10B7900002020133A2713380BDE8F081124B1B78A5
:10B7A0003BB10D4C0D4E0E4D32880E48A77AE37A10
:10B7B000C3E70C49084C0A6820796379074E084DA5
:10B7C00007320A6043EA0023C2E702F059FA98F808
:10B7D0000710D2E78242012074420120D8080020DD
:10B7E000A82500208442012083420120F8B5244B83
:10B7F0001B78064653B323490A68031F0832012BFE
:10B800000A6039D9204CE179A279A55D02F00103E3
:10B8100001F00F001F1805F00F0038440D441D44BF
:10B82000C30625D422F01002A271A25D2846FFF7BC
:10B830009BFC2846E571FFF76BFC1449A3790A8845
:10B8400023F0020301320A80A371F8BD104B1B786C
:10B850004BB10C490A68031F0832012B0A60D1D88A
:10B860000636F6B2CEE7074A136804331360C9E719
:10B8700002F006FAE179D8E70436F6B2C2E700BF73
:10B88000824201208442012074420120D808002015
:10B890008342012010B4A44CFF2323706370C305BE
:10B8A00011D5B0F5B97F44D024D8B0F58A7F3DD00A
:10B8B00040F26B13984203D100223423227063704C
:10B8C0005DF8044B70477F28FAD8984B1B78EBB98A
:10B8D000974B03EB400213F810305278D9071DD56F
:10B8E00000232370FF2A18BF0123E9D0E2545DF83A
:10B8F000044B7047B0F5BA7F20D040F275139842E0
:10B90000DED10022432322706370D9E7894B03EB19
:10B91000400213F810305278D907E1D403F0020343
:10B9200003F0FF017BB171232370DBE771232370E8
:10B93000C6E70022442322706370C1E7002242233D
:10B9400022706370BCE7FF2A40F007816938142831
:10B95000B6D801A353F820F017BA0008C1B8000800
:10B960003BBA000805BA0008C1B80008C1B8000811
:10B97000C1B8000829BA0008C1B80008F3B9000826
:10B98000F3B90008E1B90008CFB90008C1B8000850
:10B99000C1B80008C1B80008C1B80008BDB90008A6
:10B9A000C1B80008C1B80008ADB90008624B1B78E7
:10B9B000032B85D8DFE803F0AEA9A49F5E4B1B786C
:10B9C000032B3FF67DAFDFE803F0918C87825A4B63
:10B9D0001B78032B3FF674AFDFE803F04153595651
:10B9E000554B1B78032B3FF66BAFDFE803F0353880
:10B9F000476D514B1B78032B3FF662AFDFE803F036
:10BA0000292C61354C4B1B78032B3FF659AFDFE8EF
:10BA100003F0504B4641484B1B78032B3FF650AF89
:10BA2000DFE803F096918C7D434B1B78032B3FF6A8
:10BA300047AFDFE803F00B0B17433F4B1B78032B9B
:10BA40003FF63EAFDFE803F00E05171440232370E6
:10BA500036E74423237033E74223237030E7432340
:10BA600023702DE7342323702AE78223237027E7EE
:10BA70008123237024E73023237021E731232370AF
:10BA80001EE7412323701BE78323237018E733232A
:10BA9000237015E7812283232270637010E7302220
:10BAA0003323227063700BE74422412322706370BA
:10BAB00006E7342243232270637001E78423237056
:10BAC000FEE632232370FBE680232370F8E6802213
:10BAD000822322706370F3E6432242232270637054
:10BAE000EEE63122322322706370E9E642224423DB
:10BAF00022706370E4E68022832322706370DFE6A5
:10BB00003122332322706370DAE64322412322700C
:10BB10006370D5E64222432322706370D0E681220F
:10BB2000822322706370CBE664260120D037012087
:10BB3000501B0108501A0108000000203022322357
:10BB400022706370BCE64422422322706370B7E621
:10BB50003422442322706370B2E60B46E254C6E6F8
:10BB60004FF080434FF6FE7207481A820749036878
:10BB70000A6801330132C82B0A6003D1044A01214B
:10BB8000002311600360704768260120FC08002034
:10BB9000D001002000F4007292B210B5C2B9592849
:10BBA0002AD00D283DD0052841D006284ED00428A3
:10BBB0002DD02C4CFFF76EFE2078FF2812D001F01C
:10BBC00037FF6078FF280DD0BDE8104001F030BF8E
:10BBD000C0F30800592813D0224CFFF75BFE2078F1
:10BBE000FF2800D110BD01F005FF6078FF28F9D0D3
:10BBF000BDE8104001F0FEBE1B4B01221A7010BDC3
:10BC0000002001F0F7FE184B00221A7010BD174AF1
:10BC1000D2F8CC300133022B08BF0023C2F8CC305D
:10BC200010BD1349134B012008601A7010BD0F4955
:10BC300091F8C9300133DBB2042B14BF81F8C9304D
:10BC400081F8C920BDE8104001F010BF074991F804
:10BC5000C8300133DBB2022B14BF81F8C83081F841
:10BC6000C820EFE764260120D0370120FC03002024
:10BC7000E408002001000020F0B585B001F060FB71
:10BC80002D4D2E4BAC881E686846F8F727FD029AAA
:10BC90002B482C4BA0FB021024F03F042404800C02
:10BCA000240C87B23C43AC80298821F001010904AF
:10BCB000090C9E42298024D87300B2FBF3F39BB297
:10BCC000032B07F1010798BF04232F841A4A93839B
:10BCD00013889BB243F001031380138823F481631C
:10BCE00023F002031B041B0C43F480634FF48041D8
:10BCF0001380118113889BB243F00103138005B0B8
:10BD0000F0BD06EB4603B2FBF3F39BB2C3F30B02A9
:10BD10000AB943F001034FF496710B4C064D01FB39
:10BD200000F284FB0201D217C2EBA112013292B2DF
:10BD300043F400432A84C9E7005400404423002010
:10BD400083DE1B43A0860100D34D621008B50B4A69
:10BD500013889BB243F40073138013886FEA434344
:10BD60006FEA53439BB213801388C3F30E0313800F
:10BD700001F0E6FABDE80840FFF77EBF005400403E
:10BD800002288CBF00200120704700BF022838B570
:10BD90001ADD0338072817DC124C4FF40B7505FB2E
:10BDA0000040D0F82842E3070ED5012A0B4614D0F4
:10BDB000022A0FD062B9FCF717FA48B102F018F85E
:10BDC0004FF4FA63036003E002F012F80923036002
:10BDD000002038BDC1681944EDE741691944FCF7FA
:10BDE00003FAEAE77026012000286AD0F0B501289E
:10BDF00083B00C46154624D002284BD003380728C0
:10BE000062DC3A4B4FF40B7606FB0036D6F828324C
:10BE1000DB0759D50027B5F5007F5ADD01AB4FF49C
:10BE2000007221463046FCF79BFA50BB019BB3F5EC
:10BE3000007FA5EB03051C441F44ECD2384603B039
:10BE4000F0BD002A1ADD2A4E8F1806E0F8F70AFC2A
:10BE500014F8013B3360A74210D020780A28F5D1AE
:10BE600033680D2BF2D00D20F8F7FCFB2078F8F7A3
:10BE7000F9FB14F8013B3360A742EED1284603B02A
:10BE8000F0BD01F0B5FF4FF4FA6303604FF0FF30EF
:10BE900003B0F0BD002AF1DD164E8F1806E0F8F76A
:10BEA000E1FB14F8013B3360BC42E7D020780A285C
:10BEB000F5D133680D2BF2D00D20F8F7D3FB2078A5
:10BEC000EDE74FF0FF30704701F092FF0923036068
:10BED000DCE7002DB2DD2A462146304601ABFCF7F7
:10BEE0003FFA0028CDD1019B1F44A7E7702601200F
:10BEF000D43701206C260120022834DDF0B5033848
:10BF0000072883B02ADC204B4FF40B7707FB003760
:10BF1000D7F82832DB0721D50C4615460026B5F5A3
:10BF2000007F23DD01AB4FF4007221463846FCF759
:10BF3000E3FA50B9019BB3F5007FA5EB03051C4460
:10BF40001E44ECD2304603B0F0BD01F051FF4FF477
:10BF5000FA6303604FF0FF3003B0F0BD01F048FF1B
:10BF600009230360F6E74FF0FF307047002DE9DD4D
:10BF70002A462146384601ABFCF7BEFA0028E4D138
:10BF8000019B1E44DEE700BF702601202DE9F0432F
:10BF9000022883B040F39880C41E072C00F39480DD
:10BFA0004FF40B75794F05FB04F57E19D6F828324E
:10BFB000D90740F1898001A93046FCF7F9F800283B
:10BFC00050D1337C5A0663D51B066DD44FF40B75E4
:10BFD00005FB04F507EB05080198D8F82010DFF8F9
:10BFE000AC91F8F72BF900283CD1D8F82430DA7A54
:10BFF00042F02002DA72D8F8082059F805109A7633
:10C00000C2F30720D876097803296AD04FF40B725F
:10C0100002FB0472CB21D2681A77100A5877100CF1
:10C02000120E9877DA7799750022B22542205021B6
:10C030009A74DA74DD7518765976019B0122DA70EC
:10C04000019DEB78002B46D12B78032B4ED06B78DB
:10C05000022B15D94FF40B7303FB04731A7C22F0E7
:10C0600040021A744FF40B7000FB04740020D4F8E3
:10C07000283223F00103C4F8283203B0BDE8F0836E
:10C080004FF40B7303FB04731A7C22F040021A7402
:10C0900001A93046FCF78CF80028E3D14FF40B736C
:10C0A00003FB04F3F850DDE7019BF269587805F1D2
:10C0B000280139440123F7F7C7FD0028D2D1337C8A
:10C0C00003F07F03337481E701F092FE09230360DC
:10C0D0004FF0FF30D1E72846FCF748F80028B9D1E7
:10C0E000B2E7120C110A1A7559758FE72B79012BDB
:10C0F000ADD105F134010B4605F50D70002203F8B2
:10C10000012B83424FF00008F9D12869EB6885F8CC
:10C110001C024FEA102E85F81DE24FEA104E000E69
:10C120002A6A85F81EE285F81F024FEA132E180CC2
:10C1300085F820321B0E85F821E285F822024FF0A7
:10C14000550EAA2085F823325223013285F832E2B7
:10C1500085F833024FF0610E412085F8343085F8C0
:10C160003530722385F8370085F81A0285F81832C1
:10C1700085F819322A6385F836E085F81BE2012339
:10C180006878F7F761FD85F8048060E77026012084
:10C190002DE9F043DFF84C80D8F80030984283B0A6
:10C1A0001AD20F4E05460F1A06EB001600244FF068
:10C1B0001409002331462046CDF800903A4601F09C
:10C1C00067FDD8F800300135AB4204F1010406F1F7
:10C1D000100601D9142CECD103B0BDE8F08300BFE8
:10C1E00004380120DC37012003F07EBF08B5384A4F
:10C1F000536B13F0450FFBD059070DD413F0010317
:10C2000006D133490A69D2B290420AD0102008BD43
:10C210002F4B0120986308BD2D4B04229A63032005
:10C2200008BD40F2FF5218468A63F8F74BFA294BD3
:10C2300003402BB1002805DB420005D5092008BDCD
:10C24000184608BD1C2008BD830001D50A2008BD82
:10C25000C10001D50B2008BD020101D50C2008BD8D
:10C26000430101D50D2008BDC10101D50E2008BD37
:10C27000020201D50F2008BD4302C7D4810201D5B7
:10C28000112008BDC20201D5122008BD030301D54B
:10C29000132008BD410301D5142008BD820301D538
:10C2A000152008BDC30301D5162008BD010401D522
:10C2B000172008BD420401D5182008BD830401D50C
:10C2C000192008BD10F0080F0CBF00201A2008BD6F
:10C2D000002C014008E0FFFD10B5094B4020002272
:10C2E0000C244FF4806198605C6019611A60DA6018
:10C2F00001F050F82046BDE81040FFF777BF00BFBF
:10C300005C42012038B50F4A0F4B1268002012041E
:10C310004FF480610D244025D8601A609D6019613A
:10C320005C6001F037F82046FFF760FF08B102209B
:10C3300038BDF8F7C7F9C0F34320043818BF01200F
:10C3400038BD00BF043C01205C42012038B52A4BB7
:10C3500019685A69140601D5080600D438BD802131
:10C36000264A596113691906F8D413695B060ED47D
:10C37000234A1378591E072903D82248017849080F
:10C3800001700133DBB20A2B0DD8137038BD1C4A83
:10C390001378591E0729F4D81A480178490861F022
:10C3A0007F010170EDE7174C20780023F02813700F
:10C3B00013D0E02817D0144D144A2B881188184345
:10C3C000814205D0124B10801B6893B1114B18604D
:10C3D00000232B600023237038BD0B4A136843F4FD
:10C3E00000731360F6E7084A136843F48073136020
:10C3F000F0E7FFF7CFFBEBE7003C01400004024011
:10C40000E8370120D8370120E4370120E037012048
:10C41000E4080020DC080020F0B5254A254B1278FE
:10C4200083B053F8227020250023044602460E46AE
:10C4300018463946009501F02BFC224600231E4980
:10C440000095012001F024FC224600231B490095A1
:10C45000022001F01DFC009522460023184903200C
:10C4600001F016FC0095DEB933462246154904203A
:10C4700001F00EFC202522460095002312490520DC
:10C4800001F006FC114A124B92F88020009553F8F7
:10C49000221006202246002301F0FAFB03B0F0BD73
:10C4A000012322460B49042001F0F2FBE2E700BF22
:10C4B00000000020501C0108681C01082809010820
:10C4C000440901087C1C0108841C0108FC030020AD
:10C4D000601C0108701C01082DE9F04182B00024A5
:10C4E00080460094214640F2DF1340F21F324FF4A1
:10C4F000167000F033FEB8F1000F60D000944FF6D4
:10C50000FF734FF4167220216648FBF7F7FA664C6A
:10C51000664F00231E461D463B70FCF7F7FB236861
:10C520002660762B3CD0153B512B32D8DFE803F048
:10C530005E5C3131315A58565452313129B3B1AF62
:10C54000ADAB313131A9A7A5A3A131319F9D9B99F5
:10C55000979531313193918F8D8B31313189878529
:10C5600083813131317F7D317B3131313131313135
:10C570003131313131673131313131313131313175
:10C5800031606323062D04D87B5501357E55FCF7B9
:10C59000BDFB012000F092FD23682660762BC2D1FE
:10C5A00000240021009140F2DF1340F21F324FF4CB
:10C5B000167000F0D3FD204602B0BDE8F081CDF842
:10C5C00000804FF6FF734FF4167220213848FBF7B6
:10C5D00095FA9CE73223D5E77723D3E76123D1E7A8
:10C5E0007323CFE77A23CDE73123CBE77123C9E764
:10C5F000002DCED0013D7E55FCF788FBC9E7002D0C
:10C60000C7D02A48B8F1000F47D003F07FFD294A70
:10C610000346F91810681279F8500A71012000F0E9
:10C620004DFD224CBDE77023ACE76C23AAE72D2318
:10C63000A8E73923A6E73023A4E76F23A2E76923FD
:10C64000A0E76B239EE738239CE737239AE77523FF
:10C6500098E76A2396E76D2394E7362392E77923D8
:10C6600090E767238EE768238CE762238AE76E23CF
:10C6700088E7352386E7722384E7742382E76623FD
:10C6800080E776237EE733237CE734237AE765234C
:10C6900078E7642376E7782374E703F037FD064AEA
:10C6A0000346B6E7901C0108DC0800209424002013
:10C6B0009C1C010880040108780401082DE9F04F52
:10C6C00091B00024214640F2DF1340F21F3283462E
:10C6D00000944FF41670AD4E00F040FDAC4B34604A
:10C6E000224603A902A80293F8F74CFF00284FD076
:10C6F000002304930021A74C08468846FFF748FD15
:10C7000023684746762B454640F27519276017D0B7
:10C710005A2B29D026D9B3F5B97F13D04B4508D170
:10C720003DB1013DA84528BFA84640462946FFF730
:10C730002FFD012000F0C2FC23682760762BE7D193
:10C74000002517E03368013BAB42F2D9691CC8EB06
:10C750000103132B88BFA5F1120840460D46FFF7D1
:10C7600017FDE6E7292BE4D18B4B012003EB0515E0
:10C7700000F0A4FC0021009140F2DF1340F21F32D0
:10C780004FF4167000F0EAFC284611B0BDE8F08FB7
:10C79000039B0299049304A8F7F7B8FD0028A7D1DA
:10C7A0009DF93B30A342C0F2E5809DF81630DB06D0
:10C7B0009ED5039A0B991078CC7E8B7E032843EA92
:10C7C000042300F0D0800693D388ADF8143004A879
:10C7D00000F014FE04288BD0002889D16F4D4FF053
:10C7E0002E0803A904A8FBF7E3FC002862D1049CEF
:10C7F000042223E0F7F722FD00210246002854D14D
:10C800000B9F97F800E004A8BEF1000F75D0FB7AEB
:10C81000BEF1E50F03F03F0323F020098DF8163039
:10C8200007D0BEF12E0F04D00F2B02D0B9F1080FA4
:10C8300068D1F7F74DFB0246002836D10A9B204607
:10C840001946002BD6D1002A40F09B80534C6A72C7
:10C85000002104A8F7F73CFB042800D050BB637A02
:10C8600043B34F4C204603F051FCC3B2042B814626
:10C87000B7D9043B1C44BBF1000F2BD020464949DB
:10C8800003F006FC0028ACD13468DFF800A13F2C8F
:10C89000A7D84148424900EB041009F101020134D4
:10C8A00001F0DEFECAF800409BE7002312F0FB0F08
:10C8B0000A9323D003A904A8FBF77AFC00B90490DB
:10C8C000316801297FF616AF374B3348102202F04A
:10C8D00001F80FE73549204603F0DAFB0028D3D0F2
:10C8E0003349204603F0D4FB0028CDD020463149FF
:10C8F00003F0CEFB0028C7D073E70A9200236B72C7
:10C90000264CA5E70A9B6A72244C002BA0D0114646
:10C9100007F1FF3E1EF8013F202B01F1010107D076
:10C92000052B08BFE523092926D0A8180132437238
:10C930000B29EFD12A447B7FF98B97F817E0002071
:10C94000507243EA01213B7FFA7A2A7243EA0121BD
:10C95000BA7D787E3B7E296042EA0E2243EA0023BC
:10C96000EA80AB8074E7487D097D41EA002143EA13
:10C97000014328E7039A27E7A818013280F80980C5
:10C98000D3E7042A0A9395D1B8E700BFDC3701202A
:10C99000AC1C0108DC08002004380120EC37012021
:10C9A000F5370120B01C0108E9C100087004010836
:10C9B000780401088004010843695869704700BF82
:10C9C000C36858699B691840704700BFC3685869BD
:10C9D00000F00100704700BF30B4C4786CB900EBC0
:10C9E000820003339B10D0F8D05006D0224601328B
:10C9F00051F8040B28609342F9D1002030BC7047F5
:10CA000080B586B000AF78607B685B691B69BB60EE
:10CA10003B7BC3F3C303DBB27A685B01134403F5CA
:10CA20006F731B6803339B08FB8296E03B899B0076
:10CA3000BB82BA8A3B7BC3F3C303DBB279685B0179
:10CA40000B4403F56F731B689A4219D93B7BC3F300
:10CA5000C303DBB27A685B01134403F56F731B6891
:10CA6000BB8200233B61FB7C43F00403FB747B68C7
:10CA7000DB687A68D26891693A69D2430A409A6160
:10CA80003B7BC3F3C303DBB27A685B01134403F55A
:10CA90006F731B6803339B08FB823B7BC3F3C303A9
:10CAA000DBB27A6815335B01134403F58C731968A4
:10CAB0003B7BC3F3C303DBB21A46BB8A7868FFF73C
:10CAC0008BFF3B7BC3F3C303DBB218463B7BC3F353
:10CAD000C303DBB27A6815335B01134403F58C732F
:10CAE0001A68BB8A1A44796800F115035B010B448C
:10CAF00003F58C731A603B7BC3F3C303DBB21846A8
:10CB00003B7BC3F3C303DBB27A685B01134403F5D9
:10CB10006F731A68BB8AD21A796843010B4403F514
:10CB20006F731A603B7BC3F3C303DBB218463B7BD6
:10CB3000C3F3C303DBB27A685B01134403F570737C
:10CB40001A68BB8A1A44796843010B4403F5707371
:10CB50001A607B685B691B69BB603B89FA8A9A42F1
:10CB60000CD23B7BC3F3C303DBB27A685B01134493
:10CB700003F56F731B68002B7FF458AF0123184631
:10CB80001837BD4680BD00BF80B588B000AF786063
:10CB90007B68DB68DB6AFB603B7CC3F3C303DBB20F
:10CBA0007A685B01134403F56F731B6803339B08BA
:10CBB000FB8396E0BB899B00BB83BA8B3B7CC3F3B2
:10CBC000C303DBB279685B010B4403F56F731B6829
:10CBD0009A4219D93B7CC3F3C303DBB27A685B0189
:10CBE000134403F56F731B68BB830023BB613B7E5B
:10CBF00043F020033B767B68DB687A68D2689169F2
:10CC0000BA69D2430A409A613B7CC3F3C303DBB2E7
:10CC10007A685B01134403F56F731B6803339B0849
:10CC2000FB833B7CC3F3C303DBB27A6815335B0140
:10CC3000134403F58C7319683B7CC3F3C303DBB265
:10CC40001A46BB8B7868FFF7C7FE3B7CC3F3C30370
:10CC5000DBB218463B7CC3F3C303DBB27A681533FF
:10CC60005B01134403F58C731A68BB8B1A44796813
:10CC700000F115035B010B4403F58C731A603B7CD8
:10CC8000C3F3C303DBB218463B7CC3F3C303DBB27D
:10CC90007A685B01134403F56F731A68BB8BD21A71
:10CCA000796843010B4403F56F731A603B7CC3F34F
:10CCB000C303DBB218463B7CC3F3C303DBB27A6821
:10CCC0005B01134403F570731A68BB8B1A447968CF
:10CCD00043010B4403F570731A607B68DB68DB6A01
:10CCE000FB60BB89FA8B9A420CD23B7CC3F3C30333
:10CCF000DBB27A685B01134403F56F731B68002B8A
:10CD00007FF458AF012318462037BD4680BD00BFD1
:10CD100080B584B000AF78600023FB60084B1B68CF
:10CD20009B6878689847FB7B43F02003FB737B6824
:10CD3000DB68FA685A61012318461037BD4680BD8A
:10CD40003C18010880B584B000AF78600023FB6018
:10CD5000084B1B681B68786898473B7B43F00803C7
:10CD60003B737B68DB68FA685A6101231846103709
:10CD7000BD4680BD3C18010800EB81014FF0004327
:10CD8000D1F89020012060F3DC431361D1F89020AA
:10CD90001368002043F0004360F39E7313607047F4
:10CDA00000EB810186B0D1F89020136843F0404336
:10CDB00059030AD541690969C1F3074109B96FF3FC
:10CDC000DF730020136006B07047C168C96AC1F301
:10CDD00007410029F3D00020136006B0704700BF60
:10CDE000F0B54C01051987B0D5F8BC330022D3B19A
:10CDF000B5F8B263013B3344B3FBF6F39BB2B3F532
:10CE0000807F64D93602C5F8BC6305194FF480777A
:10CE100095F8AE633B466EB1B5F8B26303FB06F31B
:10CE2000C5F8BC3308E001273B46051995F8AE6309
:10CE3000002EF1D1D5F8BC3301F1150600EB4615F3
:10CE400000EB810163F3120295F814E1D1F8903000
:10CE500067F3DC426EF35E721A61C378012B39D03E
:10CE6000D1F8905042692B68926802F0010282F07A
:10CE7000010262F35D7343F000436FF39E732B6016
:10CE8000C3780BBB021992F8AE33EBB9D2F8BC33BE
:10CE9000D3B192F8B123032A2BD8DFE802F02102A4
:10CEA0002102426915690195DA1CADB2C2F38F0205
:10CEB00095421ED2C268936943F080639361044433
:10CEC000C278D4F8BC33A2B1002007B0F0BDC3F3E0
:10CED0000907AAE7D1F89030D5F818215A61BFE7C1
:10CEE000C768FD6A0395DA1CADB2C2F38F029542A2
:10CEF00011D300EB4610D1F8D040D0F8182198B2E9
:10CF000003308010E0D00023013352F8041B21606D
:10CF10009842F9D1D8E7BB6943F02003BB610444D0
:10CF2000C278D4F8BC33002ACED1E2E7F0B400EBEB
:10CF300081054FF0FF34D5F890204B019460C41860
:10CF4000C27894F8B163012A14BF0024042400229B
:10CF5000032E13D8DFE806F002550249C61844F440
:10CF6000936496F8AE7344F00104002F46D196F80E
:10CF7000B06344F040040EB144F02004D5F8906052
:10CF8000F46047690126BC6906FA01F12143B961E1
:10CF9000C468A169184441F00073A36190F8AC73B0
:10CFA00090F8AF3390F8AD6390F8AE4390F8B113BA
:10CFB000B0F8B20367F39C52A3F1020366F3CE22EA
:10CFC000B3FA83F364F3CF325B0963F3514261F345
:10CFD000934260F30A02D5F89030032908BF42F06B
:10CFE00000521A600020F0BC7047C61844F4D364A5
:10CFF00096F8AE6344F00104002EBFD044F4807470
:10D00000BCE7C61844F4087496F8AE6344F0010413
:10D01000002EB3D044F4C074B0E700BF4269136877
:10D0200061F301031360704730B403329210D0F8FB
:10D03000D05009D00846002301332C6840F8044B37
:10D040009A42F9D101EB8201084630BC704700BF1B
:10D05000094A0A4B02FB00F0A3FB0023C21A82B06C
:10D0600003EB5202002392080193019B01339A4281
:10D070000193FAD202B07047C0D40100254992242E
:10D0800010B504460A20D4F8CC2013686FF382034D
:10D090006FF341036FF3C3036FF3451343F48071E0
:10D0A0001160FFF7D5FFD4F8CC306FF30821196079
:10D0B0001420FFF7CDFF012010BD00BF2DE9F8437C
:10D0C0000446FBF7C5FA1D4B1B78012B10D01C4AF8
:10D0D0001178994218BF13701A4B1A680AB9BDE843
:10D0E000F88319494020002208831A60BDE8F883BC
:10D0F000144A1168E1B1154E154D3168DFF85880BA
:10D10000144FA9462B688B4203F10102E7D0202A75
:10D1100038F8130008D0C9F800200CB13860F1E7E6
:10D12000FEF738FD3168EDE70023C9F80030F4E779
:10D130000549402048831360DDE700BF60260120D9
:10D14000AD0000200C3C012000000240B42501206D
:10D15000083C0120DC080020B825012070B55C1ACD
:10D160000D461E461146131A013403FB0444FAF718
:10D1700023FC31462846FAF70BFC4FF0C0432C2223
:10D180001A803CB10449BDF81020002301339C42B1
:10D190000A80FBD170BD00BF0000086080B586B07A
:10D1A00000AF786000237B6100233B617868FFF764
:10D1B00003FC0346FB6000237B612AE0BB891A461F
:10D1C0007B6942FA03F303F00103002B1ED07A6857
:10D1D0007B6922339B0013449B681B68BB607B7A8E
:10D1E00023F07F03DBB2002B08D079697868FDF764
:10D1F000DBF802463B6913433B6107E079697868D5
:10D20000FDF7ACFB02463B6913433B617B6901338D
:10D210007B617B681B781A467B699A42CED83B6952
:10D2200018461837BD4680BD80B584B000AF786021
:10D230000023FB600023BB607868FFF7C7FB034651
:10D24000002B71D07868FFF7BBFB0346BB60BB685F
:10D25000002B01D1002368E03B7A03F00803DBB226
:10D26000002B06D07868FFF76DFD0246FB6813437C
:10D27000FB603B7A03F01003DBB2002B06D078682A
:10D28000FCF7C6FF0246FB681343FB603B7A03F0E2
:10D290002003DBB2002B06D07868FFF775FC02464E
:10D2A000FB681343FB60FB7A03F00403DBB2002B43
:10D2B00006D07868FFF7A4FB0246FB681343FB60C7
:10D2C000FB7A03F00203DBB2002B06D07868FFF78D
:10D2D00065FF0246FB681343FB60FB7A03F0010322
:10D2E000DBB2002B06D07868FDF7E2FD0246FB6852
:10D2F0001343FB60FB7A03F02003DBB2002B06D064
:10D300007868FFF705FD0246FB681343FB60BB7AB4
:10D3100003F02003DBB2002B06D07868FCF750FF47
:10D320000246FB681343FB60FB6818461037BD4696
:10D3300080BD00BF0148FFF777BF00BF2C3C012034
:10D34000044B1A6A42F400121A621A6A22F400129A
:10D350001A6270470038024082B00023020F0C4965
:10D360000093019301910092009B20F07F4053B104
:10D37000019B14330193019B1B68034214BF0120DE
:10D38000002002B07047019B1833000C0193F2E7B4
:10D390000054004070B40A4A0A4913688B6056680A
:10D3A0009568D468CB68106946EA0502224323F4E5
:10D3B000FF6323F0070302431343CB6070BC704745
:10D3C0005C420120002C014070B40A4B0A49DD6820
:10D3D00093E8450048621C698A625869CA6A46EA4D
:10D3E0000503234322F0F70203431343CB6270BCCF
:10D3F000704700BF143C0120002C014038B5816803
:10D4000005680023036129B92B78022B14D9AB6A74
:10D4100093B119466B89E3B90446284605E0012813
:10D420000CD9AB69984209D22068FAF7BFFB431CBC
:10D430000146F4D1012038BD2B890BB9022038BD3B
:10D44000AB6A83614161002BF8D03435C56100209F
:10D4500038BDAA698C1E023A944236BFEA6A00239C
:10D4600004FB03238361EDE738B50546652405E039
:10D47000013C4FF0320009D0F7F76CF82846FFF76F
:10D480006BFF0028F4D00124204638BDFEF75EFC77
:10D49000FAE700BF10B4154B18790022012140248F
:10D4A00007289C711A705A709A7083F82020D970DE
:10D4B000197783F8211008D80D4A00F5317002EB76
:10D4C00040008288C2F30E0282805B79072B08D865
:10D4D000074A03F5317302EB43039A88C2F30E0245
:10D4E0009A8000205DF8044B704700BFD8410120AE
:10D4F0002C3C0120031F012B09D9062800D07047BE
:10D50000074B0A21D3F8802019701368184710B50B
:10D51000034CD4F880305B6C98470A23237010BD0D
:10D52000D8410120F8B5194C194DFF2740F440703F
:10D53000802306220E4640F2094EE0822375627572
:10D5400021463B4605F588722846A4F818E0678313
:10D55000FDF746FF18B995F81131032B00D0F8BD3F
:10D5600095F810110239B942A8BF394689B249B1BC
:10D570000346EA1802339BB292F8122106F8012BF7
:10D580009942F6D800233370F8BD00BFD84101207E
:10D590002C3C01202DE9F04FDFF830B2874C0546D6
:10D5A0000346802106224FF400708BF814108BF88C
:10D5B0001520ABF816008DB00026594604F5887288
:10D5C0002046ABF81A50ABF81860FDF709FF844607
:10D5D000002840F0D08094F8132194F8101194F8AA
:10D5E00012318BF8341094F8111194F815018BF85E
:10D5F000351003EB022394F8161194F814218BF8DC
:10D6000039009BB294F817018BF83A10092D94F861
:10D610001811ABF836308BF838208BF83B008BF8BC
:10D620003C1040F2A880022A00F29C80644A6549BE
:10D6300092F800900D8809920A9104F5887ECDF841
:10D6400000C04FF009080BF1500A984580F0848023
:10D650009EF80020964490449EF80120042A1FFA68
:10D6600088F8F2D19EF80340022CEED89EF8040010
:10D670000228EAD89EF8002003929EF805209EF822
:10D68000023004929EF8062005929EF8072001932E
:10D6900006925BB29EF8082007924B4902931AB299
:10D6A00002EBC203120108920B440022CDF82CC0F9
:10D6B00082424ADA9EF800108E4441449EF801608E
:10D6C000052E1FFA81F8F3D102999EF8057089455D
:10D6D00055D09DF80C1019704FF0040159709DF849
:10D6E000101059719DF8141099719DF81810D97186
:10D6F0009DF81C10DDF80490197201259EF80410A5
:10D7000083F80290DC7018713F02009508252E46C0
:10D71000089D16FB02567D1801320AEB06019EF8A1
:10D7200000700AF8067052B29EF802709EF803600C
:10D730008F70ADB24FF0050C9EF806708D8082425E
:10D7400081F801C0CE708F71B4DBBBF83630DDF8E4
:10D750002CC09845FFF47CAF009B3BB1099B83F83C
:10D76000009003E0164B0993164B0A930A9A002384
:10D770001380099A137060460DB0BDE8F08F9EF8D3
:10D7800004103F027E18B542DFDC9DF80C501D707E
:10D790004FF004055D709DF804509D709DF8105089
:10D7A0005D719DF814509D719DF81850DD719DF8C4
:10D7B0001C50DC7018711D72A8E700BF2C3C0120C2
:10D7C000103C01207042012016420120D841012066
:10D7D000F8B52E4C2E4D06468021062203464FF406
:10D7E0008070002721756275E082214605F58872F8
:10D7F000284666832783FDF7F3FD00B1F8BD95F851
:10D80000132195F8123195F8101195F811E184F86B
:10D81000221003EB022395F8147195F81511A384D7
:10D8200095F8162195F8173184F823E0082E84F82E
:10D83000267084F8271084F8282084F82930DDD950
:10D8400095F819E195F8181195F81B7195F81D6177
:10D8500095F81A2195F81C3101EB0E2102EB0722F5
:10D8600003EB062395F81EE195F81F71618595F885
:10D87000206195F82111A285E38584F830E084F8D1
:10D88000317084F8326084F83310F8BDD84101203B
:10D890002C3C01202DE9F0411A491B4800F03AFDCB
:10D8A00050B304460025194FDFF8748006E0236862
:10D8B0005A1C2260187808F8060001356368013B9D
:10D8C000002B6360AEB2F2DA2146386801F0CAF983
:10D8D000431CF0D10E4B20461E8000F0F5FA0622C4
:10D8E0000C490D4802F036F820B90C4B01221A60A1
:10D8F000BDE8F081BDE8F0810348BDE8F04100F0EB
:10D90000A7BF00BF4C040108DC010020200100205B
:10D9100080420120241D0108165E0020F80300202B
:10D92000A825002010B54368013B002B0C4643603E
:10D9300006DB03685A1C026018782070012010BDB5
:10D94000044B0146186801F08DF9431CF5D1002005
:10D9500010BD00BF2001002030B583B00D460DF191
:10D9600007010446FFF7DEFF10B9002003B030BD09
:10D9700020460DF10601FFF7D5FF0028F5D09DF8F0
:10D9800006209DF80730012043EA02232B8003B0D4
:10D9900030BD00BF70B506460D46FF203146144627
:10D9A00001F04EFE3146FF2001F04AFE2846314686
:10D9B00004F57F5501F044FE064B3F35013C1D4404
:10D9C0001C4414F8010F314601F03AFEAC42F8D184
:10D9D00070BD00BFA825002038B505460C46C8B26A
:10D9E000294601F02DFE2946200ABDE8384001F005
:10D9F00027BE00BF0209130700F00F000AD410B4BD
:10DA0000094901238C5C03FA00F0204388545DF837
:10DA1000044B7047054901220B7802FA00F023EA13
:10DA200000000870704700BFB4000020724201205F
:10DA300003091A0700F00F000BD410B4094C0121A0
:10DA4000E25C01FA00F022EA0000E0545DF8044BC9
:10DA50007047054901220B7802FA00F0184308705C
:10DA6000704700BFB400002072420120184A92F8AB
:10DA7000C83092F8C910B3FA83F302294FEA53135E
:10DA800023D003291ED0012919D0002182F8C91002
:10DA9000104913F0010F0B6014BF002208229907F0
:10DAA00048BF42F002025B0748BF42F001024FF05C
:10DAB000C041094B92B2362008801A80704743F06B
:10DAC0000403E5E743F00603E2E743F00203DFE780
:10DAD000FC030020B000002000000860F0B5134AED
:10DAE000134C14491448154FDFF868E0144E154DD7
:10DAF000DFF864C000231360536093602380124AF0
:10DB00000B70124C1249037003203B7023601360AA
:10DB1000536093600870AEF8003033702B70BDE82E
:10DB2000F040ACF80030FDF7BBBB00BF74420120F1
:10DB3000D8080020EE02002082420120834201200A
:10DB4000F4030020D8010020DC02002084420120E0
:10DB5000BC00002002090020F002002030B5154D65
:10DB6000154C83B000230193FBF708FAEB681A69A0
:10DB7000019206E0FBF702FAEB68013C1A69019298
:10DB800015D0019A002AF5DA01990B4A41F00101FA
:10DB90000191019919611969019103E019690191D4
:10DBA000013A02D00199C907F8D4FBF7E7F9002040
:10DBB00003B030BD2C3C0120400D0300034A0B880C
:10DBC00012889A429CBF024AD0547047804201207A
:10DBD000A825002070B4214B1B78FBB9204B1B7883
:10DBE0005BB906292BD01F4C1F4D2268695C083297
:10DBF00022608170038070BC70471B4B194C9E7A69
:10DC0000D97A2368194D41EA06210A4492B21733A2
:10DC100023600280AB5C837070BC70471249114C6A
:10DC20000E7A4B7A2168114D43EA06231A4492B2C8
:10DC3000173121600280AB5C837070BC70470A4C66
:10DC4000084925790A686379084C43EA05230F32AD
:10DC50000A600380E35C8370CDE700BF824201204D
:10DC6000834201208442012074420120A825002023
:10DC7000024A937943F00403937170477442012080
:10DC8000024A937943F01003937170477442012064
:10DC900070B5824204469DF8106019D04FF6E072CC
:10DCA0004FF6FF75012B08BF15460B460A4A0B4875
:10DCB000152102F0BBF904FB06F1002204922B4669
:10DCC00020314FF416720548BDE87040F9F716BFD1
:10DCD0004FF47845E9E700BF2C1D01088842012078
:10DCE0000649074A074B9A42BEBF51F8040B42F857
:10DCF000040BF8E7044880470448004778250108EA
:10DD0000000000203001002079780008E5010008BB
:10DD10003349344A002301E041F8043B9142FBD3EC
:10DD2000F4F72AFDFEE7FEE7FEE7FEE7FEE7FEE783
:10DD3000FEE7FEE7FEE7FEE7FEE7FEE7FEE7FEE7BB
:10DD4000FEE7FEE7FEE7FEE7FEE7FEE7FEE7FEE7AB
:10DD5000FEE7FEE7FEE7FEE7FEE7FEE7FEE7FEE79B
:10DD6000FEE7FEE7FEE7FEE7FEE7FEE7FEE7FEE78B
:10DD7000FEE7FEE7FEE7FEE7FEE7FEE7FEE7FEE77B
:10DD8000FEE7FEE7FEE7FEE7FEE7FEE7FEE7FEE76B
:10DD9000FEE7FEE7FEE7FEE7FEE7FEE7FEE7FEE75B
:10DDA000FEE7FEE7FEE7FEE7FEE7FEE7FEE7FEE74B
:10DDB000FEE7FEE7FEE7FEE7FEE7FEE7FEE7FEE73B
:10DDC000FEE7FEE7FEE7FEE7FEE7FEE7FEE7FEE72B
:10DDD000FEE7FEE7FEE7FEE7FEE7FEE7FEE7000000
:10DDE00030010020B04201200A22002101F026BAB1
:10DDF000014B1868704700BF2001002008B5074B91
:10DE0000044613B10021AFF30080054B1868836A04
:10DE100003B19847204601F02DFD00BF000000002F
:10DE2000981D010870B505460C4609B9002070BD63
:10DE300018B183690BB900F0BFF9204B9C4201D1A6
:10DE40006C6808E01E4B9C4201D1AC6803E01D4B9E
:10DE50009C4208BFEC68B4F90C30002BE6D0214698
:10DE6000284600F039F8236B064633B1216A28466C
:10DE700098470028B8BF4FF0FF36A3891B0603D58B
:10DE80002169284600F000FC616B41B104F14403B4
:10DE9000994202D0284600F0F7FB00236363A16C8F
:10DEA00021B1284600F0F0FB0023A36400F0F0F954
:10DEB0000023A38100F0EDF9304670BD341D010848
:10DEC000541D0108741D0108024B01461868FFF734
:10DED000A9BF00BF200100208A892DE9F041054635
:10DEE00010070C4659D44B68002B02DC0B6C002B3E
:10DEF00017DDE66AAEB102F48052002392B22F68B9
:10DF00002B600AB1606D15E0216A01232846B047F5
:10DF1000411C0FD12B686BB11D2B01D0162B03D1E7
:10DF20002F600020BDE8F081A38943F04003A38166
:10DF3000BDE8F081A3895A0705D56368C01A636BF1
:10DF40000BB1236CC01A00230246E66A216A2846F8
:10DF5000B047431CA38906D129681D293AD8214A14
:10DF6000CA40D60736D500226260D90422692260F1
:10DF700004D5421C01D12B6803B96065616B2F6029
:10DF80000029CED004F14403994202D0284600F083
:10DF90007BFB00206063BDE8F0810F69002FC0D0DB
:10DFA00093070E6808BF4B690F6018BF0023C7EBCB
:10DFB00006088B6002E00744C0EB0808B8F1000FC8
:10DFC000AFDD43463A46216AA66A2846B047002894
:10DFD000F1DCA38943F04003A3814FF0FF30BDE89B
:10DFE000F08100BF0100402038B50B6905460C46A2
:10DFF000DBB118B183690BB900F0DEF80C4B9C4221
:10E0000001D16C6808E00B4B9C4201D1AC6803E085
:10E01000094B9C4208BFEC68B4F90C302BB1214687
:10E020002846BDE83840FFF757BF002038BD00BF85
:10E03000341D0108541D0108741D0108014620B952
:10E04000044B0549186800F017BA044B1868FFF72D
:10E05000CBBF00BF981D0108E9DF000820010020A8
:10E06000012A2DE9F04781460E4690461C4602DC07
:10E070000020BDE8F08718B183690BB900F09CF867
:10E08000254B9C4202D1D9F804400AE0234B9C4224
:10E0900002D1D9F8084004E0214B9C4208BFD9F8CE
:10E0A0000C4008F1FF383746656845B921464846B7
:10E0B00000F050FD10B1B74229D1D9E76568D4F816
:10E0C00000A0454528BF45462A460A21504600F093
:10E0D00077FA636868B10130CAEB00055B1B84E81E
:10E0E00009002A465146384600F0BAFA00237B550B
:10E0F0000FE05B1B636023682B44384623602A468D
:10E10000514600F0ADFAB8EB05082F44CCD10023FE
:10E110003B703046BDE8F087341D0108541D0108EE
:10E12000741D010813460A46014602480068FFF7BD
:10E1300097BF00BF20010020014900F09DB900BF3A
:10E14000E9DF0008002310B50446036043608360E4
:10E1500081814366C281036143618361194608225C
:10E160005C3000F088FA054B6362054BA362054BF7
:10E17000E362054B2462236310BD00BFDDEC0008A1
:10E18000FFEC000837ED00085BED000870B5682370
:10E190004D1E5D430E4605F1740100F0C3FA0446BE
:10E1A00040B1002180E842000C30A06005F1680217
:10E1B00000F061FA204670BD836910B5044633BB98
:10E1C0008364C3640365124B124A1B6882629842DF
:10E1D00004BF0123836100F01FF86060204600F057
:10E1E0001BF8A060204600F017F80022E060042130
:10E1F0006068FFF7A7FF01220921A068FFF7A2FFCF
:10E2000002221221E068FFF79DFF0123A36110BDE8
:10E21000981D010839E10008F8B51C4B1E68B36968
:10E22000074613B93046FFF7C7FF4836B46873682E
:10E23000013B04D4B4F90C507DB16834F8E733687D
:10E240000BB13668F2E704213846FFF79FFF3060D4
:10E250000028F6D10C233B60F8BD4FF6FF73E38135
:10E260000123A38165662560A56065602561656100
:10E27000A5610822294604F15C0000F0FCF9656301
:10E28000A563A564E5642046F8BD00BF981D01089C
:10E2900070477047F7B50F46114601AA054601F0D1
:10E2A00073F9064608B9002029E02846FFF7B4FFB5
:10E2B00004460028F7D04FF4DB73019A394628460C
:10E2C00000F08EFA002806DA0025FFF7E1FFA581AD
:10E2D000FFF7DFFFE7E70B4B63620B4BA3620B4BD0
:10E2E000E3620B4B2363F305E081A681246205D52D
:10E2F000022300222146284600F014F8204603B0ED
:10E30000F0BD00BFDDEC0008FFEC000837ED0008B1
:10E310005BED0008024B0A4601461868FFF7BABFDA
:10E320002001002000F000B82DE9F8430C4690468B
:10E330001E46054618B183690BB9FFF73DFF3D4BFB
:10E340009C4201D16C6808E03B4B9C4201D1AC6817
:10E3500003E03A4B9C4208BFEC68A38903F4847342
:10E36000B3F5847F03D121462846FFF73DFEE76AD7
:10E370000FB91D232BE0012E04D0022E2BD056B353
:10E38000162324E021462846FFF72EFEA28902F438
:10E39000805292B20AB1606D05E0216A3346284688
:10E3A000B847411C14D0A3895A0706D56368C01A20
:10E3B000636B4BB1236CC01A06E01B0704D52368BE
:10E3C00013B122699B1A18448044002603E02B6095
:10E3D0004FF0FF392BE023691BB92146284600F096
:10E3E000B3F821462846FFF7FFFD81460028EFD10C
:10E3F00033464246216A2846B8470130E8D0616B6F
:10E4000041B104F14403994202D0284600F03CF99E
:10E410000023636323692360A389002123F402633B
:10E420006160A381082204F15C0000F024F94846F1
:10E43000BDE8F883341D0108541D0108741D01084E
:10E440002DE9F041884600F1480400268CB1A5680A
:10E450006768013F0BD4AB89012B06D9B5F90E30A3
:10E46000013302D02846C04706436835F1E72468E7
:10E47000ECE73046BDE8F0812DE9F8438046894657
:10E4800000F14804002694B1A5686768013F0CD4E8
:10E49000AB89012B07D9B5F90E30013303D02946DA
:10E4A0004046C84706436835F0E72468EBE7304646
:10E4B000BDE8F88370B50E4B0E4CE41AA41000258D
:10E4C0001E46A54204D056F8253098470135F8E796
:10E4D00001F0A0FF084C094BE41AA41000251E46C9
:10E4E000A54204D056F8253098470135F8E770BDAD
:10E4F00028010020280100202C01002028010020F4
:10E5000070B50E46B1F90E10002990B014461D46A4
:10E5100006DA00232B60B3891A060ED540230EE0DD
:10E5200001AA01F0E3F80028F3DB029A02F470423A
:10E53000A2F500535A425A412A604FF480630020EA
:10E54000236010B070BD00008B8973B59E0705462F
:10E550000C4610D401AB6A46FFF7D2FF009906467D
:10E56000284600F0DFF868B9B4F90C309A0522D4D7
:10E5700043F00203A38104F14703236023610123D5
:10E58000636118E00D4BAB62A389206043F0800308
:10E59000A381009B6361019B20614BB1B4F90E1014
:10E5A000284601F0B5F818B1A38943F00103A3810F
:10E5B000A0893043A08102B070BD00BF39E10008DE
:10E5C00001F0FF01102A2BDB10F0070F08D010F824
:10E5D000013B013A8B422DD010F0070F42B3F6D128
:10E5E000F0B441EA012141EA014122F007047FF041
:10E5F00000070023F0E80256083C85EA010586EA98
:10E60000010685FA47F5A3FA87F586FA47F6A5FAD3
:10E6100087F68EB9EED1F0BC01F0FF0102F00702DF
:10E6200032B110F8013B013A83EA010313B1F8D18A
:10E630000020704701387047002D06BF354603386B
:10E64000073815F0010F07D1013015F4807F02BFA4
:10E65000013015F4C03F0130F0BC0138704700BFF5
:10E6600010B5431E0A44914204D011F8014B03F83F
:10E67000014FF8E710BD02440346934202D003F86D
:10E68000011BFAE77047000038B50546002946D05F
:10E6900051F8043C0C1F002BB8BFE41801F05AF8E5
:10E6A0001F4A1368114613B96360146032E0A34235
:10E6B0000ED92268A018834204BF18685B686360A3
:10E6C00004BF121822600C6024E0A24203D8134653
:10E6D0005A68002AF9D118681918A1420BD121688B
:10E6E000014458188242196014D1106852685A6067
:10E6F000014419600EE002D90C232B600AE0216866
:10E700006018824204BF10685268626004BF091832
:10E7100021605C602846BDE8384001F01CB838BD77
:10E72000A442012070B5CD1C25F0030508350C2D41
:10E7300038BF0C25002D064601DBA94202D90C2367
:10E74000336046E001F006F8234B1C681A46214668
:10E75000A1B10B685B1B0ED40B2B03D90B60CC183B
:10E76000CD501EE08C420DBF63684B686360136040
:10E7700018BF0C4615E00C464968E9E7174C2368BA
:10E780001BB9304600F09AFA20602946304600F066
:10E7900095FA431C18D0C41C24F00304A0420DD1E8
:10E7A0002560304600F0D7FF04F10B00231D20F058
:10E7B0000700C31A0ED05A42E25070BD211A3046EB
:10E7C00000F07CFA0130EBD10C233360304600F0CE
:10E7D000C2FF002070BD00BFA4420120A042012062
:10E7E00038B5074C054608461146002222601A46F5
:10E7F000F9F7CCFA431C02D1236803B12B6038BD72
:10E80000AC42012037B50D46044618B183690BB9F7
:10E81000FFF7D2FC4DB12B783BB1E168284600F000
:10E820005DFFE168094800F059FF01AB0122216852
:10E83000204600F097FA10B1E16800F04FFFE16860
:10E840000A2000F0FDFE03B030BD00BF9C1D010892
:10E85000024B01461868FFF7D5BF00BF200100201A
:10E86000012B30B50ADC9208013A03680C6840F8C5
:10E87000044B002A41F8043BF6DC30BD03460D781A
:10E880001C7803F8015B01F8014BD41A0444002CF6
:10E89000F5DC30BDF8B50F46144606461D469847D0
:10E8A0000028214638460BDAA847002801DA384606
:10E8B000F8BD21463046A847002809DB3046F8BDA0
:10E8C000A8470028F3DC21463046A8470028F5DB9E
:10E8D0002046F8BD2DE9F04F85B006468B4614461C
:10E8E0000093B20707D1A30705D1B4F1040818BFFC
:10E8F0004FF0010801E04FF002083319BBF1060F99
:10E90000019326D81F4604FB0B65AF4280F01681A9
:10E91000B9464E4501D32744F7E7C4EB090A4946F7
:10E920005046009B98470028F5DDB8F1000F08D14C
:10E93000D9F80030DAF80020C9F80020CAF8003011
:10E9400005E04346224651464846FFF789FFD14637
:10E95000DFE74FEA5B050BF1FF33BBF1070F04FB69
:10E960000565019326D0BBF1280F04FB036919D973
:10E970004FEADB076743F119CA19009B3046FFF7DE
:10E9800089FFEA192946009B8246E81BFFF782FFB0
:10E990000546A9EB47004A46009BC119FFF77AFFDD
:10E9A000814600E0B2462946009B4A465046FFF7A2
:10E9B00071FF0546B8F1000F04D133682A68326050
:10E9C0002B6005E04346224629463046FFF748FFC4
:10E9D000019B371904FB03653B190293A946019774
:10E9E0000023029AC4EB020A554555D303933146DE
:10E9F000009B504698470028039B24DC15D1B8F1B2
:10EA0000000F08D1019B01991B68DAF800200A6009
:10EA1000CAF8003005E04346224651460198FFF708
:10EA20001FFF019B234401930123029A2244029277
:10EA3000D7E703933146009B284698470028039B5D
:10EA400018DB03D02D1B5545F3D225E0B8F1000F9C
:10EA500006D12B68D9F800202A60C9F8003005E0FB
:10EA60004346224649462846FFF7FAFEC4EB090909
:10EA70000123E7E7B8F1000F06D1DAF800302A6881
:10EA8000CAF800202B6005E043462246294650463E
:10EA9000FFF7E6FE2D1BC7E704FB0BFB63B3019BEF
:10EAA00006EB0B079A1BC3EB0A0B5A45A8BF5A4645
:10EAB0002AB14346C2EB0A013046FFF7D1FEC9EB4B
:10EAC0000702C5EB0905121BAA4228BF2A4622B13C
:10EAD0004346B91A5046FFF7C3FE5C4506D2BBFB5E
:10EAE000F4F1009B22463046FFF7F4FEAC4225D2FB
:10EAF000B5FBF4FB7E1BF4E6B3445F451ED23D46F6
:10EB0000AE4201D32744F8E7C4EB0509294648463D
:10EB1000009B98470028F5DDB8F1000F06D12B685F
:10EB2000D9F800202A60C9F8003005E043462246A3
:10EB300049462846FFF794FE4D46E1E705B0BDE89B
:10EB4000F08F838903F00903092B01D1FFF776BA0F
:10EB500000207047F8B50C46054618B183690BB91B
:10EB6000FFF72AFB3A4B9C4201D16C6808E0394B15
:10EB70009C4201D1AC6803E0374B9C4208BFEC6873
:10EB8000B4F90C200023636093B29E065BD458074F
:10EB90001AD4D90605D4092342F040022B60A28181
:10EBA00051E01A070BD521462846FFF71DFA002829
:10EBB00049D1A389A06023F00803A381A061A389A0
:10EBC00043F00403A38110E0616B71B104F14403CD
:10EBD000994202D02846FFF757FD236C636000205E
:10EBE000606313B1E36B2360F8BD23691BB9214651
:10EBF0002846FFF7A9FCB4F90C70BEB2B3070FD0DA
:10EC00000123A381154B1649186806F00906FFF782
:10EC100017FC092EA78103D121462846FFF75CF98E
:10EC200022692260666A6369216A2846B047002823
:10EC300060600BDCA38917BF002243F0200343F080
:10EC400040036260A3814FF0FF30F8BD0020F8BDA3
:10EC5000341D0108541D0108741D0108981D010888
:10EC600043EB000838B50C46054618B183690BB96B
:10EC7000FFF7A2FA0E4B9C4201D16C6808E00D4BE5
:10EC80009C4201D1AC6803E00B4B9C4208BFEC688E
:10EC900021462846FFF75EFF38B96368013B636091
:10ECA00023685A1C2260187838BD4FF0FF3038BDF9
:10ECB000341D0108541D0108741D010838B5064CA7
:10ECC000002305460846236000F0C6FD431C02D120
:10ECD000236803B12B6038BDAC42012010B50C464F
:10ECE000B1F90E1000F094FD0028ABBF636DA3894D
:10ECF0001B1823F48053ACBF6365A38110BD2DE9BD
:10ED0000F0411F468B89DB0505460C46164605D5A6
:10ED100002230022B1F90E1000F00AFDA389B4F914
:10ED20000E1023F48053A38132463B462846BDE8AB
:10ED3000F04100F099BB10B50C46B1F90E1000F08F
:10ED4000F7FC431CA38915BF606523F4805343F48B
:10ED50008053A38118BFA38110BDB1F90E1000F03C
:10ED600003BC000010B50446084611468E2800F288
:10ED70002F81DFE810F038018F009100930095009B
:10ED8000970099009B009D00A100A300A700A90087
:10ED9000AB00AD002D01AF00B100B300B500B7006E
:10EDA000BD00BF00C500C700C900CB00CD00D10029
:10EDB000D500D700D900DB00DD00DF00E100E30073
:10EDC0002D012D012D012D012D012D012D012D01D3
:10EDD000E700EB002D012D012D012D012D012D014D
:10EDE0002D012D012D012D012D012D012D01ED00F4
:10EDF0000701EF00F1002D012D012D01F3002D0180
:10EE00002D012D01F5002D012D01F9002D012D0100
:10EE1000FB002D012D012D012D012D012D012D01B5
:10EE20002D012D012D01FD002D01FF000101030128
:10EE30002D012D0125012D012D012D012D012D016A
:10EE40002D012D012D011301050109010B010D01FA
:10EE50000F012D01110115011901E900C1002B015C
:10EE6000B900CF00BB009F00A5002901F7002D01CC
:10EE70001701C3001D011B012D012D012D012D01C5
:10EE80002D01D3002D012D012D01E50027011F01CA
:10EE900021012301554810BD554810BD554810BDEE
:10EEA000554810BD554810BD554810BD554810BDBA
:10EEB000554810BD554810BD554810BD554810BDAA
:10EEC000554810BD554810BD554810BD554810BD9A
:10EED000554810BD554810BD554810BD554810BD8A
:10EEE000554810BD554810BD554810BD554810BD7A
:10EEF000554810BD554810BD554810BD554810BD6A
:10EF0000554810BD554810BD554810BD554810BD59
:10EF1000554810BD554810BD554810BD554810BD49
:10EF2000554810BD554810BD554810BD554810BD39
:10EF3000554810BD554810BD554810BD554810BD29
:10EF4000554810BD554810BD554810BD554810BD19
:10EF5000554810BD554810BD554810BD554810BD09
:10EF6000554810BD554810BD554810BD554810BDF9
:10EF7000554810BD554810BD554810BD554810BDE9
:10EF8000554810BD554810BD554810BD554810BDD9
:10EF9000554810BD554810BD554810BD554810BDC9
:10EFA000554810BD554810BD554810BD554810BDB9
:10EFB000554810BD554810BD554810BD554810BDA9
:10EFC000554810BD554810BD554810BD554810BD99
:10EFD000002B14BF1A46224600F03AF9524B002883
:10EFE00008BF184610BD514810BD00BFA71D01083D
:10EFF000B11D0108CB1D0108DB1D0108F31D01082F
:10F00000FD1D0108171E0108291E01083B1E0108ED
:10F01000541E0108641E0108701E01088D1E01089F
:10F020009F1E0108B01E0108C21E0108CE1E010865
:10F03000E61E0108F21E0108041F0108131F010843
:10F04000231F0108301F01084F1F01085E1F010820
:10F050006F1F0108931F0108B11F0108CF1F01088E
:10F06000EF1F0108062001081520010824200108CF
:10F0700038200108502001085E2001086B2001089B
:10F0800081200108902001089C200108CB20010864
:10F09000DC200108F72001080A21010820210108CD
:10F0A00029210108402101084821010855210108B2
:10F0B0006A2101087E21010896210108A521010885
:10F0C000B6210108C9210108D5210108EE21010856
:10F0D000022201081D220108352201084F220108E1
:10F0E0005722010887220108A6220108C52201082B
:10F0F000DC220108EF220108082301081F23010870
:10F1000035230108562301086E2301088A230108CC
:10F110009D230108B3230108C7230108E92301083F
:10F120000F240108202401083B2501089F1D010828
:10F130002DE9F04780464048D0F800900F463D4604
:10F1400015F8014B09EB0400407800F0080000F0CE
:10F15000FF0608B12F46F2E72D2C03D1BD1C7C78A9
:10F16000012603E02B2C04BF7C78BD1C13B1102BAF
:10F170000AD15BE0302C57D1287800F0DF00582806
:10F180004DD16C7810230235002E14BF4FF0004C87
:10F190006FF0004C0027BCFBF3FA384603FB1ACC97
:10F1A00009EB040E9EF801E01EF0040F01D0303C84
:10F1B0000BE01EF0030E1BD0BEF1010F0CBF4FF091
:10F1C000370E4FF0570ECEEB0404A34210DDB7F11B
:10F1D000FF3F0AD0504506D801D1644503DC03FB4C
:10F1E0000040012701E04FF0FF3715F8014BD7E74A
:10F1F0007B1C0CD1002E4FF0220314BF4FF00040B7
:10F200006FF00040C8F800302AB9BDE8F08706B1B9
:10F21000404272B107B1691E1160BDE8F087302429
:10F22000002BB1D10823AFE70A23ADE7302CA3D0E0
:10F23000AAE7BDE8F08700BF2401002013460A4674
:10F24000014602480068FFF773BF00BF200100209D
:10F25000002070472DE9F0410C46496B04F144034E
:10F2600099421CD14FF48061FFF75CFA18B94FF056
:10F27000FF30BDE8F0814FF48063A36394F846301B
:10F28000606380F8FF3394F8453080F8FE3394F8DB
:10F29000443080F8FD3300F2FD30206012E0A66BB0
:10F2A00077003A4600F058FA05460028DFD000EB18
:10F2B0000608014632464046FFF7D2F9C4F80080FE
:10F2C0006563A7630020BDE8F0810000F8B54D1C20
:10F2D00006460F46144602D14FF0FF30F8BD18B174
:10F2E00083690BB9FEF768FF2E4B9C4201D174680D
:10F2F00008E02D4B9C4201D1B46803E02B4B9C42AB
:10F3000008BFF468B4F90C3023F02003A3819BB24A
:10F31000590713D4DA06DFD51B070BD52146304633
:10F32000FEF762FE0028D7D1A389A06023F008036E
:10F33000A381A061A38943F00403A381636B626886
:10F34000FDB28BB1A36B9A4207DA23685A1E226082
:10F3500003F8017C6368013320E021463046FFF763
:10F3600079FF0028F1D0B7E72169236851B19942AC
:10F3700008D213F8011C8D4204D1013B01322360F5
:10F3800062600CE0E36304F1440363630323A3635B
:10F390002346226403F8467F2360012363602846E6
:10F3A000F8BD00BF341D0108541D0108741D01087B
:10F3B000024B0A4601461868FFF788BF200100206B
:10F3C000F8B50F461446064618B183690BB9FEF727
:10F3D000F3FE224B9C4201D1746808E0204B9C4212
:10F3E00001D1B46803E01F4B9C4208BFF468A369D5
:10F3F000A360A3891A0709D523693BB12368206953
:10F40000181A63699842FDB20FDB08E021463046C6
:10F4100000F03CF80028F1D04FF0FF30F8BD214655
:10F420003046FEF7E1FD0028F6D1A368013BA3605A
:10F4300023685A1C22601F706269431C934204D0E7
:10F44000A389DB0707D50A2D05D121463046FEF7F3
:10F45000CBFD0028E0D12846F8BD00BF341D0108CF
:10F46000541D0108741D010838B5074C05460846AF
:10F470001146002222601A46FCF7B6FC431C02D15A
:10F48000236803B12B6038BDAC420120324B70B50C
:10F490001D6806460C4625B1AB6913B92846FEF730
:10F4A0008BFE2E4B9C4201D16C6808E02C4B9C4299
:10F4B00001D1AC6803E02B4B9C4208BFEC68B4F967
:10F4C0000C309AB215071DD4D00602D4092232603E
:10F4D0003AE0510712D5616B41B104F144039942FE
:10F4E00002D03046FFF7D0F800236363A38923F0EE
:10F4F0002403A3810023636023692360A38943F06D
:10F500000803A38123694BB9A38903F42073B3F5DE
:10F51000007F03D021463046FFF716F8A28912F08B
:10F52000010305D00023A36063695B42A36103E08C
:10F53000920758BF6369A36023695BB9B4F90C30C3
:10F5400003F0800080B230B143F04003A3814FF05C
:10F55000FF3070BD002070BD20010020341D010867
:10F56000541D0108741D010838B5064C00230546DA
:10F5700008462360FCF70AFD431C02D1236803B14F
:10F580002B6038BDAC4201200B78722B30B50ED009
:10F59000772B07D0612B0ED14FF4027401234FF467
:10F5A00084701AE04FF4C0640123082015E00024A1
:10F5B0002346042011E016230360002030BD622D95
:10F5C00010D0782D11D02B2D07D120F01C0023F066
:10F5D000030340F0100043F0020311F8015F002D17
:10F5E000EDD105E043F48033F7E743F40063F4E73B
:10F5F0002343136030BD000070B50E461446054627
:10F6000018B183690BB9FEF7D7FD0A4B9C4201D1B3
:10F610006C6808E0084B9C4201D1AC6803E0074BE2
:10F620009C4208BFEC68224631462846BDE870403F
:10F6300000F0B8B8341D0108541D0108741D0108FC
:10F64000024B0A4601461868FFF7D6BF200100208A
:10F6500070B50E461446054618B183690BB9FEF71E
:10F66000ABFD1B4B9C4201D16C6808E0194B9C42DE
:10F6700001D1AC6803E0184B9C4208BFEC68A38939
:10F680001B0701D523693BB921462846FFF7FEFE3B
:10F6900010B14FF0FF3070BD013E16F8011FA9B147
:10F6A000A368013B002BA36004DAA269934206DB46
:10F6B0000A2904D023685A1C22601970EDE72246FB
:10F6C0002846FFF77DFE0130E7D1E2E7084670BD2E
:10F6D000341D0108541D0108741D0108024B0A461F
:10F6E00001461868FFF7B4BF2001002038B5074C69
:10F6F0000023054608461146236000F0A5F8431C88
:10F7000002D1236803B12B6038BD00BFAC42012099
:10F7100038B5064C0023054608462360FCF730FB4D
:10F72000431C02D1236803B12B6038BDAC420120D9
:10F7300038B5074C054608461146002222601A4695
:10F74000FCF724FB431C02D1236803B12B6038BDB6
:10F75000AC42012070477047F8B5074615460E4683
:10F7600021B91146BDE8F840FEF7DCBF1AB9FEF733
:10F770008BFF2846F8BD00F05DF885420ED929467A
:10F780003846FEF7CFFF044650B131462A46FEF711
:10F7900067FF31463846FEF777FF01E03046F8BD97
:10F7A0002046F8BD70B50D461446064618B183696B
:10F7B0000BB9FEF701FD134B9C4201D1746808E0C0
:10F7C000114B9C4201D1B46803E0104B9C4208BF2E
:10F7D000F468A368013B002BA3600CDAA269934292
:10F7E00002DBEBB20A2B06D1224629463046BDE8A1
:10F7F0007040FFF7E5BD23685A1C22601D70E8B217
:10F8000070BD00BF341D0108541D0108741D01089E
:10F8100038B5074C054608461146002222601A46B4
:10F82000FCF76AFB431C02D1236803B12B6038BD8F
:10F83000AC42012051F8040C0028BEBF091851F851
:10F84000043CC01804387047024B58221A604FF02D
:10F85000FF307047AC420120044B1968024609B9D9
:10F8600003491960186802441A607047A8420120D1
:10F87000B0420120FEE700000EB403B5014603AB21
:10F88000054853F8042B0068019300F09DF802B07E
:10F890005DF804EB03B07047200100202DE9F84328
:10F8A000089C8946174602FB03F8064618B183698F
:10F8B0000BB9FEF781FC1D4B9C4201D1746808E036
:10F8C0001B4B9C4201D1B46803E01A4B9C4208BF19
:10F8D000F468A3891B0703D523690BB1002513E046
:10F8E00021463046FFF7D2FD0028F7D0002519E069
:10F8F000A36819F80510013B002BA36007DB236800
:10F900005A1C2260197001354545F1D10AE0A269FF
:10F91000934201DB0A29F2D122463046FFF750FD1F
:10F920000130F0D1B5FBF7F0BDE8F883341D0108D4
:10F93000541D0108741D010807B5009313460A46BB
:10F94000014603480068FFF7A9FF03B05DF804FB18
:10F950002001002010B501390244904207D010F870
:10F96000013B11F8014FA342F7D0181B10BD002036
:10F9700010BD9368013B002B10B4936009DA9469C1
:10F98000A34202DBCBB20A2B03D15DF8044BFFF795
:10F9900017BD1368581C10601970C8B25DF8044B8D
:10F9A0007047F8B506460F461446D518AC4208D045
:10F9B0003A4614F8011B3046FFF7DBFF431CF5D134
:10F9C00000E00020F8BD00002DE9F04F9DB00C468E
:10F9D00017460393064618B183690BB9FEF7ECFB93
:10F9E0007F4B9C4201D1746808E07E4B9C4201D160
:10F9F000B46803E07C4B9C4208BFF468A3891807F5
:10FA00000CD5236953B10023099320238DF82930A5
:10FA100030238DF82A30DFF8D4B144E02146304657
:10FA2000FFF734FD0028EED04FF0FF30D5E0039A09
:10FA3000111D12680391002A80F28C80524243F01B
:10FA400002000792049098F800302E2B00F084807A
:10FA5000032298F800106548FEF7B2FD48B1402334
:10FA6000CBEB000003FA00F0049B1843049008F16C
:10FA7000010898F800105E488DF82810062208F159
:10FA80000107FEF79DFD002800F09580594B002BE3
:10FA900040F08880039B073323F007030833039368
:10FAA000099B53440993B846454615F8013B1BB9D9
:10FAB000B8EB07090FD003E0252BF9D0A846F3E7F0
:10FAC0004B463A4621463046FFF76BFF01307FD068
:10FAD000099B4B44099398F80030002B78D0002301
:10FAE0004FF0FF3204930793059206938DF853303D
:10FAF0001A930127052229783F48FEF761FD05F199
:10FB00000108049B38B13C4A801A07FA00F01843F8
:10FB100004904546EEE7D90644BF20228DF85320D5
:10FB20001A0744BF2B228DF853202A782A2A3FF443
:10FB30007EAF079A00210A20A846013598F80030C8
:10FB4000303B092B03D800FB02320121F4E70029E6
:10FB50003FF479AF079276E798F801302A2B0BD162
:10FB6000039B1A1D1B680392002BB8BF4FF0FF3395
:10FB700008F1020805936BE70023059308F10100E3
:10FB800019460A258046013098F80020303A092AA3
:10FB900003D805FB01210123F4E7002B3FF458AF04
:10FBA000059155E703AB00932246144B04A9304658
:10FBB000AFF3008007E003AB009322460F4B04A98C
:10FBC000304600F093F8B0F1FF3F82467FF468AF13
:10FBD000A3895B063FF528AF09981DB0BDE8F08FFB
:10FBE000341D0108541D0108741D01083C2501083D
:10FBF000402501080000000036250108A3F900088F
:10FC00002DE9F04791461F460A698B68DDF8208090
:10FC10009342B8BF1346C9F8003091F84320064616
:10FC20000C4612B10133C9F800302368990642BF6F
:10FC3000D9F800300233C9F80030256815F0060500
:10FC400010D104F1190A07E0012352463946304623
:10FC5000C04701301AD00135E368D9F800209B1A5B
:10FC60009D42F1DB94F843302268003318BF012332
:10FC700092060FD5E1185A1C302081F84300224427
:10FC800094F8451082F84310023303E04FF0FF3040
:10FC9000BDE8F08704F1430239463046C0470130E1
:10FCA000F4D02268D9F80050E36802F00602042A72
:10FCB00008BF5D1B2269A3680CBF25EAE575002516
:10FCC0009342C4BF9B1AED184FF000091A344D45FA
:10FCD00009D00123224639463046C0470130D5D0ED
:10FCE00009F10109F3E70020BDE8F0872DE9F043B1
:10FCF00017460A7E85B06E2A984606460C460C9B2F
:10FD000001F1430E00F0AE8011D8632A22D009D849
:10FD1000002A00F0BB80582A40F0CA8081F84520B4
:10FD2000834955E0642A1ED0692A1CD0C0E0732A9A
:10FD300000F0B08009D86F2A2ED0702A40F0B88029
:10FD40000A6842F020020A603EE0752A24D0782A30
:10FD50003AD0ADE01A6801F14205111D196013682F
:10FD600084F84230A8E021681A6811F0800F02D0B0
:10FD7000111D196008E011F0400F02F10401196033
:10FD800002D0B2F9003000E01368002B3CDA2D22DB
:10FD90005B4284F8432037E021681A6811F0800F35
:10FDA00002D0111D196007E011F0400F02F10401AB
:10FDB000196001D0138800E01368227E5C496F2A25
:10FDC00014BF0A2208221BE078225A4984F84520F1
:10FDD0002268186812F0800F00F104051D6003D13D
:10FDE000550601D5038800E00368D00744BF42F000
:10FDF000200222601BB9226822F020022260102219
:10FE0000002084F8430001E049490A226568A560A2
:10FE1000002D08DB206820F0040020602BB9002DA5
:10FE20007DD175460CE0002B79D07546B3FBF2F01E
:10FE300002FB1033CB5C05F8013D03460028F5D1E9
:10FE4000082A0BD12368DA0708D5236962689A4229
:10FE5000DEBF302305F8013C05F1FF35C5EB0E038D
:10FE600023612EE008681A68496910F0800F03D0FA
:10FE7000101D1860136808E010F0400F02F1040034
:10FE80001860136801D0198000E019600023236115
:10FE9000754616E01A68111D196015686268002120
:10FEA0002846FEF78DFB08B1401B6060636804E0E4
:10FEB00004F1420584F8422001232361002384F8E1
:10FEC0004330CDF800803B4603AA21463046FFF779
:10FED00097FE013002D14FF0FF3026E023692A4619
:10FEE00039463046C0470130F5D023689B0710D50E
:10FEF000002504F1190907E001234A463946304636
:10FF0000C0470130E7D00135E368039A9B1A9D4250
:10FF1000F2DBE068039B9842B8BF184605E00B7817
:10FF200084F8423004F142058AE705B0BDE8F08369
:10FF300047250108582501080FB40A4B13B51C6862
:10FF400024B1A36913B92046FEF736F905AB049A2C
:10FF5000A16801932046FFF737FD02B0BDE81040CD
:10FF600004B070472001002070B50E46054618B158
:10FF700083690BB9FEF720F9AB69AC6813B9284661
:10FF8000FEF71AF9224B9C4201D16C6808E0214B24
:10FF90009C4201D1AC6803E01F4B9C4208BFEC6857
:10FFA000A3891B0701D523693BB921462846FFF7E2
:10FFB0006DFA10B14FF0FF3070BD013EA36816F826
:10FFC000011F013BA36091B1002B04DAA2699342A7
:10FFD00006DB0A2904D023685A1C22601970EDE759
:10FFE00022462846FFF7ECF90130E7D1E2E7002B83
:10FFF00008DA22460A212846FFF7E2F90130D9D073
:020000040801F1
:100000000A2070BD23680A205A1C2260187070BD37
:10001000341D0108541D0108741D0108024B0146DE
:100020001868FFF7A1BF00BF200100200CB430B555
:10003000164B0C1E9DB01D6804DA8B232B604FF00D
:10004000FF301EE04FF40273ADF8143014BF04F11A
:10005000FF332346049307934FF6FF7302900690F5
:10006000ADF81630209A21AB02A92846019300F082
:10007000DDF8431CBCBF8B232B6014B1029B002214
:100080001A701DB0BDE8304002B07047200100205A
:100090000D4B30B51D6810F8013BEA18527802F09C
:1000A0000302012A11F8012B05EB020408BF2033DB
:1000B000647804F00304012C08BF20329B1A01D19C
:1000C000002AE8D1184630BD24010020C9B20346F9
:1000D00010F8012B1AB19142F9D118467047002946
:1000E0000CBF18460020704710F8012B11F8013B97
:1000F000012A28BF9A42F7D0D01A7047034611F858
:10010000012B03F8012B002AF9D17047034613F89D
:10011000012B002AFBD1181A0138704710B503468D
:1001200042B111F8014B03F8014B013A002CF7D111
:100130001A4400E010BD934202D003F8014BFAE7E5
:1001400010BD884210B501EB020301D8421E0BE03E
:100150009842FBD28118D21AD34204D013F8014D31
:1001600001F8014DF8E710BD994204D011F8014B98
:1001700002F8014FF8E710BD2DE9F0478E689E4266
:1001800082460C46914698463ED88A8912F4906F72
:100190003AD0256809696F1A6569022305EB4505A0
:1001A00095FBF3F57B1C43449D4238BF1D46530528
:1001B0000FD52946FEF7B6FA064698B13A462169A8
:1001C000FEF74EFAA38923F4906343F08003A381E2
:1001D00013E02A46FFF7C0FA064670B92169504677
:1001E000FEF752FA0C23CAF80030A38943F040030B
:1001F000A3814FF0FF30BDE8F087266165613E4482
:10020000ED1B2660A5604646464528BF4646324659
:1002100049462068FFF795FFA3689B1BA3602368EE
:100220001E4426600020BDE8F08700002DE9F04F55
:100230009DB0804603938B891C060D4616460DD54E
:100240000B695BB94021FEF76DFA2860286118B987
:100250000C23C8F80030CDE040236B6100230993E4
:1002600020238DF82930DFF89CB130238DF82A3017
:1002700037463C4614F8013B1BB9B7EB060910D0D2
:1002800003E0252BF9D02746F3E74B4632462946B3
:100290004046FFF771FF013000F0A780099B4B44F7
:1002A00009933B78002B00F0A08000234FF0FF3231
:1002B00004930793059206938DF853301A93012601
:1002C000052221784E48FEF77BF9671C049B38B164
:1002D0004B4A801A06FA00F0184304903C46EFE7B8
:1002E000D90644BF20228DF853201A0744BF2B2281
:1002F0008DF8532022782A2A03D0079A00210A2059
:100300000BE0039A111D12680391002A10DA524281
:1003100043F00200079204900BE0274601343B783B
:10032000303B092B03D800FB02320121F5E701B174
:1003300007923B782E2B1ED17B782A2B0AD1039B68
:100340001A1D1B680392002BB8BF4FF0FF33023712
:10035000059310E000230593781C19460A240746EC
:1003600001303A78303A092A03D804FB01210123ED
:10037000F5E703B10591032239782248FEF720F909
:1003800040B14023CBEB000003FA00F0049B18437C
:100390000490013739781C488DF8281006227E1CFD
:1003A000FEF70EF988B1194B33B9039B073323F0DD
:1003B00007030833039314E003AB00932A46144B5E
:1003C00004A94046AFF3008007E003AB00932A4640
:1003D0000F4B04A94046FFF789FCB0F1FF3F82466E
:1003E00003D0099B5344099342E7AB895B0601D4D0
:1003F000099801E04FF0FF301DB0BDE8F08F00BF5D
:10040000362501083C2501084025010800000000B0
:1004100079010108F8B500BFF8BC08BC9E467047DA
:10042000F8B500BFF8BC08BC9E46704700001E002F
:1004300000F01EF080079E0780F79EF700001F0067
:1004400000F81FF8E007FF07E0FFFFFF72620000FF
:1004500076657273696F6E20313A20646174615FF2
:10046000636F6D707265737365643D25640A000087
:100470002E746170000000002E747A780000000075
:100480002E7A383000000000776200007A38303A67
:1004900020556E68616E646C6564206F70636F6474
:1004A000653A20253032582050433D253034580AD3
:1004B00000000000008000C0FFFFFFFF00400000C0
:1004C0000100000100010100000101000100000124
:1004D0000001010001000001010000010001010014
:1004E0000001010001000001010000010001010004
:1004F00001000001000101000001010001000001F4
:1005000000010100010000010100000100010100E3
:1005100001000001000101000001010001000001D3
:1005200001000001000101000001010001000001C3
:1005300000010100010000010100000100010100B3
:1005400000010100010000010100000100010100A3
:100550000100000100010100000101000100000193
:100560000100000100010100000101000100000183
:100570000001010001000001010000010001010073
:100580000100000100010100000101000100000163
:100590000001010001000001010000010001010053
:1005A0000001010001000001010000010001010043
:1005B0000100000100010100000101000100000133
:1005C0000D0A57656C636F6D6520746F2053544539
:1005D0004343590D0A0000005344206361726420B4
:1005E000616C7265616479206D6F756E746564000D
:1005F00053442063617264206D6F756E7465642C62
:1006000020726574727920636F756E74203D2025A9
:10061000640A00006D6F756E7400000025733A2047
:1006200000000000612068617264206572726F7260
:10063000206F6363757272656420696E20746865EB
:10064000206C6F77206C6576656C206469736B2015
:10065000492F4F206C617965720A000061737365E0
:100660007274696F6E206661696C65640A000000CF
:10067000706879736963616C206472697665206360
:10068000616E6E6F7420776F726B0A006E6F2073ED
:100690007563682066696C650A0000006E6F2073E0
:1006A0007563682066696C65206F72206469726585
:1006B00063746F72790A000070617468206E616DF6
:1006C0006520666F726D617420697320696E766152
:1006D0006C69640A000000006163636573732064E1
:1006E000656E6965642064756520746F2070726F33
:1006F0006869626974656420616363657373206F00
:1007000072206469726563746F72792066756C6CAF
:100710000A0000006163636573732064656E696538
:10072000642064756520746F2070726F68696269F7
:10073000746564206163636573730A0066696C6540
:100740002F6469726563746F7279206F626A656382
:100750007420697320696E76616C69640A00000018
:10076000706879736963616C206472697665206969
:10077000732077726974652070726F746563746535
:10078000640A00006C6F676963616C20647269764B
:1007900065206E756D62657220697320696E766181
:1007A0006C69640A00000000766F6C756D652068E6
:1007B0006173206E6F20776F726B20617265610AC2
:1007C000000000007468657265206973206E6F20F8
:1007D00076616C69642046415420766F6C756D6556
:1007E0000A000000665F6D6B667328292061626FE6
:1007F000727465642064756520746F20616E792061
:1008000070726F626C656D0A00000000636F756C3A
:1008100064206E6F74206765742061206772616E5A
:100820007420746F2061636365737320746865203E
:10083000766F6C756D652077697468696E20646584
:1008400066696E656420706572696F640A000000F5
:100850006F7065726174696F6E2069732072656A6A
:100860006563746564206163636F7264696E672099
:10087000746F207468652066696C652073686172A6
:10088000696E6720706F6C6963790A006C464E2050
:10089000776F726B696E672062756666657220633A
:1008A0006F756C64206E6F7420626520616C6C6F74
:1008B00063617465640A00006E756D626572206F15
:1008C00066206F70656E2066696C6573203E2046F9
:1008D000465F46535F4C4F434B0A0000676976659D
:1008E0006E20706172616D65746572206973206934
:1008F0006E76616C69640A00756E6B6E6F776E2040
:100900006572726F720A000034382E726F6D0000CB
:10091000720000007374656363792E696E6900006C
:100920005041544800000000524F4D004155544F73
:100930005354415254000000594553004E4F00009B
:100940004155544F4C4F4144000000004B45594223
:100950004F415244000000005053320055534200B2
:100960005A5800004F5249454E544154494F4E0089
:100970005247420043554541414141434545454960
:10098000494941414592924F4F4F5555594F554F07
:100990009C4F9E9F41494F55A5A5A6A7A8A9AAABC4
:1009A000ACADAEAFB0B1B2B3B4414141B8B9BABB6E
:1009B000BCBDBEBFC0C1C2C3C4C54141C8C9CACB0A
:1009C000CCCDCECFD1D145454549494949D9DADBCE
:1009D000DCDD49DF4FE14F4F4F4FE6E8E855555515
:1009E0005959EEEFF0F1F2F3F4F5F6F7F8F9FAFBF6
:1009F000FCFDFEFF4641543332000000222A2B2C1E
:100A00003A3B3C3D3E3F5B5D7C7F00007A38305F87
:100A1000657874643A20696E76616C6964206F70E1
:100A2000636F64653A203078253032580A00000040
:100A3000747A785F6765745F776F72643A20756E59
:100A4000657870656374656420454F460A00000050
:100A5000747A785F6765745F627974653A20756E41
:100A6000657870656374656420454F460A00000030
:100A7000747A785F726561645F626C6F636B5F74D8
:100A800061703A20756E65787065637465642045A1
:100A90004F460A00747A785F726561645F626C6FBA
:100AA000636B5F7461703A20636865636B73756D27
:100AB000206572726F720A00747A785F7265616481
:100AC0005F626C6F636B5F31303A20756E65787072
:100AD000656374656420454F460A0000747A785F48
:100AE000726561645F626C6F636B5F31323A20756F
:100AF0006E657870656374656420454F460A000032
:100B0000747A785F726561645F626C6F636B5F318A
:100B1000343A20756E657870656374656420454F5E
:100B2000460A00007061757365203D2025640A0047
:100B3000537472696E67206C656E677468203D201F
:100B400025640A00747A785F626C6F636B5F333080
:100B50003A20756E657870656374656420454F460C
:100B60000A000000746170655F6C6F61643A207503
:100B70006E6B6E6F776E20626C6F636B2069643A88
:100B8000203078253032580A00000000746170650A
:100B90005F6C6F61643A20454F46207265616368FF
:100BA00065640A00747A785F726561645F626C6F75
:100BB000636B5F31313A20756E657870656374657B
:100BC0006420454F460A0000747A785F726561645C
:100BD0005F6865616465723A20756E6578706563FB
:100BE00074656420454F460A000000005A5854615D
:100BF00070652100696E76616C696420545A5820D2
:100C00007369676E61747572650A000077726F6E42
:100C10006720456E64206F6620746578742066696D
:100C20006C65206D61726B65723A203078253032C8
:100C3000580A000000000000000000000000000052
:100C400000000000000000000000000000000000A4
:100C50000000000000000000000000000000000094
:100C60000000000000000000000000000000000084
:100C70000000000000000000000000000000000074
:100C80000000000000000000000000000000000064
:100C90000000000000000000000000000000000054
:100CA0000000000000000000000000000000000044
:100CB0000000000000000000000000000000000034
:100CC0000000000000000000000000000000000024
:100CD0000000000000000000000000000000000014
:100CE0000000000000000000000000000000000004
:100CF00000000000000000000000000000000000F4
:100D000000000000000000000000000000000000E3
:100D100000000000000000000000000000000000D3
:100D200000000000000000000000000000000000C3
:100D300000000000000000000000000000000000B3
:100D400000000000000000000000000000000000A3
:100D50000000000000000000000000000000000093
:100D60000000000000000000000000000000000083
:100D70000000000000000000000000000000000073
:100D80000000000000000000000000000000000063
:100D90000000000000000000000000000000000053
:100DA0000000000000000000000000000000000043
:100DB0000000000000000000000000000000000033
:100DC0000030787878303000303000000066666699
:100DD0002400000000000000006C6CFE6C6C6CFED7
:100DE0006C6C000030307CC0C0780C0CF8303000E7
:100DF000000000C4CC183060CC8C00000070D8D843
:100E000070FADECCDC76000000303030600000008C
:100E100000000000000C183060606030180C00000A
:100E2000006030180C0C0C183060000000000066E8
:100E30003CFF3C660000000000000018187E1818F7
:100E400000000000000000000000000038386000D2
:100E50000000000000FE0000000000000000000094
:100E60000000000038380000000002060C18306056
:100E7000C0800000007CC6CEDED6F6E6C67C000050
:100E8000001030F03030303030FC00000078CCCC36
:100E90000C183060CCFC00000078CC0C0C380C0C2A
:100EA000CC780000000C1C3C6CCCFE0C0C1E00002E
:100EB00000FCC0C0C0F80C0CCC780000003860C04A
:100EC000C0F8CCCCCC78000000FEC6C6060C1830AA
:100ED000303000000078CCCCCC78CCCCCC78000082
:100EE0000078CCCCCC7C18183070000000000038A2
:100EF00038000038380000000000003838000038A2
:100F000038183000000C183060C06030180C000039
:100F1000000000007E007E0000000000006030182D
:100F20000C060C18306000000078CC0C1830300033
:100F300030300000007CC6C6DEDEDEC0C07C0000B3
:100F4000003078CCCCCCFCCCCCCC000000FC66666D
:100F5000667C666666FC0000003C66C6C0C0C0C613
:100F6000663C000000F86C66666666666CF8000019
:100F700000FE6260647C646062FE000000FE6662E7
:100F8000647C646060F00000003C66C6C0C0CEC6F1
:100F9000663E000000CCCCCCCCFCCCCCCCCC000051
:100FA000007830303030303030780000001E0C0CCB
:100FB0000C0CCCCCCC78000000E6666C6C786C6CC9
:100FC00066E6000000F060606060626666FE000039
:100FD00000C6EEFEFED6C6C6C6C6000000C6C6E601
:100FE000F6FEDECEC6C6000000386CC6C6C6C6C653
:100FF0006C38000000FC6666667C606060F0000093
:1010000000386CC6C6C6CEDE7C0C1E0000FC6666D0
:10101000667C6C6666E600000078CCCCC07018CCAC
:10102000CC78000000FCB430303030303078000034
:1010300000CCCCCCCCCCCCCCCC78000000CCCCCC74
:10104000CCCCCCCC7830000000C6C6C6C6D6D66C98
:101050006C6C000000CCCCCC783078CCCCCC0000D0
:1010600000CCCCCCCC7830303078000000FECE986C
:1010700018306062C6FE0000003C30303030303046
:10108000303C0000000080C06030180C06020000F8
:10109000003C0C0C0C0C0C0C0C3C000010386CC60A
:1010A0000000000000000000000000000000000040
:1010B0000000FF00303018000000000000000000B9
:1010C00000000000780C7CCCCC76000000E0606072
:1010D0007C66666666DC00000000000078CCC0C05C
:1010E000CC780000001C0C0C7CCCCCCCCC76000066
:1010F0000000000078CCFCC0CC78000000386C60A8
:1011000060F8606060F000000000000076CCCCCC9D
:101110007C0CCC7800E060606C76666666E6000069
:101120000018180078181818187E0000000C0C0021
:101130003C0C0C0C0CCCCC7800E06060666C786CDD
:1011400066E600000078181818181818187E0000B5
:1011500000000000FCD6D6D6D6C600000000000075
:10116000F8CCCCCCCCCC00000000000078CCCCCCAF
:10117000CC78000000000000DC666666667C60F0EB
:101180000000000076CCCCCCCC7C0C1E0000000013
:10119000EC6E766060F000000000000078CC601813
:1011A000CC78000000002060FC6060606C380000BB
:1011B00000000000CCCCCCCCCC76000000000000BD
:1011C000CCCCCCCC7830000000000000C6C6D6D60F
:1011D0006C6C000000000000C66C38386CC6000063
:1011E00000000000666666663C0C18F00000000017
:1011F000FC8C1860C4FC0000001C303060C0603003
:10120000301C0000001818181800181818180000D2
:1012100000E03030180C183030E000000073DACEF7
:10122000000000000000000000000010386CC6C67E
:10123000FE0000000010387CFEFE7C38100000002C
:1012400024924924924924924924924900000000A2
:10125000000000000000000000000000000000008E
:10126000000000000000000000000000000000007E
:10127000000000000000000000000000000000006E
:10128000000000000000000000000000000000005E
:10129000000000000000000000000000000000004E
:1012A00000000000000000000000000018181818DE
:1012B00018F80000000000000000000000F81818F6
:1012C0001818181800000000001F1818181818180F
:1012D00018181818181F0000000000001818181817
:1012E00018FF181818181818000000000000000057
:1012F00000000000000000000000000000000000EE
:101300000000000000FF00000000000000000000DE
:1013100000000000000000000000000000000000CD
:101320000000000018181818181F18181818181896
:101330001818181818F818181818181800000000AD
:1013400000000000000000000000000000FF18186E
:10135000181818181818181818181818181818180D
:10136000000000000000000000000000000000007D
:10137000000000000000000000000000000000006D
:10138000000000000000000000000000000000005D
:10139000000000000000000000000000000000004D
:1013A000000000000000000000000000000000003D
:1013B000000000000000000000000000000000002D
:1013C00000303000303078787830000000303078ED
:1013D000CCC0C0CC783030003C66606060FC60609F
:1013E000C0FE00000000000000C67C6C7CC600004F
:1013F000CCCCCCCC78FC30FC303000000018181875
:101400001800181818180000007E63303C66663C0F
:101410000CC67E0000CC00000000000000000000B0
:10142000003844BAA2A2A2BA443800000078CCCC5A
:101430007E00FE0000000000000000003366CCCCFF
:10144000663300000000000000FC0C0C0C000000E3
:101450000000000000FC000000000000003844BA5A
:10146000AABAB2AA4438000000FC00000000000044
:1014700000000000003C6666663C000000000000C2
:1014800000003030FC303000FC00000000780C1808
:10149000307C00000000000000780C380C78000060
:1014A000000000000C1830000000000000000000E8
:1014B0000000000066666666667B60C0007FDBDB5E
:1014C000DB7B1B1B1B1B0000000000000018000042
:1014D000000000000000000000000000000030706C
:1014E0000030703030780000000000000078CCCC74
:1014F0007800FE000000000000000000CC663333DE
:1015000066CC00000063E66C78376FDBB33F030006
:101510000062E66C78306EC3860C1F00E033663CD8
:10152000F8376FDBB33F0300003030003060C0C0DD
:10153000CC7800006030003078CCCCFCCCCC000003
:101540000C18003078CCCCFCCCCC000078CC00302F
:1015500078CCCCFCCCCC000076DC003078CCCCFC59
:10156000CCCC000000CC003078CCCCFCCCCC000043
:1015700078CCCC7878CCCCFCCCCC0000003E78D8B1
:10158000D8FED8D8D8DE00000078CCCCC0C0C0CC03
:10159000CC783060603000FCC4C0F8C0C4FC0000EF
:1015A0000C1800FCC4C0F8C0C4FC000078CC00FCDF
:1015B000C4C0F8C0C4FC000000CC00FCC4C0F8C02B
:1015C000C4FC0000603000783030303030780000EB
:1015D00018300078303030303078000078CC007827
:1015E000303030303078000000CC0078303030308F
:1015F0003078000000F86C6666F666666CF80000ED
:1016000076DC00C6E6F6DECEC6C6000060300078A6
:10161000CCCCCCCCCC78000018300078CCCCCCCC66
:10162000CC78000078CC0078CCCCCCCCCC78000046
:1016300076DC0078CCCCCCCCCC78000000CC007828
:10164000CCCCCCCCCC7800000000000000C66C38BC
:101650006CC60000003A6CCED6D6D6E66CB8000058
:10166000603000CCCCCCCCCCCC780000183000CC96
:10167000CCCCCCCCCC78000078CC00CCCCCCCCCCB6
:10168000CC780000CC00CCCCCCCCCCCCCC7800003E
:10169000183000CCCCCC78303078000000F0607C82
:1016A0006666667C60F000000078CCCCD8CCCCCCF0
:1016B000F8C06000C0603000780C7CCCCC760000B4
:1016C0000C183000780C7CCCCC7600003078CC0044
:1016D000780C7CCCCC7600000076DC00780C7CCCDE
:1016E000CC76000000CCCC00780C7CCCCC76000012
:1016F000386C6C38F80C7CCCCC7600000000000014
:10170000FE1B7FD8D8EF00000000000078CCC0C0DE
:10171000CC783060C060300078CCFCC0C07C000069
:101720000C18300078CCFCC0CC7800003078CC00AD
:1017300078CCFCC0C07C000000CCCC0078CCFCC0D5
:10174000C07C00006030180078181818187E00005F
:101750000C18300078181818187E000010386C002B
:1017600078181818187E0000006C6C00781818188B
:10177000187E0000CC30D80C067EC6C6C67C0000A1
:101780000076DC00F8CCCCCCCCCC0000C0603000C3
:1017900078CCCCCCCC7800000C18300078CCCCCCF9
:1017A000CC7800003078CC0078CCCCCCCC78000061
:1017B0000076DC0078CCCCCCCC78000000CCCC001F
:1017C00078CCCCCCCC7800000000303000FC00306D
:1017D000300000000000000078CCDCECCC78000089
:1017E000C0603000CCCCCCCCCC7600000C183000E3
:1017F000CCCCCCCCCC7600003078CC00CCCCCCCCD3
:10180000CC76000000CCCC00CCCCCCCCCC7600008C
:10181000060C1800666666663C0C18F00000E06076
:101820007C66667C60F00000006666006666666640
:101830003C0C18F04E2F41002000000098000020C2
:101840001400120011001F01140159001101270199
:1018500000000000000000001C00320021002300F6
:1018600024002B003400330043003B0042004B00B7
:101870003A00310044004D0015002D001B002C00E3
:101880003C002A001D00220035001A0016001E0030
:10189000260025002E0036003D003E004600450093
:1018A0005A00760066000D0029004E00000000007E
:1018B0005B0000005D0000000000000041004900E6
:1018C0004A0000000500060004000C0003000B00A5
:1018D00083000A00010009007800070000007E0074
:1018E000000070016C0100007101690100007401C9
:1018F0006B017201750100004A017C007B007900D8
:101900005A01690072007A006B00730074006C0069
:1019100075007D00700071000000000000000000F4
:1019200000000000000000000000000000000000B7
:1019300000000000000000000000000000000000A7
:101940000000000000000000000000000000000097
:101950000000000000000000000071000000000016
:101960000000000000000000000000000000000077
:101970000000000000000000000000000000000067
:101980000000000000000000000000000000000057
:101990000000000000000000000000000000000047
:1019A0000000000000000000000000000000000037
:1019B0000000000000000000000000000000000027
:1019C0000000000000000000000000000000000017
:1019D0000000000000000000000000000000000007
:1019E00000000000000000000000000000000000F7
:1019F00000000000000000000000000000000000E7
:101A000000000000000000000000000000000000D6
:101A100000000000000000000000000000000000C6
:101A200000000000000000000000000000000000B6
:101A300000000000000000000000000000000000A6
:101A40000000000000000000000000000000000096
:101A500000FF00FF00FF00FF00FF00FF00FF00FF8E
:101A600000FF00FF00FF00FF00FF00FF00FF00FF7E
:101A700000FF00FF000000FF01710120023000FFA5
:101A800000FF00FF0154011101100121025000FF6D
:101A900000FF01030102011201220233003200FFA4
:101AA00000FF01700104011301240123023400FF2F
:101AB00000FF01730174016401140101024400FF7D
:101AC00000FF00FF0172016301530204024200FFA4
:101AD00000FF02510162015201510261024100FF07
:101AE00000FF02010240016100FF0050020300FFFD
:101AF00000FF00FF00FF00FF00FF00FF00FF00FFEE
:101B000000FF00FF0060027400FF024300FF00FFBF
:101B100000FF022400FF00FF00FF00FF014000FF64
:101B200000FF00FF00FF00FF00FF00FF00FF00FFBD
:101B300000FF00FF00FF00FF00FF00FF017000FF3B
:101B400000FF00FF00FF00FF00FF00FF00FF00FF9D
:101B500000FF00FF00FF00FF00FF00FF00FF00FF8D
:101B600000FF00FF00FF00FF00FF00FF00FF00FF7D
:101B700000FF00FF000000FF00710020003000FFA8
:101B800000FF00FF0001001100100021003100FFE4
:101B900000FF00030002001200220033003200FFA9
:101BA00000FF00700004001300240023003400FF35
:101BB00000FF00730074006400140054004400FF30
:101BC00000FF00FF0072006300530043004200FF6B
:101BD00000FF02730062005200510040004100FF0C
:101BE00000FF02720263006100FF005000FF00FF6F
:101BF00000FF00FF00FF00FF00FF00FF00FF00FFED
